Archive member included because of file (symbol)

c:/program files/codesourcery/sourcery g++ lite/bin/../lib/gcc/m68k-elf/4.4.1/m5208\libgcc.a(_float.o)
                              ./bin/main.o (__addsf3)
c:/program files/codesourcery/sourcery g++ lite/bin/../lib/gcc/m68k-elf/4.4.1/m5208\libgcc.a(_floatex.o)
                              c:/program files/codesourcery/sourcery g++ lite/bin/../lib/gcc/m68k-elf/4.4.1/m5208\libgcc.a(_float.o) (_fpCCR)
c:/program files/codesourcery/sourcery g++ lite/bin/../lib/gcc/m68k-elf/4.4.1/m5208\libgcc.a(_fixunssfsi.o)
                              ./bin/main.o (__fixunssfsi)
c:/program files/codesourcery/sourcery g++ lite/bin/../lib/gcc/m68k-elf/4.4.1/m5208\libgcc.a(fpgnulib.o)
                              ./bin/main.o (__floatunsisf)
c:/program files/codesourcery/sourcery g++ lite/bin/../lib/gcc/m68k-elf/4.4.1/m5208\libgcc.a(_gesf2.o)
                              c:/program files/codesourcery/sourcery g++ lite/bin/../lib/gcc/m68k-elf/4.4.1/m5208\libgcc.a(_fixunssfsi.o) (__gesf2)
c:/program files/codesourcery/sourcery g++ lite/bin/../lib/gcc/m68k-elf/4.4.1/../../../../m68k-elf/lib/m5208\libc.a(lib_a-atexit.o)
                              (atexit)
c:/program files/codesourcery/sourcery g++ lite/bin/../lib/gcc/m68k-elf/4.4.1/../../../../m68k-elf/lib/m5208\libc.a(lib_a-atoi.o)
                              ./bin/riadenie.o (atoi)
c:/program files/codesourcery/sourcery g++ lite/bin/../lib/gcc/m68k-elf/4.4.1/../../../../m68k-elf/lib/m5208\libc.a(lib_a-exit.o)
                              (exit)
c:/program files/codesourcery/sourcery g++ lite/bin/../lib/gcc/m68k-elf/4.4.1/../../../../m68k-elf/lib/m5208\libc.a(lib_a-impure.o)
                              c:/program files/codesourcery/sourcery g++ lite/bin/../lib/gcc/m68k-elf/4.4.1/../../../../m68k-elf/lib/m5208\libc.a(lib_a-exit.o) (_global_impure_ptr)
c:/program files/codesourcery/sourcery g++ lite/bin/../lib/gcc/m68k-elf/4.4.1/../../../../m68k-elf/lib/m5208\libc.a(lib_a-memcmp.o)
                              ./bin/tasks.o (memcmp)
c:/program files/codesourcery/sourcery g++ lite/bin/../lib/gcc/m68k-elf/4.4.1/../../../../m68k-elf/lib/m5208\libc.a(lib_a-memcpy.o)
                              ./bin/flashUtilities.o (memcpy)
c:/program files/codesourcery/sourcery g++ lite/bin/../lib/gcc/m68k-elf/4.4.1/../../../../m68k-elf/lib/m5208\libc.a(lib_a-memset.o)
                              ./bin/tasks.o (memset)
c:/program files/codesourcery/sourcery g++ lite/bin/../lib/gcc/m68k-elf/4.4.1/../../../../m68k-elf/lib/m5208\libc.a(lib_a-puts.o)
                              ./bin/psock.o (puts)
c:/program files/codesourcery/sourcery g++ lite/bin/../lib/gcc/m68k-elf/4.4.1/../../../../m68k-elf/lib/m5208\libc.a(lib_a-strcat.o)
                              ./bin/tasks.o (strcat)
c:/program files/codesourcery/sourcery g++ lite/bin/../lib/gcc/m68k-elf/4.4.1/../../../../m68k-elf/lib/m5208\libc.a(lib_a-strchr.o)
                              ./bin/httpd.o (strchr)
c:/program files/codesourcery/sourcery g++ lite/bin/../lib/gcc/m68k-elf/4.4.1/../../../../m68k-elf/lib/m5208\libc.a(lib_a-strcmp.o)
                              ./bin/riadenie.o (strcmp)
c:/program files/codesourcery/sourcery g++ lite/bin/../lib/gcc/m68k-elf/4.4.1/../../../../m68k-elf/lib/m5208\libc.a(lib_a-strcpy.o)
                              ./bin/console_reader.o (strcpy)
c:/program files/codesourcery/sourcery g++ lite/bin/../lib/gcc/m68k-elf/4.4.1/../../../../m68k-elf/lib/m5208\libc.a(lib_a-strlen.o)
                              ./bin/LCD.o (strlen)
c:/program files/codesourcery/sourcery g++ lite/bin/../lib/gcc/m68k-elf/4.4.1/../../../../m68k-elf/lib/m5208\libc.a(lib_a-strncmp.o)
                              ./bin/riadenie.o (strncmp)
c:/program files/codesourcery/sourcery g++ lite/bin/../lib/gcc/m68k-elf/4.4.1/../../../../m68k-elf/lib/m5208\libc.a(lib_a-strncpy.o)
                              ./bin/tasks.o (strncpy)
c:/program files/codesourcery/sourcery g++ lite/bin/../lib/gcc/m68k-elf/4.4.1/../../../../m68k-elf/lib/m5208\libc.a(lib_a-strrchr.o)
                              ./bin/httpd.o (strrchr)
c:/program files/codesourcery/sourcery g++ lite/bin/../lib/gcc/m68k-elf/4.4.1/../../../../m68k-elf/lib/m5208\libc.a(lib_a-strtok.o)
                              ./bin/riadenie.o (strtok)
c:/program files/codesourcery/sourcery g++ lite/bin/../lib/gcc/m68k-elf/4.4.1/../../../../m68k-elf/lib/m5208\libc.a(lib_a-strtok_r.o)
                              c:/program files/codesourcery/sourcery g++ lite/bin/../lib/gcc/m68k-elf/4.4.1/../../../../m68k-elf/lib/m5208\libc.a(lib_a-strtok.o) (__strtok_r)
c:/program files/codesourcery/sourcery g++ lite/bin/../lib/gcc/m68k-elf/4.4.1/../../../../m68k-elf/lib/m5208\libc.a(lib_a-strtol.o)
                              c:/program files/codesourcery/sourcery g++ lite/bin/../lib/gcc/m68k-elf/4.4.1/../../../../m68k-elf/lib/m5208\libc.a(lib_a-atoi.o) (_strtol_r)
c:/program files/codesourcery/sourcery g++ lite/bin/../lib/gcc/m68k-elf/4.4.1/../../../../m68k-elf/lib/m5208\libc.a(lib_a-__atexit.o)
                              c:/program files/codesourcery/sourcery g++ lite/bin/../lib/gcc/m68k-elf/4.4.1/../../../../m68k-elf/lib/m5208\libc.a(lib_a-atexit.o) (__register_exitproc)
c:/program files/codesourcery/sourcery g++ lite/bin/../lib/gcc/m68k-elf/4.4.1/../../../../m68k-elf/lib/m5208\libc.a(lib_a-__call_atexit.o)
                              c:/program files/codesourcery/sourcery g++ lite/bin/../lib/gcc/m68k-elf/4.4.1/../../../../m68k-elf/lib/m5208\libc.a(lib_a-exit.o) (__call_exitprocs)
c:/program files/codesourcery/sourcery g++ lite/bin/../lib/gcc/m68k-elf/4.4.1/../../../../m68k-elf/lib/m5208\libc.a(lib_a-ctype_.o)
                              c:/program files/codesourcery/sourcery g++ lite/bin/../lib/gcc/m68k-elf/4.4.1/../../../../m68k-elf/lib/m5208\libc.a(lib_a-strtol.o) (__ctype_ptr__)
c:/program files/codesourcery/sourcery g++ lite/bin/../lib/gcc/m68k-elf/4.4.1/../../../../m68k-elf/lib/m5208\libc.a(lib_a-fini.o)
                              c:/program files/codesourcery/sourcery g++ lite/bin/../lib/gcc/m68k-elf/4.4.1/../../../../m68k-elf/lib/m5208\libc.a(lib_a-__call_atexit.o) (__libc_fini_array)
c:/program files/codesourcery/sourcery g++ lite/bin/../lib/gcc/m68k-elf/4.4.1/../../../../m68k-elf/lib/m5208\libc.a(lib_a-fvwrite.o)
                              c:/program files/codesourcery/sourcery g++ lite/bin/../lib/gcc/m68k-elf/4.4.1/../../../../m68k-elf/lib/m5208\libc.a(lib_a-puts.o) (__sfvwrite_r)
c:/program files/codesourcery/sourcery g++ lite/bin/../lib/gcc/m68k-elf/4.4.1/../../../../m68k-elf/lib/m5208\libc.a(lib_a-mallocr.o)
                              c:/program files/codesourcery/sourcery g++ lite/bin/../lib/gcc/m68k-elf/4.4.1/../../../../m68k-elf/lib/m5208\libc.a(lib_a-fvwrite.o) (_malloc_r)
c:/program files/codesourcery/sourcery g++ lite/bin/../lib/gcc/m68k-elf/4.4.1/../../../../m68k-elf/lib/m5208\libc.a(lib_a-memchr.o)
                              c:/program files/codesourcery/sourcery g++ lite/bin/../lib/gcc/m68k-elf/4.4.1/../../../../m68k-elf/lib/m5208\libc.a(lib_a-fvwrite.o) (memchr)
c:/program files/codesourcery/sourcery g++ lite/bin/../lib/gcc/m68k-elf/4.4.1/../../../../m68k-elf/lib/m5208\libc.a(lib_a-memmove.o)
                              c:/program files/codesourcery/sourcery g++ lite/bin/../lib/gcc/m68k-elf/4.4.1/../../../../m68k-elf/lib/m5208\libc.a(lib_a-fvwrite.o) (memmove)
c:/program files/codesourcery/sourcery g++ lite/bin/../lib/gcc/m68k-elf/4.4.1/../../../../m68k-elf/lib/m5208\libc.a(lib_a-mlock.o)
                              c:/program files/codesourcery/sourcery g++ lite/bin/../lib/gcc/m68k-elf/4.4.1/../../../../m68k-elf/lib/m5208\libc.a(lib_a-mallocr.o) (__malloc_lock)
c:/program files/codesourcery/sourcery g++ lite/bin/../lib/gcc/m68k-elf/4.4.1/../../../../m68k-elf/lib/m5208\libc.a(lib_a-reallocr.o)
                              c:/program files/codesourcery/sourcery g++ lite/bin/../lib/gcc/m68k-elf/4.4.1/../../../../m68k-elf/lib/m5208\libc.a(lib_a-fvwrite.o) (_realloc_r)
c:/program files/codesourcery/sourcery g++ lite/bin/../lib/gcc/m68k-elf/4.4.1/../../../../m68k-elf/lib/m5208\libc.a(lib_a-sbrkr.o)
                              c:/program files/codesourcery/sourcery g++ lite/bin/../lib/gcc/m68k-elf/4.4.1/../../../../m68k-elf/lib/m5208\libc.a(lib_a-mallocr.o) (_sbrk_r)
c:/program files/codesourcery/sourcery g++ lite/bin/../lib/gcc/m68k-elf/4.4.1/../../../../m68k-elf/lib/m5208\libc.a(lib_a-wsetup.o)
                              c:/program files/codesourcery/sourcery g++ lite/bin/../lib/gcc/m68k-elf/4.4.1/../../../../m68k-elf/lib/m5208\libc.a(lib_a-fvwrite.o) (__swsetup_r)
c:/program files/codesourcery/sourcery g++ lite/bin/../lib/gcc/m68k-elf/4.4.1/../../../../m68k-elf/lib/m5208\libc.a(lib_a-fflush.o)
                              c:/program files/codesourcery/sourcery g++ lite/bin/../lib/gcc/m68k-elf/4.4.1/../../../../m68k-elf/lib/m5208\libc.a(lib_a-fvwrite.o) (_fflush_r)
c:/program files/codesourcery/sourcery g++ lite/bin/../lib/gcc/m68k-elf/4.4.1/../../../../m68k-elf/lib/m5208\libc.a(lib_a-findfp.o)
                              c:/program files/codesourcery/sourcery g++ lite/bin/../lib/gcc/m68k-elf/4.4.1/../../../../m68k-elf/lib/m5208\libc.a(lib_a-wsetup.o) (__sinit)
c:/program files/codesourcery/sourcery g++ lite/bin/../lib/gcc/m68k-elf/4.4.1/../../../../m68k-elf/lib/m5208\libc.a(lib_a-freer.o)
                              c:/program files/codesourcery/sourcery g++ lite/bin/../lib/gcc/m68k-elf/4.4.1/../../../../m68k-elf/lib/m5208\libc.a(lib_a-fvwrite.o) (_free_r)
c:/program files/codesourcery/sourcery g++ lite/bin/../lib/gcc/m68k-elf/4.4.1/../../../../m68k-elf/lib/m5208\libc.a(lib_a-fwalk.o)
                              c:/program files/codesourcery/sourcery g++ lite/bin/../lib/gcc/m68k-elf/4.4.1/../../../../m68k-elf/lib/m5208\libc.a(lib_a-findfp.o) (_fwalk)
c:/program files/codesourcery/sourcery g++ lite/bin/../lib/gcc/m68k-elf/4.4.1/../../../../m68k-elf/lib/m5208\libc.a(lib_a-makebuf.o)
                              c:/program files/codesourcery/sourcery g++ lite/bin/../lib/gcc/m68k-elf/4.4.1/../../../../m68k-elf/lib/m5208\libc.a(lib_a-wsetup.o) (__smakebuf_r)
c:/program files/codesourcery/sourcery g++ lite/bin/../lib/gcc/m68k-elf/4.4.1/../../../../m68k-elf/lib/m5208\libc.a(lib_a-reent.o)
                              c:/program files/codesourcery/sourcery g++ lite/bin/../lib/gcc/m68k-elf/4.4.1/../../../../m68k-elf/lib/m5208\libc.a(lib_a-sbrkr.o) (errno)
c:/program files/codesourcery/sourcery g++ lite/bin/../lib/gcc/m68k-elf/4.4.1/../../../../m68k-elf/lib/m5208\libc.a(lib_a-stdio.o)
                              c:/program files/codesourcery/sourcery g++ lite/bin/../lib/gcc/m68k-elf/4.4.1/../../../../m68k-elf/lib/m5208\libc.a(lib_a-findfp.o) (__sclose)
c:/program files/codesourcery/sourcery g++ lite/bin/../lib/gcc/m68k-elf/4.4.1/../../../../m68k-elf/lib/m5208\libc.a(lib_a-writer.o)
                              c:/program files/codesourcery/sourcery g++ lite/bin/../lib/gcc/m68k-elf/4.4.1/../../../../m68k-elf/lib/m5208\libc.a(lib_a-stdio.o) (_write_r)
c:/program files/codesourcery/sourcery g++ lite/bin/../lib/gcc/m68k-elf/4.4.1/../../../../m68k-elf/lib/m5208\libc.a(lib_a-closer.o)
                              c:/program files/codesourcery/sourcery g++ lite/bin/../lib/gcc/m68k-elf/4.4.1/../../../../m68k-elf/lib/m5208\libc.a(lib_a-stdio.o) (_close_r)
c:/program files/codesourcery/sourcery g++ lite/bin/../lib/gcc/m68k-elf/4.4.1/../../../../m68k-elf/lib/m5208\libc.a(lib_a-fclose.o)
                              c:/program files/codesourcery/sourcery g++ lite/bin/../lib/gcc/m68k-elf/4.4.1/../../../../m68k-elf/lib/m5208\libc.a(lib_a-findfp.o) (fclose)
c:/program files/codesourcery/sourcery g++ lite/bin/../lib/gcc/m68k-elf/4.4.1/../../../../m68k-elf/lib/m5208\libc.a(lib_a-fstatr.o)
                              c:/program files/codesourcery/sourcery g++ lite/bin/../lib/gcc/m68k-elf/4.4.1/../../../../m68k-elf/lib/m5208\libc.a(lib_a-makebuf.o) (_fstat_r)
c:/program files/codesourcery/sourcery g++ lite/bin/../lib/gcc/m68k-elf/4.4.1/../../../../m68k-elf/lib/m5208\libc.a(lib_a-isattyr.o)
                              c:/program files/codesourcery/sourcery g++ lite/bin/../lib/gcc/m68k-elf/4.4.1/../../../../m68k-elf/lib/m5208\libc.a(lib_a-makebuf.o) (_isatty_r)
c:/program files/codesourcery/sourcery g++ lite/bin/../lib/gcc/m68k-elf/4.4.1/../../../../m68k-elf/lib/m5208\libc.a(lib_a-lseekr.o)
                              c:/program files/codesourcery/sourcery g++ lite/bin/../lib/gcc/m68k-elf/4.4.1/../../../../m68k-elf/lib/m5208\libc.a(lib_a-stdio.o) (_lseek_r)
c:/program files/codesourcery/sourcery g++ lite/bin/../lib/gcc/m68k-elf/4.4.1/../../../../m68k-elf/lib/m5208\libc.a(lib_a-readr.o)
                              c:/program files/codesourcery/sourcery g++ lite/bin/../lib/gcc/m68k-elf/4.4.1/../../../../m68k-elf/lib/m5208\libc.a(lib_a-stdio.o) (_read_r)
c:/program files/codesourcery/sourcery g++ lite/bin/../lib/gcc/m68k-elf/4.4.1/../../../../m68k-elf/lib/m5208\libcs3.a(start_c.o)
                              (__cs3_start_c)
c:/program files/codesourcery/sourcery g++ lite/bin/../lib/gcc/m68k-elf/4.4.1/../../../../m68k-elf/lib/m5208\libcs3.a(m52235evb-reset.o)
                              (__cs3_reset_m52235evb)
c:/program files/codesourcery/sourcery g++ lite/bin/../lib/gcc/m68k-elf/4.4.1/../../../../m68k-elf/lib/m5208\libcs3hosted.a(hosted-_exit.o)
                              c:/program files/codesourcery/sourcery g++ lite/bin/../lib/gcc/m68k-elf/4.4.1/../../../../m68k-elf/lib/m5208\libc.a(lib_a-exit.o) (_exit)
c:/program files/codesourcery/sourcery g++ lite/bin/../lib/gcc/m68k-elf/4.4.1/../../../../m68k-elf/lib/m5208\libcs3hosted.a(hosted-close.o)
                              c:/program files/codesourcery/sourcery g++ lite/bin/../lib/gcc/m68k-elf/4.4.1/../../../../m68k-elf/lib/m5208\libc.a(lib_a-closer.o) (close)
c:/program files/codesourcery/sourcery g++ lite/bin/../lib/gcc/m68k-elf/4.4.1/../../../../m68k-elf/lib/m5208\libcs3hosted.a(hosted-fstat.o)
                              c:/program files/codesourcery/sourcery g++ lite/bin/../lib/gcc/m68k-elf/4.4.1/../../../../m68k-elf/lib/m5208\libc.a(lib_a-fstatr.o) (fstat)
c:/program files/codesourcery/sourcery g++ lite/bin/../lib/gcc/m68k-elf/4.4.1/../../../../m68k-elf/lib/m5208\libcs3hosted.a(hosted-isatty.o)
                              c:/program files/codesourcery/sourcery g++ lite/bin/../lib/gcc/m68k-elf/4.4.1/../../../../m68k-elf/lib/m5208\libc.a(lib_a-isattyr.o) (isatty)
c:/program files/codesourcery/sourcery g++ lite/bin/../lib/gcc/m68k-elf/4.4.1/../../../../m68k-elf/lib/m5208\libcs3hosted.a(hosted-lseek.o)
                              c:/program files/codesourcery/sourcery g++ lite/bin/../lib/gcc/m68k-elf/4.4.1/../../../../m68k-elf/lib/m5208\libc.a(lib_a-lseekr.o) (lseek)
c:/program files/codesourcery/sourcery g++ lite/bin/../lib/gcc/m68k-elf/4.4.1/../../../../m68k-elf/lib/m5208\libcs3hosted.a(hosted-read.o)
                              c:/program files/codesourcery/sourcery g++ lite/bin/../lib/gcc/m68k-elf/4.4.1/../../../../m68k-elf/lib/m5208\libc.a(lib_a-readr.o) (read)
c:/program files/codesourcery/sourcery g++ lite/bin/../lib/gcc/m68k-elf/4.4.1/../../../../m68k-elf/lib/m5208\libcs3hosted.a(hosted-sbrk.o)
                              c:/program files/codesourcery/sourcery g++ lite/bin/../lib/gcc/m68k-elf/4.4.1/../../../../m68k-elf/lib/m5208\libc.a(lib_a-sbrkr.o) (sbrk)
c:/program files/codesourcery/sourcery g++ lite/bin/../lib/gcc/m68k-elf/4.4.1/../../../../m68k-elf/lib/m5208\libcs3hosted.a(hosted-gdb.o)
                              c:/program files/codesourcery/sourcery g++ lite/bin/../lib/gcc/m68k-elf/4.4.1/../../../../m68k-elf/lib/m5208\libcs3hosted.a(hosted-lseek.o) (__cs3_hosted_to_gdb_lseek_flags)
c:/program files/codesourcery/sourcery g++ lite/bin/../lib/gcc/m68k-elf/4.4.1/../../../../m68k-elf/lib/m5208\libcs3hosted.a(hosted-start.o)
                              (_start)
c:/program files/codesourcery/sourcery g++ lite/bin/../lib/gcc/m68k-elf/4.4.1/../../../../m68k-elf/lib/m5208\libcs3coldfire.a(coldfire-vector.o)
                              (__cs3_interrupt_vector_coldfire)
c:/program files/codesourcery/sourcery g++ lite/bin/../lib/gcc/m68k-elf/4.4.1/../../../../m68k-elf/lib/m5208\libcs3coldfire.a(coldfire_isr_other_interrupt.o)
                              (__cs3_isr_interrupt_6)
c:/program files/codesourcery/sourcery g++ lite/bin/../lib/gcc/m68k-elf/4.4.1/../../../../m68k-elf/lib/m5208\libcs3coldfire.a(coldfire_isr_unimplemented_opcode.o)
                              (__cs3_isr_unimplemented_line_a_opcode)
c:/program files/codesourcery/sourcery g++ lite/bin/../lib/gcc/m68k-elf/4.4.1/../../../../m68k-elf/lib/m5208\libcs3coldfire.a(coldfire_isr_breakpoint_debug_interrupt.o)
                              (__cs3_isr_non_pc_breakpoint_debug_interrupt)
c:/program files/codesourcery/sourcery g++ lite/bin/../lib/gcc/m68k-elf/4.4.1/../../../../m68k-elf/lib/m5208\libcs3coldfire.a(coldfire_isr_trap_interrupt.o)
                              (__cs3_isr_trap0)
c:/program files/codesourcery/sourcery g++ lite/bin/../lib/gcc/m68k-elf/4.4.1/../../../../m68k-elf/lib/m5208\libcs3coldfire.a(coldfire_isr_fp_interrupt.o)
                              (__cs3_isr_fp_branch_unordered)
c:/program files/codesourcery/sourcery g++ lite/bin/../lib/gcc/m68k-elf/4.4.1/../../../../m68k-elf/lib/m5208\libcs3coldfire.a(coldfire_isr_access_error.o)
                              (__cs3_isr_access_error)
c:/program files/codesourcery/sourcery g++ lite/bin/../lib/gcc/m68k-elf/4.4.1/../../../../m68k-elf/lib/m5208\libcs3coldfire.a(coldfire_isr_address_error.o)
                              (__cs3_isr_address_error)
c:/program files/codesourcery/sourcery g++ lite/bin/../lib/gcc/m68k-elf/4.4.1/../../../../m68k-elf/lib/m5208\libcs3coldfire.a(coldfire_isr_illegal_instruction.o)
                              (__cs3_isr_illegal_instruction)
c:/program files/codesourcery/sourcery g++ lite/bin/../lib/gcc/m68k-elf/4.4.1/../../../../m68k-elf/lib/m5208\libcs3coldfire.a(coldfire_isr_divide_by_zero.o)
                              (__cs3_isr_divide_by_zero)
c:/program files/codesourcery/sourcery g++ lite/bin/../lib/gcc/m68k-elf/4.4.1/../../../../m68k-elf/lib/m5208\libcs3coldfire.a(coldfire_isr_privilege_violation.o)
                              (__cs3_isr_privilege_violation)
c:/program files/codesourcery/sourcery g++ lite/bin/../lib/gcc/m68k-elf/4.4.1/../../../../m68k-elf/lib/m5208\libcs3coldfire.a(coldfire_isr_trace.o)
                              (__cs3_isr_trace)
c:/program files/codesourcery/sourcery g++ lite/bin/../lib/gcc/m68k-elf/4.4.1/../../../../m68k-elf/lib/m5208\libcs3coldfire.a(coldfire_isr_format_error.o)
                              (__cs3_isr_format_error)
c:/program files/codesourcery/sourcery g++ lite/bin/../lib/gcc/m68k-elf/4.4.1/../../../../m68k-elf/lib/m5208\libcs3coldfire.a(coldfire_isr_spurious_interrupt.o)
                              (__cs3_isr_spurious_interrupt)
c:/program files/codesourcery/sourcery g++ lite/bin/../lib/gcc/m68k-elf/4.4.1/../../../../m68k-elf/lib/m5208\libcs3coldfire.a(coldfire_isr_unsupported_instruction.o)
                              (__cs3_isr_unsupported_instruction)
c:/program files/codesourcery/sourcery g++ lite/bin/../lib/gcc/m68k-elf/4.4.1/../../../../m68k-elf/lib/m5208\libc.a(lib_a-errno.o)
                              c:/program files/codesourcery/sourcery g++ lite/bin/../lib/gcc/m68k-elf/4.4.1/../../../../m68k-elf/lib/m5208\libcs3hosted.a(hosted-close.o) (__errno)
c:/program files/codesourcery/sourcery g++ lite/bin/../lib/gcc/m68k-elf/4.4.1/../../../../m68k-elf/lib/m5208\libc.a(lib_a-init.o)
                              c:/program files/codesourcery/sourcery g++ lite/bin/../lib/gcc/m68k-elf/4.4.1/../../../../m68k-elf/lib/m5208\libcs3.a(start_c.o) (__libc_init_array)
c:/program files/codesourcery/sourcery g++ lite/bin/../lib/gcc/m68k-elf/4.4.1/../../../../m68k-elf/lib/m5208\libcs3.a(heap.o)
                              c:/program files/codesourcery/sourcery g++ lite/bin/../lib/gcc/m68k-elf/4.4.1/../../../../m68k-elf/lib/m5208\libcs3hosted.a(hosted-sbrk.o) (__cs3_heap_limit)

Allocating common symbols
Common symbol       size              file

xTimeLast           0x4               ./bin/klavesnica.o
cam_data_Length     0x4               ./bin/webcam.o
uip_len             0x2               ./bin/uip.o
uart2_InpLen        0x2               ./bin/uart2.o
cam_podmienka       0x1               ./bin/main.o
errno               0x4               c:/program files/codesourcery/sourcery g++ lite/bin/../lib/gcc/m68k-elf/4.4.1/../../../../m68k-elf/lib/m5208\libc.a(lib_a-reent.o)
pcStatus            0x4               ./bin/httpd-cgi.o
komOutSocketbuffer  0x64              ./bin/main.o
xHighPriorityTask   0x4               ./bin/QPeek.o
uip_sappdata        0x4               ./bin/uip.o
casovacQueue        0x4               ./bin/main.o
uip_acc32           0x4               ./bin/uip.o
xMediumPriorityTask
                    0x4               ./bin/QPeek.o
CamPictureMutex     0x4               ./bin/main.o
command             0x6               ./bin/webcam.o
xQueueRegistry      0x50              ./bin/queue.o
uip_flags           0x1               ./bin/uip.o
uart0_InpLen        0x2               ./bin/uart0.o
uart1_Mutex         0xc               ./bin/main.o
komOutSocketQueue   0x4               ./bin/main.o
uart1_OutLen        0x2               ./bin/uart1.o
uart1_InpLen        0x2               ./bin/uart1.o
uip_appdata         0x4               ./bin/uip.o
uip_conn            0x4               ./bin/uip.o
pripojenie          0x4               ./bin/main.o
uip_conns           0x1680            ./bin/uip.o
uart2_Mutex         0xc               ./bin/main.o
xHighestPriorityTask
                    0x4               ./bin/QPeek.o
klavesnicaGetKeyMutex
                    0x4               ./bin/main.o
kom_podmienka       0x1               ./bin/main.o
uip_listenports     0xa               ./bin/uip.o
uip_draddr          0x4               ./bin/uip.o
uip_stat            0x2c              ./bin/uip.o
uip_surglen         0x2               ./bin/uip.o
uart0_OutLen        0x2               ./bin/uart0.o
uart2_OutLen        0x2               ./bin/uart2.o
rxfifo              0x80              ./bin/webcam.o
temp_velkost        0x4               ./bin/console_reader.o
komInSocketQueue    0x4               ./bin/main.o
uart0_Mutex         0xc               ./bin/main.o
uip_urgdata         0x4               ./bin/uip.o
uip_netmask         0x4               ./bin/uip.o
uip_hostaddr        0x4               ./bin/uip.o
uip_urglen          0x2               ./bin/uip.o
uip_buf             0x4               ./bin/FEC.o
uip_slen            0x2               ./bin/uip.o

Memory Configuration

Name             Origin             Length             Attributes
ram              0x20000000         0x00008000         rw
vectorrom        0x00000000         0x00000400         xr
cfmprotrom       0x00000400         0x00000020         xr
rom              0x00000420         0x0003fbe0         xr
variable0        0x00035801         0x00007ffc         xr
variable1        0x00036000         0x00007ffc         xr
ipsbar           0x40000000         0x00200000         rw
*default*        0x00000000         0xffffffff

Linker script and memory map

LOAD ./bin/main.o
LOAD ./bin/uart0.o
LOAD ./bin/uart1.o
LOAD ./bin/uart2.o
LOAD ./bin/LCD.o
LOAD ./bin/klavesnica.o
LOAD ./bin/flashUtilities.o
LOAD ./bin/riadenie.o
LOAD ./bin/webcam.o
LOAD ./bin/kom_modul.o
LOAD ./bin/rfid_reader.o
LOAD ./bin/ParTest.o
LOAD ./bin/flash.o
LOAD ./bin/FreeRTOS_Tick_Setup.o
LOAD ./bin/PollQ.o
LOAD ./bin/semtest.o
LOAD ./bin/GenQTest.o
LOAD ./bin/QPeek.o
LOAD ./bin/FEC.o
LOAD ./bin/blocktim.o
LOAD ./bin/recmutex.o
LOAD ./bin/console_reader.o
LOAD ./bin/printf-stdarg.o
LOAD ./bin/portasm.o
LOAD ./bin/port.o
LOAD ./bin/list.o
LOAD ./bin/tasks.o
LOAD ./bin/queue.o
LOAD ./bin/heap_1.o
LOAD ./bin/timer.o
LOAD ./bin/uip.o
LOAD ./bin/uip_arp.o
LOAD ./bin/uiplib.o
LOAD ./bin/uip-split.o
LOAD ./bin/psock.o
LOAD ./bin/uIP_Task.o
LOAD ./bin/httpd.o
LOAD ./bin/httpd-cgi.o
LOAD ./bin/httpd-fs.o
LOAD ./bin/http-strings.o
LOAD c:/program files/codesourcery/sourcery g++ lite/bin/../lib/gcc/m68k-elf/4.4.1/m5208\libgcc.a
LOAD c:/program files/codesourcery/sourcery g++ lite/bin/../lib/gcc/m68k-elf/4.4.1/../../../../m68k-elf/lib/m5208\libc.a
LOAD c:/program files/codesourcery/sourcery g++ lite/bin/../lib/gcc/m68k-elf/4.4.1/m5208\libgcc.a
START GROUP
LOAD c:/program files/codesourcery/sourcery g++ lite/bin/../lib/gcc/m68k-elf/4.4.1/m5208\libgcc.a
LOAD c:/program files/codesourcery/sourcery g++ lite/bin/../lib/gcc/m68k-elf/4.4.1/../../../../m68k-elf/lib/m5208\libc.a
LOAD c:/program files/codesourcery/sourcery g++ lite/bin/../lib/gcc/m68k-elf/4.4.1/../../../../m68k-elf/lib/m5208\libcs3.a
LOAD c:/program files/codesourcery/sourcery g++ lite/bin/../lib/gcc/m68k-elf/4.4.1/../../../../m68k-elf/lib/m5208\libcs3hosted.a
LOAD c:/program files/codesourcery/sourcery g++ lite/bin/../lib/gcc/m68k-elf/4.4.1/../../../../m68k-elf/lib/m5208\libcs3coldfire.a
END GROUP
                0x200065f8                PROVIDE (__cs3_heap_start, _end)
                0x20008000                PROVIDE (__cs3_heap_end, (__cs3_region_start_ram + __cs3_region_size_ram))
                0x00000001                PROVIDE (__cs3_region_num, ((__cs3_regions_end - __cs3_regions) / 0x14))
                0x20008000                PROVIDE (__cs3_stack, (__cs3_region_start_ram + __cs3_region_size_ram))

.vectors_table  0x00000000      0x400
 CREATE_OBJECT_SYMBOLS
                0x00000000                __cs3_region_start_rom = .
 *(.cs3.region-head.rom)
                0x00000001                ASSERT ((. == __cs3_region_start_rom), .cs3.region-head.rom not permitted)
                0x00000000                __cs3_interrupt_vector = __cs3_interrupt_vector_coldfire
 *(.cs3.interrupt_vector)
 .cs3.interrupt_vector
                0x00000000      0x400 c:/program files/codesourcery/sourcery g++ lite/bin/../lib/gcc/m68k-elf/4.4.1/../../../../m68k-elf/lib/m5208\libcs3coldfire.a(coldfire-vector.o)
                0x00000000                __cs3_interrupt_vector_coldfire
                0x00000001                ASSERT ((. != __cs3_interrupt_vector_coldfire), No interrupt vector)

.cfmprotect     0x00000400       0x18
 *(.cfmconfig)
 .cfmconfig     0x00000400       0x18 ./bin/main.o
                0x00000418                . = ALIGN (0x4)

.cfmvariable0   0x00035801        0xf
 *(.cfmvarTemp)
 .cfmvarTemp    0x00035801        0xc ./bin/flashUtilities.o
                0x00035801                Settings2
                0x00035810                . = ALIGN (0x4)
 *fill*         0x0003580d        0x3 00

.cfmvariable1   0x00036000        0xc
 *(.cfmvar)
 .cfmvar        0x00036000        0xc ./bin/flashUtilities.o
                0x00036000                Settings
                0x0003600c                . = ALIGN (0x4)

.text           0x00000420    0x155e4
                0x000158d0                PROVIDE (__cs3_reset_m52235evb, _start)
                0x00000420                __cs3_reset = __cs3_reset_m52235evb
 *(.cs3.reset)
 .cs3.reset     0x00000420       0x22 c:/program files/codesourcery/sourcery g++ lite/bin/../lib/gcc/m68k-elf/4.4.1/../../../../m68k-elf/lib/m5208\libcs3.a(m52235evb-reset.o)
                0x00000420                __cs3_reset_m52235evb
 *(.text .text.* .gnu.linkonce.t.*)
 *fill*         0x00000442        0x2 00
 .text          0x00000444        0x0 ./bin/main.o
 .text.outbyte  0x00000444       0x20 ./bin/main.o
 .text.main     0x00000464      0x13a ./bin/main.o
                0x00000464                main
 .text.init_eport
                0x0000059e       0x48 ./bin/main.o
 .text.init_uarts
                0x000005e6       0x88 ./bin/main.o
 .text.init_interrupt_controller
                0x0000066e      0x2b2 ./bin/main.o
 .text.ulGetErrorCode
                0x00000920        0xe ./bin/main.o
                0x00000920                ulGetErrorCode
 .text.prvSetupHardware
                0x0000092e       0x7e ./bin/main.o
 .text.vApplicationIdleHook
                0x000009ac      0x10a ./bin/main.o
                0x000009ac                vApplicationIdleHook
 .text.vApplicationStackOverflowHook
                0x00000ab6       0x5c ./bin/main.o
                0x00000ab6                vApplicationStackOverflowHook
 .text.vRegTest1Task
                0x00000b12       0xfc ./bin/main.o
 .text.vRegTest2Task
                0x00000c0e       0xfc ./bin/main.o
 .text.init_pin_assignments
                0x00000d0a       0xac ./bin/main.o
 *fill*         0x00000db6        0x2 00
 .text          0x00000db8        0x0 ./bin/uart0.o
 .text.HWEnDi   0x00000db8       0x6e ./bin/uart0.o
 .text.uart0_Enable
                0x00000e26       0x22 ./bin/uart0.o
                0x00000e26                uart0_Enable
 .text.uart0_Disable
                0x00000e48       0x22 ./bin/uart0.o
                0x00000e48                uart0_Disable
 .text.uart0_RecvChar
                0x00000e6a       0xac ./bin/uart0.o
                0x00000e6a                uart0_RecvChar
 .text.uart0_SendChar
                0x00000f16       0x94 ./bin/uart0.o
                0x00000f16                uart0_SendChar
 .text.uart0_RecvBlock
                0x00000faa       0x98 ./bin/uart0.o
                0x00000faa                uart0_RecvBlock
 .text.uart0_InterruptRx
                0x00001042       0xa0 ./bin/uart0.o
 .text.uart0_InterruptTx
                0x000010e2       0xfc ./bin/uart0.o
 .text.__cs3_isr_interrupt_77
                0x000011de       0xcc ./bin/uart0.o
                0x000011de                __cs3_isr_interrupt_77
 .text.uart0_Init
                0x000012aa       0xe8 ./bin/uart0.o
                0x000012aa                uart0_Init
 .text.uart0_OnTxChar
                0x00001392        0x8 ./bin/uart0.o
                0x00001392                uart0_OnTxChar
 .text.uart0_OnRxChar
                0x0000139a       0x42 ./bin/uart0.o
                0x0000139a                uart0_OnRxChar
 .text.uart0_OnFreeTxBuf
                0x000013dc        0x8 ./bin/uart0.o
                0x000013dc                uart0_OnFreeTxBuf
 .text.uart0_SendCharCritical
                0x000013e4       0x3c ./bin/uart0.o
                0x000013e4                uart0_SendCharCritical
 .text.critical_ERROR_WRITE
                0x00001420       0x4e ./bin/uart0.o
                0x00001420                critical_ERROR_WRITE
 *fill*         0x0000146e        0x2 00
 .text          0x00001470        0x0 ./bin/uart1.o
 .text.HWEnDi_uart1
                0x00001470       0x20 ./bin/uart1.o
 .text.uart1_RecvChar
                0x00001490       0xac ./bin/uart1.o
                0x00001490                uart1_RecvChar
 .text.uart1_RecvBlock
                0x0000153c       0x98 ./bin/uart1.o
                0x0000153c                uart1_RecvBlock
 .text.uart1_ClearRxBuf
                0x000015d4       0x36 ./bin/uart1.o
                0x000015d4                uart1_ClearRxBuf
 .text.uart1_ClearTxBuf
                0x0000160a       0x36 ./bin/uart1.o
                0x0000160a                uart1_ClearTxBuf
 .text.uart1_SendChar
                0x00001640       0x94 ./bin/uart1.o
                0x00001640                uart1_SendChar
 .text.uart1_InterruptRx
                0x000016d4       0x9e ./bin/uart1.o
 .text.uart1_InterruptTx
                0x00001772       0xfc ./bin/uart1.o
 .text.__cs3_isr_interrupt_78
                0x0000186e       0xcc ./bin/uart1.o
                0x0000186e                __cs3_isr_interrupt_78
 .text.uart1_Init
                0x0000193a       0xe0 ./bin/uart1.o
                0x0000193a                uart1_Init
 .text.uart1_OnTxChar
                0x00001a1a        0x8 ./bin/uart1.o
                0x00001a1a                uart1_OnTxChar
 .text.uart1_OnRxChar
                0x00001a22       0x42 ./bin/uart1.o
                0x00001a22                uart1_OnRxChar
 .text.uart1_OnFreeTxBuf
                0x00001a64        0x8 ./bin/uart1.o
                0x00001a64                uart1_OnFreeTxBuf
 .text.uart1_SendCharCritical
                0x00001a6c       0x3c ./bin/uart1.o
                0x00001a6c                uart1_SendCharCritical
 .text.critical_ERROR_WRITE_uart1
                0x00001aa8       0x4e ./bin/uart1.o
                0x00001aa8                critical_ERROR_WRITE_uart1
 *fill*         0x00001af6        0x2 00
 .text          0x00001af8        0x0 ./bin/uart2.o
 .text.HWEnDi_uart2
                0x00001af8       0x20 ./bin/uart2.o
 .text.uart2_RecvChar
                0x00001b18       0xac ./bin/uart2.o
                0x00001b18                uart2_RecvChar
 .text.uart2_RecvBlock
                0x00001bc4       0x98 ./bin/uart2.o
                0x00001bc4                uart2_RecvBlock
 .text.uart2_ClearRxBuf
                0x00001c5c       0x36 ./bin/uart2.o
                0x00001c5c                uart2_ClearRxBuf
 .text.uart2_ClearTxBuf
                0x00001c92       0x36 ./bin/uart2.o
                0x00001c92                uart2_ClearTxBuf
 .text.uart2_SendChar
                0x00001cc8       0x94 ./bin/uart2.o
                0x00001cc8                uart2_SendChar
 .text.uart2_InterruptRx
                0x00001d5c       0x9e ./bin/uart2.o
 .text.uart2_InterruptTx
                0x00001dfa       0xfc ./bin/uart2.o
 .text.__cs3_isr_interrupt_79
                0x00001ef6       0xcc ./bin/uart2.o
                0x00001ef6                __cs3_isr_interrupt_79
 .text.uart2_Init
                0x00001fc2       0xe0 ./bin/uart2.o
                0x00001fc2                uart2_Init
 .text.uart2_OnTxChar
                0x000020a2        0x8 ./bin/uart2.o
                0x000020a2                uart2_OnTxChar
 .text.uart2_OnRxChar
                0x000020aa       0x42 ./bin/uart2.o
                0x000020aa                uart2_OnRxChar
 .text.uart2_OnFreeTxBuf
                0x000020ec        0x8 ./bin/uart2.o
                0x000020ec                uart2_OnFreeTxBuf
 .text.uart2_SendCharCritical
                0x000020f4       0x3c ./bin/uart2.o
                0x000020f4                uart2_SendCharCritical
 .text.critical_ERROR_WRITE_uart2
                0x00002130       0x4e ./bin/uart2.o
                0x00002130                critical_ERROR_WRITE_uart2
 *fill*         0x0000217e        0x2 00
 .text          0x00002180        0x0 ./bin/LCD.o
 .text.E_PutVal
                0x00002180       0x30 ./bin/LCD.o
                0x00002180                E_PutVal
 .text.RS_PutVal
                0x000021b0       0x30 ./bin/LCD.o
                0x000021b0                RS_PutVal
 .text.RW_PutVal
                0x000021e0       0x30 ./bin/LCD.o
                0x000021e0                RW_PutVal
 .text.LCD_DATA_GetMsk
                0x00002210       0x32 ./bin/LCD.o
 .text.LCD_DATA_GetVal
                0x00002242       0x46 ./bin/LCD.o
                0x00002242                LCD_DATA_GetVal
 .text.LCD_DATA_PutVal
                0x00002288       0x44 ./bin/LCD.o
                0x00002288                LCD_DATA_PutVal
 .text.LCD_DATA_GetBit
                0x000022cc       0x8a ./bin/LCD.o
                0x000022cc                LCD_DATA_GetBit
 .text.LCD_DATA_PutBit
                0x00002356       0x52 ./bin/LCD.o
                0x00002356                LCD_DATA_PutBit
 .text.LCD_DATA_ClrBit
                0x000023a8       0x36 ./bin/LCD.o
                0x000023a8                LCD_DATA_ClrBit
 .text.LCD_DATA_SetBit
                0x000023de       0x30 ./bin/LCD.o
                0x000023de                LCD_DATA_SetBit
 .text.LCD_DATA_NegBit
                0x0000240e       0x4a ./bin/LCD.o
                0x0000240e                LCD_DATA_NegBit
 .text.LCD_DATA_SetDir
                0x00002458       0x50 ./bin/LCD.o
                0x00002458                LCD_DATA_SetDir
 .text.Cpu_Delay50US
                0x000024a8       0x30 ./bin/LCD.o
                0x000024a8                Cpu_Delay50US
 .text.LCD_Delay
                0x000024d8       0x20 ./bin/LCD.o
                0x000024d8                LCD_Delay
 .text.LCD_Write_4bit
                0x000024f8       0x44 ./bin/LCD.o
                0x000024f8                LCD_Write_4bit
 .text.LCD_Write_Data
                0x0000253c       0x64 ./bin/LCD.o
                0x0000253c                LCD_Write_Data
 .text.LCD_Write_Inst
                0x000025a0       0x64 ./bin/LCD.o
                0x000025a0                LCD_Write_Inst
 .text.LCD_Clear
                0x00002604       0x20 ./bin/LCD.o
                0x00002604                LCD_Clear
 .text.LCD_Clear_Line
                0x00002624       0x16 ./bin/LCD.o
                0x00002624                LCD_Clear_Line
 .text.LCD_Init
                0x0000263a       0xce ./bin/LCD.o
                0x0000263a                LCD_Init
 .text.LCD_DefChar
                0x00002708       0x6e ./bin/LCD.o
                0x00002708                LCD_DefChar
 .text.LCD_SetPosition
                0x00002776       0x58 ./bin/LCD.o
                0x00002776                LCD_SetPosition
 .text.LCD_PutString
                0x000027ce       0x74 ./bin/LCD.o
                0x000027ce                LCD_PutString
 .text.LCD_Write
                0x00002842       0x48 ./bin/LCD.o
                0x00002842                LCD_Write
 .text.LCD_SetCursorOn
                0x0000288a       0x2c ./bin/LCD.o
                0x0000288a                LCD_SetCursorOn
 .text.LCD_SetCursorOff
                0x000028b6       0x14 ./bin/LCD.o
                0x000028b6                LCD_SetCursorOff
 .text.LCD_PutCenterString
                0x000028ca       0x4e ./bin/LCD.o
                0x000028ca                LCD_PutCenterString
 .text          0x00002918        0x0 ./bin/klavesnica.o
 .text.Klavesnica_Enable
                0x00002918       0x32 ./bin/klavesnica.o
                0x00002918                Klavesnica_Enable
 .text.KlavesnicaValue_GetVal
                0x0000294a       0x4e ./bin/klavesnica.o
                0x0000294a                KlavesnicaValue_GetVal
 .text.__cs3_isr_interrupt_68
                0x00002998       0x74 ./bin/klavesnica.o
                0x00002998                __cs3_isr_interrupt_68
 .text          0x00002a0c        0x0 ./bin/flashUtilities.o
 .text.CFMinit  0x00002a0c       0x4c ./bin/flashUtilities.o
                0x00002a0c                CFMinit
 .text.SaveNastavenia
                0x00002a58        0x8 ./bin/flashUtilities.o
                0x00002a58                SaveNastavenia
 .text.CFMrom2ram
                0x00002a60       0x5a ./bin/flashUtilities.o
                0x00002a60                CFMrom2ram
 .text.CFMcommand
                0x00002aba       0x5c ./bin/flashUtilities.o
                0x00002aba                CFMcommand
 .text.CFMcommandEND
                0x00002b16        0x8 ./bin/flashUtilities.o
                0x00002b16                CFMcommandEND
 *fill*         0x00002b1e        0x2 00
 .text          0x00002b20        0x0 ./bin/riadenie.o
 .text.LCDwrite2
                0x00002b20       0x20 ./bin/riadenie.o
                0x00002b20                LCDwrite2
 .text.NormalnyStav
                0x00002b40       0x26 ./bin/riadenie.o
                0x00002b40                NormalnyStav
 .text.buzzerOK
                0x00002b66       0x40 ./bin/riadenie.o
                0x00002b66                buzzerOK
 .text.buzzerChyba
                0x00002ba6       0x1c ./bin/riadenie.o
                0x00002ba6                buzzerChyba
 .text.dvere    0x00002bc2       0x1c ./bin/riadenie.o
                0x00002bc2                dvere
 .text.OpenDvere
                0x00002bde      0x104 ./bin/riadenie.o
                0x00002bde                OpenDvere
 .text.Chyba    0x00002ce2      0x142 ./bin/riadenie.o
                0x00002ce2                Chyba
 .text.PIN      0x00002e24      0x322 ./bin/riadenie.o
                0x00002e24                PIN
 .text.vTaskTimer
                0x00003146      0x15c ./bin/riadenie.o
                0x00003146                vTaskTimer
 .text.vStartControlTask
                0x000032a2       0x6a ./bin/riadenie.o
                0x000032a2                vStartControlTask
 .text.command_parser
                0x0000330c      0x198 ./bin/riadenie.o
                0x0000330c                command_parser
 .text.vTaskControl
                0x000034a4      0x180 ./bin/riadenie.o
                0x000034a4                vTaskControl
 .text          0x00003624        0x0 ./bin/webcam.o
 .text.uart0_tx
                0x00003624       0x3e ./bin/webcam.o
                0x00003624                uart0_tx
 .text.uart0_rx
                0x00003662       0x3e ./bin/webcam.o
                0x00003662                uart0_rx
 .text.get_ack  0x000036a0       0xf4 ./bin/webcam.o
                0x000036a0                get_ack
 .text.get_ack_customDelay
                0x00003794      0x100 ./bin/webcam.o
                0x00003794                get_ack_customDelay
 .text.sync_camera
                0x00003894      0x1c4 ./bin/webcam.o
                0x00003894                sync_camera
 .text.init_camera
                0x00003a58       0xec ./bin/webcam.o
                0x00003a58                init_camera
 .text.poweroff_camera
                0x00003b44       0x62 ./bin/webcam.o
                0x00003b44                poweroff_camera
 .text.reset_camera
                0x00003ba6       0x70 ./bin/webcam.o
                0x00003ba6                reset_camera
 .text.set_snapshot
                0x00003c16       0x6e ./bin/webcam.o
                0x00003c16                set_snapshot
 .text.take_picture
                0x00003c84       0xdc ./bin/webcam.o
                0x00003c84                take_picture
 .text.clearbuffer
                0x00003d60       0x2a ./bin/webcam.o
                0x00003d60                clearbuffer
 .text.get_jpeg_data_packet
                0x00003d8a      0x308 ./bin/webcam.o
                0x00003d8a                get_jpeg_data_packet
 .text.get_jpeg_data_packet_end
                0x00004092       0x4a ./bin/webcam.o
                0x00004092                get_jpeg_data_packet_end
 .text.kameraBit_PutVal
                0x000040dc       0x30 ./bin/webcam.o
                0x000040dc                kameraBit_PutVal
 .text.picture_taker
                0x0000410c       0xd4 ./bin/webcam.o
                0x0000410c                picture_taker
 .text          0x000041e0        0x0 ./bin/kom_modul.o
 .text.hello_world_init
                0x000041e0       0x14 ./bin/kom_modul.o
                0x000041e0                hello_world_init
 .text.hello_world_appcall
                0x000041f4       0x98 ./bin/kom_modul.o
                0x000041f4                hello_world_appcall
 .text.handle_connection
                0x0000428c      0x122 ./bin/kom_modul.o
 .text.handle_connection2
                0x000043ae      0x18c ./bin/kom_modul.o
                0x000043ae                handle_connection2
 *fill*         0x0000453a        0x2 00
 .text          0x0000453c        0x0 ./bin/rfid_reader.o
 .text.vStartRfidTask
                0x0000453c       0x3c ./bin/rfid_reader.o
                0x0000453c                vStartRfidTask
 .text.vTaskRfid
                0x00004578      0x10e ./bin/rfid_reader.o
                0x00004578                vTaskRfid
 *fill*         0x00004686        0x2 00
 .text          0x00004688        0x0 ./bin/ParTest.o
 .text.vParTestInitialise
                0x00004688        0x8 ./bin/ParTest.o
                0x00004688                vParTestInitialise
 .text.vParTestSetLED
                0x00004690       0x92 ./bin/ParTest.o
                0x00004690                vParTestSetLED
 .text.vParTestToggleLED
                0x00004722       0xa2 ./bin/ParTest.o
                0x00004722                vParTestToggleLED
 .text.uxParTestGetLED
                0x000047c4       0x40 ./bin/ParTest.o
                0x000047c4                uxParTestGetLED
 .text          0x00004804        0x0 ./bin/flash.o
 .text.vStartLEDFlashTasks
                0x00004804       0x44 ./bin/flash.o
                0x00004804                vStartLEDFlashTasks
 .text.vLEDFlashTask
                0x00004848       0x96 ./bin/flash.o
 *fill*         0x000048de        0x2 00
 .text          0x000048e0        0x0 ./bin/FreeRTOS_Tick_Setup.o
 .text.vApplicationSetupInterrupts
                0x000048e0       0x8e ./bin/FreeRTOS_Tick_Setup.o
                0x000048e0                vApplicationSetupInterrupts
 .text.__cs3_isr_interrupt_119
                0x0000496e       0x60 ./bin/FreeRTOS_Tick_Setup.o
                0x0000496e                __cs3_isr_interrupt_119
 *fill*         0x000049ce        0x2 00
 .text          0x000049d0        0x0 ./bin/PollQ.o
 .text.vStartPolledQueueTasks
                0x000049d0       0x8e ./bin/PollQ.o
                0x000049d0                vStartPolledQueueTasks
 .text.vPolledQueueProducer
                0x00004a5e       0x8a ./bin/PollQ.o
 .text.vPolledQueueConsumer
                0x00004ae8       0xa6 ./bin/PollQ.o
 .text.xArePollingQueuesStillRunning
                0x00004b8e       0x38 ./bin/PollQ.o
                0x00004b8e                xArePollingQueuesStillRunning
 *fill*         0x00004bc6        0x2 00
 .text          0x00004bc8        0x0 ./bin/semtest.o
 .text.vStartSemaphoreTasks
                0x00004bc8      0x21a ./bin/semtest.o
                0x00004bc8                vStartSemaphoreTasks
 .text.prvSemaphoreTest
                0x00004de2      0x182 ./bin/semtest.o
 .text.xAreSemaphoreTasksStillRunning
                0x00004f64       0x86 ./bin/semtest.o
                0x00004f64                xAreSemaphoreTasksStillRunning
 *fill*         0x00004fea        0x2 00
 .text          0x00004fec        0x0 ./bin/GenQTest.o
 .text.vStartGenericQueueTasks
                0x00004fec       0xfa ./bin/GenQTest.o
                0x00004fec                vStartGenericQueueTasks
 .text.prvSendFrontAndBackTest
                0x000050e6      0x464 ./bin/GenQTest.o
 .text.prvLowPriorityMutexTask
                0x0000554a      0x124 ./bin/GenQTest.o
 .text.prvMediumPriorityMutexTask
                0x0000566e       0x1e ./bin/GenQTest.o
 .text.prvHighPriorityMutexTask
                0x0000568c       0x60 ./bin/GenQTest.o
 .text.xAreGenericQueueTasksStillRunning
                0x000056ec       0x5e ./bin/GenQTest.o
                0x000056ec                xAreGenericQueueTasksStillRunning
 *fill*         0x0000574a        0x2 00
 .text          0x0000574c        0x0 ./bin/QPeek.o
 .text.vStartQueuePeekTasks
                0x0000574c       0xe2 ./bin/QPeek.o
                0x0000574c                vStartQueuePeekTasks
 .text.prvHighestPriorityPeekTask
                0x0000582e      0x14e ./bin/QPeek.o
 .text.prvHighPriorityPeekTask
                0x0000597c       0xb6 ./bin/QPeek.o
 .text.prvMediumPriorityPeekTask
                0x00005a32       0x7c ./bin/QPeek.o
 .text.prvLowPriorityPeekTask
                0x00005aae      0x170 ./bin/QPeek.o
 .text.xAreQueuePeekTasksStillRunning
                0x00005c1e       0x3a ./bin/QPeek.o
                0x00005c1e                xAreQueuePeekTasksStillRunning
 .text          0x00005c58        0x0 ./bin/FEC.o
 .text.fec_mii_write
                0x00005c58       0xea ./bin/FEC.o
 .text.fec_mii_read
                0x00005d42       0xec ./bin/FEC.o
 .text.fec_hash_address
                0x00005e2e       0x8c ./bin/FEC.o
 .text.fec_set_address
                0x00005eba      0x134 ./bin/FEC.o
 .text.prvInitialiseFECBuffers
                0x00005fee      0x164 ./bin/FEC.o
 .text.vFECInit
                0x00006152      0x494 ./bin/FEC.o
                0x00006152                vFECInit
 .text.prvEnableFECInterrupts
                0x000065e6       0x8c ./bin/FEC.o
 .text.prvResetFEC
                0x00006672       0x64 ./bin/FEC.o
 .text.usFECGetRxedData
                0x000066d6       0x66 ./bin/FEC.o
                0x000066d6                usFECGetRxedData
 .text.vFECRxProcessingCompleted
                0x0000673c       0x66 ./bin/FEC.o
                0x0000673c                vFECRxProcessingCompleted
 .text.vFECSendData
                0x000067a2       0xe0 ./bin/FEC.o
                0x000067a2                vFECSendData
 .text.vFEC_ISR
                0x00006882      0x11c ./bin/FEC.o
                0x00006882                vFEC_ISR
 .text.__cs3_isr_interrupt_87
                0x0000699e       0x18 ./bin/FEC.o
                0x0000699e                __cs3_isr_interrupt_87
 .text.__cs3_isr_interrupt_88
                0x000069b6       0x18 ./bin/FEC.o
                0x000069b6                __cs3_isr_interrupt_88
 .text.__cs3_isr_interrupt_89
                0x000069ce       0x18 ./bin/FEC.o
                0x000069ce                __cs3_isr_interrupt_89
 .text.__cs3_isr_interrupt_90
                0x000069e6       0x18 ./bin/FEC.o
                0x000069e6                __cs3_isr_interrupt_90
 .text.__cs3_isr_interrupt_91
                0x000069fe       0x18 ./bin/FEC.o
                0x000069fe                __cs3_isr_interrupt_91
 .text.__cs3_isr_interrupt_92
                0x00006a16       0x18 ./bin/FEC.o
                0x00006a16                __cs3_isr_interrupt_92
 .text.__cs3_isr_interrupt_93
                0x00006a2e       0x18 ./bin/FEC.o
                0x00006a2e                __cs3_isr_interrupt_93
 .text.__cs3_isr_interrupt_94
                0x00006a46       0x18 ./bin/FEC.o
                0x00006a46                __cs3_isr_interrupt_94
 .text.__cs3_isr_interrupt_95
                0x00006a5e       0x18 ./bin/FEC.o
                0x00006a5e                __cs3_isr_interrupt_95
 .text.__cs3_isr_interrupt_96
                0x00006a76       0x18 ./bin/FEC.o
                0x00006a76                __cs3_isr_interrupt_96
 .text.__cs3_isr_interrupt_97
                0x00006a8e       0x18 ./bin/FEC.o
                0x00006a8e                __cs3_isr_interrupt_97
 .text.__cs3_isr_interrupt_98
                0x00006aa6       0x18 ./bin/FEC.o
                0x00006aa6                __cs3_isr_interrupt_98
 .text.__cs3_isr_interrupt_99
                0x00006abe       0x18 ./bin/FEC.o
                0x00006abe                __cs3_isr_interrupt_99
 *fill*         0x00006ad6        0x2 00
 .text          0x00006ad8        0x0 ./bin/blocktim.o
 .text.vCreateBlockTimeTasks
                0x00006ad8       0x8a ./bin/blocktim.o
                0x00006ad8                vCreateBlockTimeTasks
 .text.vPrimaryBlockTimeTestTask
                0x00006b62      0x44c ./bin/blocktim.o
 .text.vSecondaryBlockTimeTestTask
                0x00006fae      0x12e ./bin/blocktim.o
 .text.xAreBlockTimeTestTasksStillRunning
                0x000070dc       0x62 ./bin/blocktim.o
                0x000070dc                xAreBlockTimeTestTasksStillRunning
 *fill*         0x0000713e        0x2 00
 .text          0x00007140        0x0 ./bin/recmutex.o
 .text.vStartRecursiveMutexTasks
                0x00007140       0xb4 ./bin/recmutex.o
                0x00007140                vStartRecursiveMutexTasks
 .text.prvRecursiveMutexControllingTask
                0x000071f4       0xe6 ./bin/recmutex.o
 .text.prvRecursiveMutexBlockingTask
                0x000072da       0xa2 ./bin/recmutex.o
 .text.prvRecursiveMutexPollingTask
                0x0000737c       0x88 ./bin/recmutex.o
 .text.xAreRecursiveMutexTasksStillRunning
                0x00007404       0x96 ./bin/recmutex.o
                0x00007404                xAreRecursiveMutexTasksStillRunning
 *fill*         0x0000749a        0x2 00
 .text          0x0000749c        0x0 ./bin/console_reader.o
 .text.funkcia  0x0000749c       0xfa ./bin/console_reader.o
                0x0000749c                funkcia
 .text.testTlacit
                0x00007596       0x58 ./bin/console_reader.o
                0x00007596                testTlacit
 .text.testFunkcia1
                0x000075ee       0xf0 ./bin/console_reader.o
                0x000075ee                testFunkcia1
 .text.cpuVykon
                0x000076de       0x66 ./bin/console_reader.o
                0x000076de                cpuVykon
 .text.heap     0x00007744       0x56 ./bin/console_reader.o
                0x00007744                heap
 .text.camsync  0x0000779a       0x96 ./bin/console_reader.o
                0x0000779a                camsync
 .text.caminit  0x00007830       0xa6 ./bin/console_reader.o
                0x00007830                caminit
 .text.camtakepic
                0x000078d6      0x17a ./bin/console_reader.o
                0x000078d6                camtakepic
 .text.camgetpacket
                0x00007a50       0x8e ./bin/console_reader.o
                0x00007a50                camgetpacket
 .text.camnextpacket
                0x00007ade       0x36 ./bin/console_reader.o
                0x00007ade                camnextpacket
 .text.camgetpacketnext
                0x00007b14       0x8e ./bin/console_reader.o
                0x00007b14                camgetpacketnext
 .text.resetcam
                0x00007ba2      0x108 ./bin/console_reader.o
                0x00007ba2                resetcam
 .text.pinSet   0x00007caa       0xa4 ./bin/console_reader.o
                0x00007caa                pinSet
 .text.bit1Set  0x00007d4e       0x90 ./bin/console_reader.o
                0x00007d4e                bit1Set
 .text.bit2Set  0x00007dde       0x90 ./bin/console_reader.o
                0x00007dde                bit2Set
 .text.psocket_koniec
                0x00007e6e        0x8 ./bin/console_reader.o
                0x00007e6e                psocket_koniec
 .text.psocket_send
                0x00007e76       0x36 ./bin/console_reader.o
                0x00007e76                psocket_send
 .text.flashWrite
                0x00007eac      0x14a ./bin/console_reader.o
                0x00007eac                flashWrite
 .text.flashRead
                0x00007ff6       0x9a ./bin/console_reader.o
                0x00007ff6                flashRead
 .text.pause    0x00008090       0x92 ./bin/console_reader.o
                0x00008090                pause
 .text.LCDwrite
                0x00008122       0x1a ./bin/console_reader.o
                0x00008122                LCDwrite
 .text.klavesnica
                0x0000813c       0x70 ./bin/console_reader.o
                0x0000813c                klavesnica
 .text.testPIN  0x000081ac       0x16 ./bin/console_reader.o
                0x000081ac                testPIN
 .text.vStartConsole_reader
                0x000081c2       0x3e ./bin/console_reader.o
                0x000081c2                vStartConsole_reader
 .text.console_reader
                0x00008200      0x55e ./bin/console_reader.o
                0x00008200                console_reader
 .text.consoleRead
                0x0000875e      0x124 ./bin/console_reader.o
                0x0000875e                consoleRead
 *fill*         0x00008882        0x2 00
 .text          0x00008884        0x0 ./bin/printf-stdarg.o
 .text.outbyte  0x00008884       0x3c ./bin/printf-stdarg.o
 .text.printchar
                0x000088c0       0x4e ./bin/printf-stdarg.o
 .text.prints   0x0000890e       0xc6 ./bin/printf-stdarg.o
 .text.printi   0x000089d4      0x11c ./bin/printf-stdarg.o
 .text.print    0x00008af0      0x30a ./bin/printf-stdarg.o
 .text.xxprintf
                0x00008dfa       0x2a ./bin/printf-stdarg.o
                0x00008dfa                xxprintf
 .text.sprintf  0x00008e24       0x2e ./bin/printf-stdarg.o
                0x00008e24                sprintf
 .text.snprintf
                0x00008e52       0x2e ./bin/printf-stdarg.o
                0x00008e52                snprintf
 .text.write    0x00008e80        0xa ./bin/printf-stdarg.o
                0x00008e80                write
 *fill*         0x00008e8a        0x2 00
 .text          0x00008e8c       0x7c ./bin/portasm.o
                0x00008e8c                ulPortSetIPL
                0x00008ec2                mcf5xxx_wr_cacr
                0x00008ece                __cs3_isr_interrupt_80
                0x00008ef6                vPortStartFirstTask
 .text          0x00008f08        0x0 ./bin/port.o
 .text.pxPortInitialiseStack
                0x00008f08       0x5a ./bin/port.o
                0x00008f08                pxPortInitialiseStack
 .text.xPortStartScheduler
                0x00008f62       0x1c ./bin/port.o
                0x00008f62                xPortStartScheduler
 .text.vPortEndScheduler
                0x00008f7e        0x8 ./bin/port.o
                0x00008f7e                vPortEndScheduler
 .text.vPortEnterCritical
                0x00008f86       0x48 ./bin/port.o
                0x00008f86                vPortEnterCritical
 .text.vPortExitCritical
                0x00008fce       0x2a ./bin/port.o
                0x00008fce                vPortExitCritical
 .text.vPortYieldHandler
                0x00008ff8       0x34 ./bin/port.o
                0x00008ff8                vPortYieldHandler
 .text          0x0000902c        0x0 ./bin/list.o
 .text.vListInitialise
                0x0000902c       0x52 ./bin/list.o
                0x0000902c                vListInitialise
 .text.vListInitialiseItem
                0x0000907e       0x12 ./bin/list.o
                0x0000907e                vListInitialiseItem
 .text.vListInsertEnd
                0x00009090       0x8e ./bin/list.o
                0x00009090                vListInsertEnd
 .text.vListInsert
                0x0000911e       0xbc ./bin/list.o
                0x0000911e                vListInsert
 .text.vListRemove
                0x000091da       0x8e ./bin/list.o
                0x000091da                vListRemove
 .text          0x00009268        0x0 ./bin/tasks.o
 .text.xTaskGenericCreate
                0x00009268      0x1e0 ./bin/tasks.o
                0x00009268                xTaskGenericCreate
 .text.vTaskDelete
                0x00009448       0xc0 ./bin/tasks.o
                0x00009448                vTaskDelete
 .text.vTaskDelayUntil
                0x00009508      0x11a ./bin/tasks.o
                0x00009508                vTaskDelayUntil
 .text.vTaskDelay
                0x00009622       0xb4 ./bin/tasks.o
                0x00009622                vTaskDelay
 .text.uxTaskPriorityGet
                0x000096d6       0x3c ./bin/tasks.o
                0x000096d6                uxTaskPriorityGet
 .text.vTaskPrioritySet
                0x00009712      0x16a ./bin/tasks.o
                0x00009712                vTaskPrioritySet
 .text.vTaskSuspend
                0x0000987c       0x9a ./bin/tasks.o
                0x0000987c                vTaskSuspend
 .text.xTaskIsTaskSuspended
                0x00009916       0x4e ./bin/tasks.o
                0x00009916                xTaskIsTaskSuspended
 .text.vTaskResume
                0x00009964       0xce ./bin/tasks.o
                0x00009964                vTaskResume
 .text.xTaskResumeFromISR
                0x00009a32       0xdc ./bin/tasks.o
                0x00009a32                xTaskResumeFromISR
 .text.vTaskStartScheduler
                0x00009b0e       0x5a ./bin/tasks.o
                0x00009b0e                vTaskStartScheduler
 .text.vTaskEndScheduler
                0x00009b68       0x20 ./bin/tasks.o
                0x00009b68                vTaskEndScheduler
 .text.vTaskSuspendAll
                0x00009b88       0x16 ./bin/tasks.o
                0x00009b88                vTaskSuspendAll
 .text.xTaskResumeAll
                0x00009b9e      0x14e ./bin/tasks.o
                0x00009b9e                xTaskResumeAll
 .text.xTaskGetTickCount
                0x00009cec       0x22 ./bin/tasks.o
                0x00009cec                xTaskGetTickCount
 .text.uxTaskGetNumberOfTasks
                0x00009d0e        0xe ./bin/tasks.o
                0x00009d0e                uxTaskGetNumberOfTasks
 .text.vTaskList
                0x00009d1c      0x134 ./bin/tasks.o
                0x00009d1c                vTaskList
 .text.vTaskStartTrace
                0x00009e50       0x40 ./bin/tasks.o
                0x00009e50                vTaskStartTrace
 .text.ulTaskEndTrace
                0x00009e90       0x30 ./bin/tasks.o
                0x00009e90                ulTaskEndTrace
 .text.vTaskIncrementTick
                0x00009ec0      0x11c ./bin/tasks.o
                0x00009ec0                vTaskIncrementTick
 .text.vTaskSwitchContext
                0x00009fdc      0x1d2 ./bin/tasks.o
                0x00009fdc                vTaskSwitchContext
 .text.vTaskPlaceOnEventList
                0x0000a1ae       0xbc ./bin/tasks.o
                0x0000a1ae                vTaskPlaceOnEventList
 .text.xTaskRemoveFromEventList
                0x0000a26a       0xee ./bin/tasks.o
                0x0000a26a                xTaskRemoveFromEventList
 .text.vTaskSetTimeOutState
                0x0000a358       0x26 ./bin/tasks.o
                0x0000a358                vTaskSetTimeOutState
 .text.xTaskCheckForTimeOut
                0x0000a37e       0xb6 ./bin/tasks.o
                0x0000a37e                xTaskCheckForTimeOut
 .text.vTaskMissedYield
                0x0000a434       0x10 ./bin/tasks.o
                0x0000a434                vTaskMissedYield
 .text.prvIdleTask
                0x0000a444        0xc ./bin/tasks.o
 .text.prvInitialiseTCBVariables
                0x0000a450       0xb6 ./bin/tasks.o
 .text.prvInitialiseTaskLists
                0x0000a506       0x94 ./bin/tasks.o
 .text.prvCheckTasksWaitingTermination
                0x0000a59a       0xae ./bin/tasks.o
 .text.prvAllocateTCBAndStack
                0x0000a648       0x96 ./bin/tasks.o
 .text.prvListTaskWithinSingleList
                0x0000a6de      0x15a ./bin/tasks.o
 .text.usTaskCheckFreeStackSpace
                0x0000a838       0x3c ./bin/tasks.o
 .text.uxTaskGetStackHighWaterMark
                0x0000a874       0x48 ./bin/tasks.o
                0x0000a874                uxTaskGetStackHighWaterMark
 .text.prvDeleteTCB
                0x0000a8bc       0x28 ./bin/tasks.o
 .text.xTaskGetCurrentTaskHandle
                0x0000a8e4       0x16 ./bin/tasks.o
                0x0000a8e4                xTaskGetCurrentTaskHandle
 .text.vTaskPriorityInherit
                0x0000a8fa       0xf6 ./bin/tasks.o
                0x0000a8fa                vTaskPriorityInherit
 .text.vTaskPriorityDisinherit
                0x0000a9f0       0xba ./bin/tasks.o
                0x0000a9f0                vTaskPriorityDisinherit
 *fill*         0x0000aaaa        0x2 00
 .text          0x0000aaac        0x0 ./bin/queue.o
 .text.xQueueCreate
                0x0000aaac      0x12e ./bin/queue.o
                0x0000aaac                xQueueCreate
 .text.xQueueCreateMutex
                0x0000abda       0xbe ./bin/queue.o
                0x0000abda                xQueueCreateMutex
 .text.xQueueGiveMutexRecursive
                0x0000ac98       0x6c ./bin/queue.o
                0x0000ac98                xQueueGiveMutexRecursive
 .text.xQueueTakeMutexRecursive
                0x0000ad04       0x80 ./bin/queue.o
                0x0000ad04                xQueueTakeMutexRecursive
 .text.xQueueCreateCountingSemaphore
                0x0000ad84       0x32 ./bin/queue.o
                0x0000ad84                xQueueCreateCountingSemaphore
 .text.xQueueGenericSend
                0x0000adb6      0x1aa ./bin/queue.o
                0x0000adb6                xQueueGenericSend
 .text.xQueueGenericSendFromISR
                0x0000af60       0xc8 ./bin/queue.o
                0x0000af60                xQueueGenericSendFromISR
 .text.xQueueGenericReceive
                0x0000b028      0x264 ./bin/queue.o
                0x0000b028                xQueueGenericReceive
 .text.xQueueReceiveFromISR
                0x0000b28c       0xd0 ./bin/queue.o
                0x0000b28c                xQueueReceiveFromISR
 .text.uxQueueMessagesWaiting
                0x0000b35c       0x26 ./bin/queue.o
                0x0000b35c                uxQueueMessagesWaiting
 .text.uxQueueMessagesWaitingFromISR
                0x0000b382       0x1a ./bin/queue.o
                0x0000b382                uxQueueMessagesWaitingFromISR
 .text.vQueueDelete
                0x0000b39c       0x32 ./bin/queue.o
                0x0000b39c                vQueueDelete
 .text.prvCopyDataToQueue
                0x0000b3ce      0x162 ./bin/queue.o
 .text.prvCopyDataFromQueue
                0x0000b530       0x84 ./bin/queue.o
 .text.prvUnlockQueue
                0x0000b5b4       0xe8 ./bin/queue.o
 .text.prvIsQueueEmpty
                0x0000b69c       0x38 ./bin/queue.o
 .text.xQueueIsQueueEmptyFromISR
                0x0000b6d4       0x2c ./bin/queue.o
                0x0000b6d4                xQueueIsQueueEmptyFromISR
 .text.prvIsQueueFull
                0x0000b700       0x42 ./bin/queue.o
 .text.xQueueIsQueueFullFromISR
                0x0000b742       0x36 ./bin/queue.o
                0x0000b742                xQueueIsQueueFullFromISR
 .text.vQueueAddToRegistry
                0x0000b778       0x68 ./bin/queue.o
                0x0000b778                vQueueAddToRegistry
 .text.vQueueUnregisterQueue
                0x0000b7e0       0x4e ./bin/queue.o
 *fill*         0x0000b82e        0x2 00
 .text          0x0000b830        0x0 ./bin/heap_1.o
 .text.pvPortMalloc
                0x0000b830       0x7c ./bin/heap_1.o
                0x0000b830                pvPortMalloc
 .text.vPortFree
                0x0000b8ac        0x8 ./bin/heap_1.o
                0x0000b8ac                vPortFree
 .text.vPortInitialiseBlocks
                0x0000b8b4        0xe ./bin/heap_1.o
                0x0000b8b4                vPortInitialiseBlocks
 .text.xPortGetFreeHeapSize
                0x0000b8c2       0x18 ./bin/heap_1.o
                0x0000b8c2                xPortGetFreeHeapSize
 *fill*         0x0000b8da        0x2 00
 .text          0x0000b8dc        0x0 ./bin/timer.o
 .text.timer_set
                0x0000b8dc       0x26 ./bin/timer.o
                0x0000b8dc                timer_set
 .text.timer_reset
                0x0000b902       0x24 ./bin/timer.o
                0x0000b902                timer_reset
 .text.timer_restart
                0x0000b926       0x18 ./bin/timer.o
                0x0000b926                timer_restart
 .text.timer_expired
                0x0000b93e       0x2a ./bin/timer.o
                0x0000b93e                timer_expired
 .text          0x0000b968        0x0 ./bin/uip.o
 .text.uip_setipid
                0x0000b968       0x1a ./bin/uip.o
                0x0000b968                uip_setipid
 .text.uip_add32
                0x0000b982      0x11e ./bin/uip.o
                0x0000b982                uip_add32
 .text.chksum   0x0000baa0       0xe6 ./bin/uip.o
 .text.uip_chksum
                0x0000bb86       0x3c ./bin/uip.o
                0x0000bb86                uip_chksum
 .text.uip_ipchksum
                0x0000bbc2       0x44 ./bin/uip.o
                0x0000bbc2                uip_ipchksum
 .text.upper_layer_chksum
                0x0000bc06       0xe6 ./bin/uip.o
 .text.uip_tcpchksum
                0x0000bcec       0x14 ./bin/uip.o
                0x0000bcec                uip_tcpchksum
 .text.uip_udpchksum
                0x0000bd00       0x14 ./bin/uip.o
                0x0000bd00                uip_udpchksum
 .text.uip_init
                0x0000bd14       0xb8 ./bin/uip.o
                0x0000bd14                uip_init
 .text.uip_connect
                0x0000bdcc      0x246 ./bin/uip.o
                0x0000bdcc                uip_connect
 .text.uip_unlisten
                0x0000c012       0x90 ./bin/uip.o
                0x0000c012                uip_unlisten
 .text.uip_listen
                0x0000c0a2       0x84 ./bin/uip.o
                0x0000c0a2                uip_listen
 .text.uip_add_rcv_nxt
                0x0000c126       0x72 ./bin/uip.o
 .text.uip_process
                0x0000c198     0x22c8 ./bin/uip.o
                0x0000c198                uip_process
 .text.htons    0x0000e460       0x14 ./bin/uip.o
                0x0000e460                htons
 .text.uip_send
                0x0000e474       0x4c ./bin/uip.o
                0x0000e474                uip_send
 .text.uip_fast_send
                0x0000e4c0        0xa ./bin/uip.o
                0x0000e4c0                uip_fast_send
 *fill*         0x0000e4ca        0x2 00
 .text          0x0000e4cc        0x0 ./bin/uip_arp.o
 .text.uip_arp_init
                0x0000e4cc       0x66 ./bin/uip_arp.o
                0x0000e4cc                uip_arp_init
 .text.uip_arp_timer
                0x0000e532       0xce ./bin/uip_arp.o
                0x0000e532                uip_arp_timer
 .text.uip_arp_update
                0x0000e600      0x288 ./bin/uip_arp.o
 .text.uip_arp_ipin
                0x0000e888       0x90 ./bin/uip_arp.o
                0x0000e888                uip_arp_ipin
 .text.uip_arp_arpin
                0x0000e918      0x26e ./bin/uip_arp.o
                0x0000e918                uip_arp_arpin
 .text.uip_arp_out
                0x0000eb86      0x388 ./bin/uip_arp.o
                0x0000eb86                uip_arp_out
 *fill*         0x0000ef0e        0x2 00
 .text          0x0000ef10        0x0 ./bin/uiplib.o
 .text.uiplib_ipaddrconv
                0x0000ef10       0xe0 ./bin/uiplib.o
                0x0000ef10                uiplib_ipaddrconv
 .text          0x0000eff0        0x0 ./bin/uip-split.o
 .text.uip_split_output
                0x0000eff0      0x2b4 ./bin/uip-split.o
                0x0000eff0                uip_split_output
 .text          0x0000f2a4        0x0 ./bin/psock.o
 .text.buf_setup
                0x0000f2a4       0x28 ./bin/psock.o
 .text.buf_bufdata
                0x0000f2cc      0x236 ./bin/psock.o
 .text.buf_bufto
                0x0000f502       0xdc ./bin/psock.o
 .text.send_data
                0x0000f5de       0xc6 ./bin/psock.o
 .text.data_acked
                0x0000f6a4       0xd4 ./bin/psock.o
 .text.psock_send
                0x0000f778       0xba ./bin/psock.o
                0x0000f778                psock_send
 .text.psock_generator_send
                0x0000f832       0xea ./bin/psock.o
                0x0000f832                psock_generator_send
 .text.psock_datalen
                0x0000f91c       0x22 ./bin/psock.o
                0x0000f91c                psock_datalen
 .text.psock_newdata
                0x0000f93e       0x5e ./bin/psock.o
                0x0000f93e                psock_newdata
 .text.psock_readto
                0x0000f99c      0x11e ./bin/psock.o
                0x0000f99c                psock_readto
 .text.psock_readbuf
                0x0000faba      0x12e ./bin/psock.o
                0x0000faba                psock_readbuf
 .text.psock_init
                0x0000fbe8       0x66 ./bin/psock.o
                0x0000fbe8                psock_init
 *fill*         0x0000fc4e        0x2 00
 .text          0x0000fc50        0x0 ./bin/uIP_Task.o
 .text.clock_init
                0x0000fc50        0x8 ./bin/uIP_Task.o
                0x0000fc50                clock_init
 .text.clock_time
                0x0000fc58        0xe ./bin/uIP_Task.o
                0x0000fc58                clock_time
 .text.uIP_appcall
                0x0000fc66       0x38 ./bin/uIP_Task.o
                0x0000fc66                uIP_appcall
 .text.vuIP_Task
                0x0000fc9e      0x214 ./bin/uIP_Task.o
                0x0000fc9e                vuIP_Task
 *fill*         0x0000feb2        0x2 00
 .text          0x0000feb4        0x0 ./bin/httpd.o
 .text.generate_part_of_file
                0x0000feb4       0xd4 ./bin/httpd.o
 .text.send_file
                0x0000ff88      0x21c ./bin/httpd.o
 .text.send_part_of_file
                0x000101a4       0x88 ./bin/httpd.o
 .text.next_scriptstate
                0x0001022c       0x68 ./bin/httpd.o
 .text.handle_script
                0x00010294      0x34e ./bin/httpd.o
 .text.send_headers
                0x000105e2      0x3ac ./bin/httpd.o
 .text.handle_output
                0x0001098e      0x1e6 ./bin/httpd.o
 .text.handle_input
                0x00010b74      0x26c ./bin/httpd.o
 .text.handle_connection
                0x00010de0       0x38 ./bin/httpd.o
 .text.httpd_appcall
                0x00010e18      0x152 ./bin/httpd.o
                0x00010e18                httpd_appcall
 .text.httpd_init
                0x00010f6a       0x1c ./bin/httpd.o
                0x00010f6a                httpd_init
 *fill*         0x00010f86        0x2 00
 .text          0x00010f88        0x0 ./bin/httpd-cgi.o
 .text.nullfunction
                0x00010f88       0x22 ./bin/httpd-cgi.o
 .text.httpd_cgi
                0x00010faa       0x74 ./bin/httpd-cgi.o
                0x00010faa                httpd_cgi
 .text.generate_file_stats
                0x0001101e       0x42 ./bin/httpd-cgi.o
 .text.file_stats
                0x00011060       0x86 ./bin/httpd-cgi.o
 .text.generate_tcp_stats
                0x000110e6      0x1ee ./bin/httpd-cgi.o
 .text.tcp_stats
                0x000112d4       0xf4 ./bin/httpd-cgi.o
 .text.generate_net_stats
                0x000113c8       0x54 ./bin/httpd-cgi.o
 .text.net_stats
                0x0001141c       0xb6 ./bin/httpd-cgi.o
 .text.generate_rtos_stats
                0x000114d2       0x76 ./bin/httpd-cgi.o
 .text.rtos_stats
                0x00011548       0x76 ./bin/httpd-cgi.o
 .text.generate_io_state
                0x000115be       0x64 ./bin/httpd-cgi.o
 .text.led_io   0x00011622       0x76 ./bin/httpd-cgi.o
 .text.vApplicationProcessFormInput
                0x00011698       0x86 ./bin/httpd-cgi.o
                0x00011698                vApplicationProcessFormInput
 *fill*         0x0001171e        0x2 00
 .text          0x00011720        0x0 ./bin/httpd-fs.o
 .text.httpd_fs_strcmp
                0x00011720       0x9e ./bin/httpd-fs.o
 .text.httpd_fs_open
                0x000117be      0x16a ./bin/httpd-fs.o
                0x000117be                httpd_fs_open
 .text.httpd_fs_init
                0x00011928       0x42 ./bin/httpd-fs.o
                0x00011928                httpd_fs_init
 .text.httpd_fs_count
                0x0001196a       0x6c ./bin/httpd-fs.o
                0x0001196a                httpd_fs_count
 *fill*         0x000119d6        0x2 00
 .text          0x000119d8        0x0 ./bin/http-strings.o
 .text          0x000119d8      0x7ca c:/program files/codesourcery/sourcery g++ lite/bin/../lib/gcc/m68k-elf/4.4.1/m5208\libgcc.a(_float.o)
                0x00011a20                __subsf3
                0x00011a26                __addsf3
                0x00011d08                __mulsf3
                0x00011e4a                __divsf3
                0x0001203e                __negsf2
                0x00012090                __cmpsf2_internal
                0x00012130                __cmpsf2
 *fill*         0x000121a2        0x2 00
 .text          0x000121a4       0x74 c:/program files/codesourcery/sourcery g++ lite/bin/../lib/gcc/m68k-elf/4.4.1/m5208\libgcc.a(_floatex.o)
                0x000121a4                __clear_sticky_bit
                0x000121b0                $_exception_handler
 .text          0x00012218       0x58 c:/program files/codesourcery/sourcery g++ lite/bin/../lib/gcc/m68k-elf/4.4.1/m5208\libgcc.a(_fixunssfsi.o)
                0x00012218                __fixunssfsi
 .text          0x00012270      0x4ca c:/program files/codesourcery/sourcery g++ lite/bin/../lib/gcc/m68k-elf/4.4.1/m5208\libgcc.a(fpgnulib.o)
                0x00012270                __unordsf2
                0x000122d2                __unorddf2
                0x0001234c                __floatunsidf
                0x000123b8                __floatsidf
                0x00012460                __floatunsisf
                0x0001247a                __floatsisf
                0x00012494                __extendsfdf2
                0x0001252e                __truncdfsf2
                0x0001269e                __fixdfsi
                0x00012720                __fixsfsi
 *fill*         0x0001273a        0x2 00
 .text          0x0001273c       0x1a c:/program files/codesourcery/sourcery g++ lite/bin/../lib/gcc/m68k-elf/4.4.1/m5208\libgcc.a(_gesf2.o)
                0x0001273c                __gesf2
 *fill*         0x00012756        0x2 00
 .text          0x00012758       0x18 c:/program files/codesourcery/sourcery g++ lite/bin/../lib/gcc/m68k-elf/4.4.1/../../../../m68k-elf/lib/m5208\libc.a(lib_a-atexit.o)
                0x00012758                atexit
 .text          0x00012770       0x34 c:/program files/codesourcery/sourcery g++ lite/bin/../lib/gcc/m68k-elf/4.4.1/../../../../m68k-elf/lib/m5208\libc.a(lib_a-atoi.o)
                0x00012770                _atoi_r
                0x0001278c                atoi
 .text          0x000127a4       0x32 c:/program files/codesourcery/sourcery g++ lite/bin/../lib/gcc/m68k-elf/4.4.1/../../../../m68k-elf/lib/m5208\libc.a(lib_a-exit.o)
                0x000127a4                exit
 *fill*         0x000127d6        0x2 00
 .text          0x000127d8        0x0 c:/program files/codesourcery/sourcery g++ lite/bin/../lib/gcc/m68k-elf/4.4.1/../../../../m68k-elf/lib/m5208\libc.a(lib_a-impure.o)
 .text          0x000127d8       0x76 c:/program files/codesourcery/sourcery g++ lite/bin/../lib/gcc/m68k-elf/4.4.1/../../../../m68k-elf/lib/m5208\libc.a(lib_a-memcmp.o)
                0x000127d8                memcmp
 *fill*         0x0001284e        0x2 00
 .text          0x00012850       0x70 c:/program files/codesourcery/sourcery g++ lite/bin/../lib/gcc/m68k-elf/4.4.1/../../../../m68k-elf/lib/m5208\libc.a(lib_a-memcpy.o)
                0x00012850                memcpy
 .text          0x000128c0       0x6c c:/program files/codesourcery/sourcery g++ lite/bin/../lib/gcc/m68k-elf/4.4.1/../../../../m68k-elf/lib/m5208\libc.a(lib_a-memset.o)
                0x000128c0                memset
 .text          0x0001292c       0xae c:/program files/codesourcery/sourcery g++ lite/bin/../lib/gcc/m68k-elf/4.4.1/../../../../m68k-elf/lib/m5208\libc.a(lib_a-puts.o)
                0x0001292c                _puts_r
                0x000129c4                puts
 *fill*         0x000129da        0x2 00
 .text          0x000129dc       0x4e c:/program files/codesourcery/sourcery g++ lite/bin/../lib/gcc/m68k-elf/4.4.1/../../../../m68k-elf/lib/m5208\libc.a(lib_a-strcat.o)
                0x000129dc                strcat
 *fill*         0x00012a2a        0x2 00
 .text          0x00012a2c      0x148 c:/program files/codesourcery/sourcery g++ lite/bin/../lib/gcc/m68k-elf/4.4.1/../../../../m68k-elf/lib/m5208\libc.a(lib_a-strchr.o)
                0x00012a2c                strchr
 .text          0x00012b74       0x78 c:/program files/codesourcery/sourcery g++ lite/bin/../lib/gcc/m68k-elf/4.4.1/../../../../m68k-elf/lib/m5208\libc.a(lib_a-strcmp.o)
                0x00012b74                strcmp
 .text          0x00012bec       0x1c c:/program files/codesourcery/sourcery g++ lite/bin/../lib/gcc/m68k-elf/4.4.1/../../../../m68k-elf/lib/m5208\libc.a(lib_a-strcpy.o)
                0x00012bec                strcpy
 .text          0x00012c08       0x18 c:/program files/codesourcery/sourcery g++ lite/bin/../lib/gcc/m68k-elf/4.4.1/../../../../m68k-elf/lib/m5208\libc.a(lib_a-strlen.o)
                0x00012c08                strlen
 .text          0x00012c20       0xc6 c:/program files/codesourcery/sourcery g++ lite/bin/../lib/gcc/m68k-elf/4.4.1/../../../../m68k-elf/lib/m5208\libc.a(lib_a-strncmp.o)
                0x00012c20                strncmp
 *fill*         0x00012ce6        0x2 00
 .text          0x00012ce8       0x86 c:/program files/codesourcery/sourcery g++ lite/bin/../lib/gcc/m68k-elf/4.4.1/../../../../m68k-elf/lib/m5208\libc.a(lib_a-strncpy.o)
                0x00012ce8                strncpy
 *fill*         0x00012d6e        0x2 00
 .text          0x00012d70       0x58 c:/program files/codesourcery/sourcery g++ lite/bin/../lib/gcc/m68k-elf/4.4.1/../../../../m68k-elf/lib/m5208\libc.a(lib_a-strrchr.o)
                0x00012d70                strrchr
 .text          0x00012dc8       0x26 c:/program files/codesourcery/sourcery g++ lite/bin/../lib/gcc/m68k-elf/4.4.1/../../../../m68k-elf/lib/m5208\libc.a(lib_a-strtok.o)
                0x00012dc8                strtok
 *fill*         0x00012dee        0x2 00
 .text          0x00012df0       0xc0 c:/program files/codesourcery/sourcery g++ lite/bin/../lib/gcc/m68k-elf/4.4.1/../../../../m68k-elf/lib/m5208\libc.a(lib_a-strtok_r.o)
                0x00012df0                __strtok_r
                0x00012e94                strtok_r
 .text          0x00012eb0      0x180 c:/program files/codesourcery/sourcery g++ lite/bin/../lib/gcc/m68k-elf/4.4.1/../../../../m68k-elf/lib/m5208\libc.a(lib_a-strtol.o)
                0x00012eb0                _strtol_r
                0x00013012                strtol
 .text          0x00013030       0xec c:/program files/codesourcery/sourcery g++ lite/bin/../lib/gcc/m68k-elf/4.4.1/../../../../m68k-elf/lib/m5208\libc.a(lib_a-__atexit.o)
                0x00013030                __register_exitproc
 .text          0x0001311c      0x132 c:/program files/codesourcery/sourcery g++ lite/bin/../lib/gcc/m68k-elf/4.4.1/../../../../m68k-elf/lib/m5208\libc.a(lib_a-__call_atexit.o)
                0x0001311c                __call_exitprocs
 *fill*         0x0001324e        0x2 00
 .text          0x00013250        0x0 c:/program files/codesourcery/sourcery g++ lite/bin/../lib/gcc/m68k-elf/4.4.1/../../../../m68k-elf/lib/m5208\libc.a(lib_a-ctype_.o)
 .text          0x00013250       0x40 c:/program files/codesourcery/sourcery g++ lite/bin/../lib/gcc/m68k-elf/4.4.1/../../../../m68k-elf/lib/m5208\libc.a(lib_a-fini.o)
                0x00013250                __libc_fini_array
 .text          0x00013290      0x3e0 c:/program files/codesourcery/sourcery g++ lite/bin/../lib/gcc/m68k-elf/4.4.1/../../../../m68k-elf/lib/m5208\libc.a(lib_a-fvwrite.o)
                0x00013290                __sfvwrite_r
 .text          0x00013670      0x734 c:/program files/codesourcery/sourcery g++ lite/bin/../lib/gcc/m68k-elf/4.4.1/../../../../m68k-elf/lib/m5208\libc.a(lib_a-mallocr.o)
                0x00013670                _malloc_r
 .text          0x00013da4       0xc0 c:/program files/codesourcery/sourcery g++ lite/bin/../lib/gcc/m68k-elf/4.4.1/../../../../m68k-elf/lib/m5208\libc.a(lib_a-memchr.o)
                0x00013da4                memchr
 .text          0x00013e64       0xfa c:/program files/codesourcery/sourcery g++ lite/bin/../lib/gcc/m68k-elf/4.4.1/../../../../m68k-elf/lib/m5208\libc.a(lib_a-memmove.o)
                0x00013e64                memmove
 *fill*         0x00013f5e        0x2 00
 .text          0x00013f60       0x10 c:/program files/codesourcery/sourcery g++ lite/bin/../lib/gcc/m68k-elf/4.4.1/../../../../m68k-elf/lib/m5208\libc.a(lib_a-mlock.o)
                0x00013f60                __malloc_lock
                0x00013f68                __malloc_unlock
 .text          0x00013f70      0x45c c:/program files/codesourcery/sourcery g++ lite/bin/../lib/gcc/m68k-elf/4.4.1/../../../../m68k-elf/lib/m5208\libc.a(lib_a-reallocr.o)
                0x00013f70                _realloc_r
 .text          0x000143cc       0x32 c:/program files/codesourcery/sourcery g++ lite/bin/../lib/gcc/m68k-elf/4.4.1/../../../../m68k-elf/lib/m5208\libc.a(lib_a-sbrkr.o)
                0x000143cc                _sbrk_r
 *fill*         0x000143fe        0x2 00
 .text          0x00014400      0x134 c:/program files/codesourcery/sourcery g++ lite/bin/../lib/gcc/m68k-elf/4.4.1/../../../../m68k-elf/lib/m5208\libc.a(lib_a-wsetup.o)
                0x00014400                __swsetup_r
 .text          0x00014534      0x1ca c:/program files/codesourcery/sourcery g++ lite/bin/../lib/gcc/m68k-elf/4.4.1/../../../../m68k-elf/lib/m5208\libc.a(lib_a-fflush.o)
                0x00014534                _fflush_r
                0x000146cc                fflush
 *fill*         0x000146fe        0x2 00
 .text          0x00014700      0x266 c:/program files/codesourcery/sourcery g++ lite/bin/../lib/gcc/m68k-elf/4.4.1/../../../../m68k-elf/lib/m5208\libc.a(lib_a-findfp.o)
                0x00014778                __sinit
                0x00014800                _cleanup_r
                0x0001481a                _cleanup
                0x0001482e                __sfmoreglue
                0x00014884                __sfp
 *fill*         0x00014966        0x2 00
 .text          0x00014968      0x3e2 c:/program files/codesourcery/sourcery g++ lite/bin/../lib/gcc/m68k-elf/4.4.1/../../../../m68k-elf/lib/m5208\libc.a(lib_a-freer.o)
                0x00014968                _malloc_trim_r
                0x00014a56                _free_r
 *fill*         0x00014d4a        0x2 00
 .text          0x00014d4c       0xd4 c:/program files/codesourcery/sourcery g++ lite/bin/../lib/gcc/m68k-elf/4.4.1/../../../../m68k-elf/lib/m5208\libc.a(lib_a-fwalk.o)
                0x00014d4c                _fwalk
                0x00014db4                _fwalk_reent
 .text          0x00014e20      0x176 c:/program files/codesourcery/sourcery g++ lite/bin/../lib/gcc/m68k-elf/4.4.1/../../../../m68k-elf/lib/m5208\libc.a(lib_a-makebuf.o)
                0x00014e20                __smakebuf_r
 *fill*         0x00014f96        0x2 00
 .text          0x00014f98      0x172 c:/program files/codesourcery/sourcery g++ lite/bin/../lib/gcc/m68k-elf/4.4.1/../../../../m68k-elf/lib/m5208\libc.a(lib_a-reent.o)
                0x00014f98                _wrapup_reent
                0x00015000                cleanup_glue
                0x00015036                _reclaim_reent
 *fill*         0x0001510a        0x2 00
 .text          0x0001510c      0x14c c:/program files/codesourcery/sourcery g++ lite/bin/../lib/gcc/m68k-elf/4.4.1/../../../../m68k-elf/lib/m5208\libc.a(lib_a-stdio.o)
                0x0001510c                __sclose
                0x00015124                __sseek
                0x0001517c                __swrite
                0x0001520e                __sread
 .text          0x00015258       0x3c c:/program files/codesourcery/sourcery g++ lite/bin/../lib/gcc/m68k-elf/4.4.1/../../../../m68k-elf/lib/m5208\libc.a(lib_a-writer.o)
                0x00015258                _write_r
 .text          0x00015294       0x32 c:/program files/codesourcery/sourcery g++ lite/bin/../lib/gcc/m68k-elf/4.4.1/../../../../m68k-elf/lib/m5208\libc.a(lib_a-closer.o)
                0x00015294                _close_r
 *fill*         0x000152c6        0x2 00
 .text          0x000152c8       0xf6 c:/program files/codesourcery/sourcery g++ lite/bin/../lib/gcc/m68k-elf/4.4.1/../../../../m68k-elf/lib/m5208\libc.a(lib_a-fclose.o)
                0x000152c8                _fclose_r
                0x000153a8                fclose
 *fill*         0x000153be        0x2 00
 .text          0x000153c0       0x36 c:/program files/codesourcery/sourcery g++ lite/bin/../lib/gcc/m68k-elf/4.4.1/../../../../m68k-elf/lib/m5208\libc.a(lib_a-fstatr.o)
                0x000153c0                _fstat_r
 *fill*         0x000153f6        0x2 00
 .text          0x000153f8       0x32 c:/program files/codesourcery/sourcery g++ lite/bin/../lib/gcc/m68k-elf/4.4.1/../../../../m68k-elf/lib/m5208\libc.a(lib_a-isattyr.o)
                0x000153f8                _isatty_r
 *fill*         0x0001542a        0x2 00
 .text          0x0001542c       0x3c c:/program files/codesourcery/sourcery g++ lite/bin/../lib/gcc/m68k-elf/4.4.1/../../../../m68k-elf/lib/m5208\libc.a(lib_a-lseekr.o)
                0x0001542c                _lseek_r
 .text          0x00015468       0x3c c:/program files/codesourcery/sourcery g++ lite/bin/../lib/gcc/m68k-elf/4.4.1/../../../../m68k-elf/lib/m5208\libc.a(lib_a-readr.o)
                0x00015468                _read_r
 .text          0x000154a4       0xbc c:/program files/codesourcery/sourcery g++ lite/bin/../lib/gcc/m68k-elf/4.4.1/../../../../m68k-elf/lib/m5208\libcs3.a(start_c.o)
                0x000154a4                __cs3_start_c
 .text          0x00015560        0x0 c:/program files/codesourcery/sourcery g++ lite/bin/../lib/gcc/m68k-elf/4.4.1/../../../../m68k-elf/lib/m5208\libcs3.a(m52235evb-reset.o)
 .text          0x00015560       0x16 c:/program files/codesourcery/sourcery g++ lite/bin/../lib/gcc/m68k-elf/4.4.1/../../../../m68k-elf/lib/m5208\libcs3hosted.a(hosted-_exit.o)
                0x00015560                _exit
 *fill*         0x00015576        0x2 00
 .text          0x00015578       0x40 c:/program files/codesourcery/sourcery g++ lite/bin/../lib/gcc/m68k-elf/4.4.1/../../../../m68k-elf/lib/m5208\libcs3hosted.a(hosted-close.o)
                0x00015578                close
 .text          0x000155b8       0x56 c:/program files/codesourcery/sourcery g++ lite/bin/../lib/gcc/m68k-elf/4.4.1/../../../../m68k-elf/lib/m5208\libcs3hosted.a(hosted-fstat.o)
                0x000155b8                fstat
 *fill*         0x0001560e        0x2 00
 .text          0x00015610       0x40 c:/program files/codesourcery/sourcery g++ lite/bin/../lib/gcc/m68k-elf/4.4.1/../../../../m68k-elf/lib/m5208\libcs3hosted.a(hosted-isatty.o)
                0x00015610                isatty
 .text          0x00015650       0x60 c:/program files/codesourcery/sourcery g++ lite/bin/../lib/gcc/m68k-elf/4.4.1/../../../../m68k-elf/lib/m5208\libcs3hosted.a(hosted-lseek.o)
                0x00015650                lseek
 .text          0x000156b0       0x4c c:/program files/codesourcery/sourcery g++ lite/bin/../lib/gcc/m68k-elf/4.4.1/../../../../m68k-elf/lib/m5208\libcs3hosted.a(hosted-read.o)
                0x000156b0                read
 .text          0x000156fc       0x50 c:/program files/codesourcery/sourcery g++ lite/bin/../lib/gcc/m68k-elf/4.4.1/../../../../m68k-elf/lib/m5208\libcs3hosted.a(hosted-sbrk.o)
                0x000156fc                sbrk
 .text          0x0001574c      0x184 c:/program files/codesourcery/sourcery g++ lite/bin/../lib/gcc/m68k-elf/4.4.1/../../../../m68k-elf/lib/m5208\libcs3hosted.a(hosted-gdb.o)
                0x0001574c                __cs3_hosted_to_gdb_mode_t
                0x000157c6                __cs3_hosted_to_gdb_open_flags
                0x00015814                __cs3_hosted_to_gdb_lseek_flags
                0x0001583a                __cs3_hosted_from_gdb_stat
                0x00015896                __cs3_hosted_from_gdb_timeval
                0x000158ae                __cs3_hosted_from_gdb_errno
 .text          0x000158d0       0x14 c:/program files/codesourcery/sourcery g++ lite/bin/../lib/gcc/m68k-elf/4.4.1/../../../../m68k-elf/lib/m5208\libcs3hosted.a(hosted-start.o)
                0x000158d0                _start
 .text          0x000158e4        0xc c:/program files/codesourcery/sourcery g++ lite/bin/../lib/gcc/m68k-elf/4.4.1/../../../../m68k-elf/lib/m5208\libcs3coldfire.a(coldfire-vector.o)
 .text          0x000158f0        0xa c:/program files/codesourcery/sourcery g++ lite/bin/../lib/gcc/m68k-elf/4.4.1/../../../../m68k-elf/lib/m5208\libcs3coldfire.a(coldfire_isr_other_interrupt.o)
                0x000158f0                __cs3_isr_interrupt_181
                0x000158f0                __cs3_isr_interrupt_194
                0x000158f0                __cs3_isr_interrupt_74
                0x000158f0                __cs3_isr_interrupt_157
                0x000158f0                __cs3_isr_interrupt_133
                0x000158f0                __cs3_isr_interrupt_221
                0x000158f0                __cs3_isr_interrupt_145
                0x000158f0                __cs3_isr_interrupt_100
                0x000158f0                __cs3_isr_interrupt_250
                0x000158f0                __cs3_isr_interrupt_114
                0x000158f0                __cs3_isr_interrupt_152
                0x000158f0                __cs3_isr_interrupt_82
                0x000158f0                __cs3_isr_interrupt_237
                0x000158f0                __cs3_isr_interrupt_143
                0x000158f0                __cs3_isr_interrupt_148
                0x000158f0                __cs3_isr_interrupt_107
                0x000158f0                __cs3_isr_interrupt_103
                0x000158f0                __cs3_isr_interrupt_219
                0x000158f0                __cs3_isr_interrupt_174
                0x000158f0                __cs3_isr_interrupt_220
                0x000158f0                __cs3_isr_interrupt_254
                0x000158f0                __cs3_isr_interrupt_189
                0x000158f0                __cs3_isr_interrupt_233
                0x000158f0                __cs3_isr_interrupt_238
                0x000158f0                __cs3_isr_interrupt_227
                0x000158f0                __cs3_isr_interrupt_162
                0x000158f0                __cs3_isr_interrupt_173
                0x000158f0                __cs3_isr_interrupt_208
                0x000158f0                __cs3_isr_interrupt_244
                0x000158f0                __cs3_isr_interrupt_139
                0x000158f0                __cs3_isr_interrupt_149
                0x000158f0                __cs3_isr_interrupt_201
                0x000158f0                __cs3_isr_interrupt_247
                0x000158f0                __cs3_isr_interrupt_104
                0x000158f0                __cs3_isr_interrupt_155
                0x000158f0                __cs3_isr_interrupt_204
                0x000158f0                __cs3_isr_interrupt_179
                0x000158f0                __cs3_isr_interrupt_112
                0x000158f0                __cs3_isr_interrupt_184
                0x000158f0                __cs3_isr_interrupt_242
                0x000158f0                __cs3_isr_interrupt_84
                0x000158f0                __cs3_isr_interrupt_108
                0x000158f0                __cs3_isr_interrupt_30
                0x000158f0                __cs3_isr_interrupt_158
                0x000158f0                __cs3_isr_interrupt_215
                0x000158f0                __cs3_isr_interrupt_156
                0x000158f0                __cs3_isr_interrupt_115
                0x000158f0                __cs3_isr_interrupt_113
                0x000158f0                __cs3_isr_interrupt_125
                0x000158f0                __cs3_isr_interrupt_27
                0x000158f0                __cs3_isr_interrupt_146
                0x000158f0                __cs3_isr_interrupt_131
                0x000158f0                __cs3_isr_interrupt_101
                0x000158f0                __cs3_isr_interrupt_65
                0x000158f0                __cs3_isr_interrupt_192
                0x000158f0                __cs3_isr_interrupt_141
                0x000158f0                __cs3_isr_interrupt_150
                0x000158f0                __cs3_isr_interrupt_231
                0x000158f0                __cs3_isr_interrupt_154
                0x000158f0                __cs3_isr_interrupt_111
                0x000158f0                __cs3_isr_interrupt_248
                0x000158f0                __cs3_isr_interrupt_191
                0x000158f0                __cs3_isr_interrupt_178
                0x000158f0                __cs3_isr_interrupt_205
                0x000158f0                __cs3_isr_interrupt_17
                0x000158f0                __cs3_isr_interrupt_140
                0x000158f0                __cs3_isr_interrupt_6
                0x000158f0                __cs3_isr_interrupt_226
                0x000158f0                __cs3_isr_interrupt_252
                0x000158f0                __cs3_isr_interrupt_209
                0x000158f0                __cs3_isr_interrupt_202
                0x000158f0                __cs3_isr_interrupt_245
                0x000158f0                __cs3_isr_interrupt_19
                0x000158f0                __cs3_isr_interrupt_171
                0x000158f0                __cs3_isr_interrupt_234
                0x000158f0                __cs3_isr_interrupt_232
                0x000158f0                __cs3_isr_interrupt_239
                0x000158f0                __cs3_isr_interrupt_21
                0x000158f0                __cs3_isr_interrupt_62
                0x000158f0                __cs3_isr_interrupt_240
                0x000158f0                __cs3_isr_interrupt_106
                0x000158f0                __cs3_isr_interrupt_109
                0x000158f0                __cs3_isr_interrupt_190
                0x000158f0                __cs3_isr_interrupt_193
                0x000158f0                __cs3_isr_interrupt_57
                0x000158f0                __cs3_isr_interrupt_168
                0x000158f0                __cs3_isr_interrupt_153
                0x000158f0                __cs3_isr_interrupt_81
                0x000158f0                __cs3_isr_interrupt_110
                0x000158f0                __cs3_isr_interrupt_163
                0x000158f0                __cs3_isr_interrupt_123
                0x000158f0                __cs3_isr_interrupt_185
                0x000158f0                __cs3_isr_interrupt_70
                0x000158f0                __cs3_isr_interrupt_136
                0x000158f0                __cs3_isr_interrupt_134
                0x000158f0                __cs3_isr_interrupt_230
                0x000158f0                __cs3_isr_interrupt_85
                0x000158f0                __cs3_isr_interrupt_186
                0x000158f0                __cs3_isr_interrupt_58
                0x000158f0                __cs3_isr_interrupt_196
                0x000158f0                __cs3_isr_interrupt_132
                0x000158f0                __cs3_isr_interrupt_29
                0x000158f0                __cs3_isr_interrupt_15
                0x000158f0                __cs3_isr_interrupt_224
                0x000158f0                __cs3_isr_interrupt_207
                0x000158f0                __cs3_isr_interrupt_182
                0x000158f0                __cs3_isr_interrupt_127
                0x000158f0                __cs3_isr_interrupt_255
                0x000158f0                __cs3_isr_interrupt_217
                0x000158f0                __cs3_isr_interrupt_128
                0x000158f0                __cs3_isr_interrupt_212
                0x000158f0                __cs3_isr_interrupt_210
                0x000158f0                __cs3_isr_interrupt_188
                0x000158f0                __cs3_isr_interrupt_117
                0x000158f0                __cs3_isr_interrupt_144
                0x000158f0                __cs3_isr_interrupt_175
                0x000158f0                __cs3_isr_interrupt_172
                0x000158f0                __cs3_isr_interrupt_83
                0x000158f0                __cs3_isr_interrupt_253
                0x000158f0                __cs3_isr_interrupt_73
                0x000158f0                __cs3_isr_interrupt_75
                0x000158f0                __cs3_isr_interrupt_228
                0x000158f0                __cs3_isr_interrupt_169
                0x000158f0                __cs3_isr_interrupt_7
                0x000158f0                __cs3_isr_interrupt_124
                0x000158f0                __cs3_isr_interrupt_170
                0x000158f0                __cs3_isr_interrupt_22
                0x000158f0                __cs3_isr_interrupt_63
                0x000158f0                __cs3_isr_interrupt_183
                0x000158f0                __cs3_isr_interrupt_161
                0x000158f0                __cs3_isr_interrupt_137
                0x000158f0                __cs3_isr_interrupt_31
                0x000158f0                __cs3_isr_interrupt_195
                0x000158f0                __cs3_isr_interrupt_229
                0x000158f0                __cs3_isr_interrupt_243
                0x000158f0                __cs3_isr_interrupt_200
                0x000158f0                __cs3_isr_interrupt_187
                0x000158f0                __cs3_isr_interrupt_236
                0x000158f0                __cs3_isr_interrupt_151
                0x000158f0                __cs3_isr_interrupt_105
                0x000158f0                __cs3_isr_interrupt_199
                0x000158f0                __cs3_isr_interrupt_166
                0x000158f0                __cs3_isr_interrupt_121
                0x000158f0                __cs3_isr_interrupt_71
                0x000158f0                __cs3_isr_interrupt_20
                0x000158f0                __cs3_isr_interrupt_218
                0x000158f0                __cs3_isr_interrupt_213
                0x000158f0                __cs3_isr_interrupt_86
                0x000158f0                __cs3_isr_interrupt_138
                0x000158f0                __cs3_isr_interrupt_180
                0x000158f0                __cs3_isr_interrupt_225
                0x000158f0                __cs3_isr_interrupt_59
                0x000158f0                __cs3_isr_interrupt_56
                0x000158f0                __cs3_isr_interrupt_249
                0x000158f0                __cs3_isr_interrupt_167
                0x000158f0                __cs3_isr_interrupt_206
                0x000158f0                __cs3_isr_interrupt_122
                0x000158f0                __cs3_isr_interrupt_147
                0x000158f0                __cs3_isr_interrupt_25
                0x000158f0                __cs3_isr_interrupt_159
                0x000158f0                __cs3_isr_interrupt_102
                0x000158f0                __cs3_isr_interrupt_142
                0x000158f0                __cs3_isr_interrupt_16
                0x000158f0                __cs3_isr_interrupt_176
                0x000158f0                __cs3_isr_interrupt_135
                0x000158f0                __cs3_isr_interrupt_130
                0x000158f0                __cs3_isr_interrupt_60
                0x000158f0                __cs3_isr_interrupt_116
                0x000158f0                __cs3_isr_interrupt_222
                0x000158f0                __cs3_isr_interrupt_28
                0x000158f0                __cs3_isr_interrupt_177
                0x000158f0                __cs3_isr_interrupt_165
                0x000158f0                __cs3_isr_interrupt_160
                0x000158f0                __cs3_isr_interrupt_120
                0x000158f0                __cs3_isr_interrupt_67
                0x000158f0                __cs3_isr_interrupt_198
                0x000158f0                __cs3_isr_interrupt_66
                0x000158f0                __cs3_isr_interrupt_129
                0x000158f0                __cs3_isr_interrupt_76
                0x000158f0                __cs3_isr_interrupt_214
                0x000158f0                __cs3_isr_interrupt_69
                0x000158f0                __cs3_isr_interrupt_26
                0x000158f0                __cs3_isr_other_interrupt
                0x000158f0                __cs3_isr_interrupt_18
                0x000158f0                __cs3_isr_interrupt_241
                0x000158f0                __cs3_isr_interrupt_235
                0x000158f0                __cs3_isr_interrupt_216
                0x000158f0                __cs3_isr_interrupt_211
                0x000158f0                __cs3_isr_interrupt_246
                0x000158f0                __cs3_isr_interrupt_118
                0x000158f0                __cs3_isr_interrupt_223
                0x000158f0                __cs3_isr_interrupt_203
                0x000158f0                __cs3_isr_interrupt_126
                0x000158f0                __cs3_isr_interrupt_197
                0x000158f0                __cs3_isr_interrupt_23
                0x000158f0                __cs3_isr_interrupt_64
                0x000158f0                __cs3_isr_interrupt_251
                0x000158f0                __cs3_isr_interrupt_164
                0x000158f0                __cs3_isr_interrupt_72
 *fill*         0x000158fa        0x2 00
 .text          0x000158fc        0xa c:/program files/codesourcery/sourcery g++ lite/bin/../lib/gcc/m68k-elf/4.4.1/../../../../m68k-elf/lib/m5208\libcs3coldfire.a(coldfire_isr_unimplemented_opcode.o)
                0x000158fc                __cs3_isr_unimplemented_line_a_opcode
                0x000158fc                __cs3_isr_unimplemented_line_f_opcode
                0x000158fc                __cs3_isr_unimplemented_opcode
 *fill*         0x00015906        0x2 00
 .text          0x00015908        0xa c:/program files/codesourcery/sourcery g++ lite/bin/../lib/gcc/m68k-elf/4.4.1/../../../../m68k-elf/lib/m5208\libcs3coldfire.a(coldfire_isr_breakpoint_debug_interrupt.o)
                0x00015908                __cs3_isr_pc_breakpoint_debug_interrupt
                0x00015908                __cs3_isr_non_pc_breakpoint_debug_interrupt
                0x00015908                __cs3_isr_breakpoint_debug_interrupt
 *fill*         0x00015912        0x2 00
 .text          0x00015914        0xa c:/program files/codesourcery/sourcery g++ lite/bin/../lib/gcc/m68k-elf/4.4.1/../../../../m68k-elf/lib/m5208\libcs3coldfire.a(coldfire_isr_trap_interrupt.o)
                0x00015914                __cs3_isr_trap7
                0x00015914                __cs3_isr_trap2
                0x00015914                __cs3_isr_trap14
                0x00015914                __cs3_isr_trap13
                0x00015914                __cs3_isr_trap_interrupt
                0x00015914                __cs3_isr_trap8
                0x00015914                __cs3_isr_trap9
                0x00015914                __cs3_isr_trap1
                0x00015914                __cs3_isr_trap4
                0x00015914                __cs3_isr_trap15
                0x00015914                __cs3_isr_trap6
                0x00015914                __cs3_isr_trap10
                0x00015914                __cs3_isr_trap5
                0x00015914                __cs3_isr_trap0
                0x00015914                __cs3_isr_trap3
                0x00015914                __cs3_isr_trap12
                0x00015914                __cs3_isr_trap11
 *fill*         0x0001591e        0x2 00
 .text          0x00015920        0xa c:/program files/codesourcery/sourcery g++ lite/bin/../lib/gcc/m68k-elf/4.4.1/../../../../m68k-elf/lib/m5208\libcs3coldfire.a(coldfire_isr_fp_interrupt.o)
                0x00015920                __cs3_isr_fp_divide_by_zero
                0x00015920                __cs3_isr_fp_interrupt
                0x00015920                __cs3_isr_fp_operand_error
                0x00015920                __cs3_isr_fp_inexact_result
                0x00015920                __cs3_isr_fp_input_not_a_number
                0x00015920                __cs3_isr_fp_overflow
                0x00015920                __cs3_isr_fp_input_denormalized_number
                0x00015920                __cs3_isr_fp_branch_unordered
                0x00015920                __cs3_isr_fp_underflow
 *fill*         0x0001592a        0x2 00
 .text          0x0001592c        0xa c:/program files/codesourcery/sourcery g++ lite/bin/../lib/gcc/m68k-elf/4.4.1/../../../../m68k-elf/lib/m5208\libcs3coldfire.a(coldfire_isr_access_error.o)
                0x0001592c                __cs3_isr_access_error
 *fill*         0x00015936        0x2 00
 .text          0x00015938        0xa c:/program files/codesourcery/sourcery g++ lite/bin/../lib/gcc/m68k-elf/4.4.1/../../../../m68k-elf/lib/m5208\libcs3coldfire.a(coldfire_isr_address_error.o)
                0x00015938                __cs3_isr_address_error
 *fill*         0x00015942        0x2 00
 .text          0x00015944        0xa c:/program files/codesourcery/sourcery g++ lite/bin/../lib/gcc/m68k-elf/4.4.1/../../../../m68k-elf/lib/m5208\libcs3coldfire.a(coldfire_isr_illegal_instruction.o)
                0x00015944                __cs3_isr_illegal_instruction
 *fill*         0x0001594e        0x2 00
 .text          0x00015950        0xa c:/program files/codesourcery/sourcery g++ lite/bin/../lib/gcc/m68k-elf/4.4.1/../../../../m68k-elf/lib/m5208\libcs3coldfire.a(coldfire_isr_divide_by_zero.o)
                0x00015950                __cs3_isr_divide_by_zero
 *fill*         0x0001595a        0x2 00
 .text          0x0001595c        0xa c:/program files/codesourcery/sourcery g++ lite/bin/../lib/gcc/m68k-elf/4.4.1/../../../../m68k-elf/lib/m5208\libcs3coldfire.a(coldfire_isr_privilege_violation.o)
                0x0001595c                __cs3_isr_privilege_violation
 *fill*         0x00015966        0x2 00
 .text          0x00015968        0xa c:/program files/codesourcery/sourcery g++ lite/bin/../lib/gcc/m68k-elf/4.4.1/../../../../m68k-elf/lib/m5208\libcs3coldfire.a(coldfire_isr_trace.o)
                0x00015968                __cs3_isr_trace
 *fill*         0x00015972        0x2 00
 .text          0x00015974        0xa c:/program files/codesourcery/sourcery g++ lite/bin/../lib/gcc/m68k-elf/4.4.1/../../../../m68k-elf/lib/m5208\libcs3coldfire.a(coldfire_isr_format_error.o)
                0x00015974                __cs3_isr_format_error
 *fill*         0x0001597e        0x2 00
 .text          0x00015980        0xa c:/program files/codesourcery/sourcery g++ lite/bin/../lib/gcc/m68k-elf/4.4.1/../../../../m68k-elf/lib/m5208\libcs3coldfire.a(coldfire_isr_spurious_interrupt.o)
                0x00015980                __cs3_isr_spurious_interrupt
 *fill*         0x0001598a        0x2 00
 .text          0x0001598c        0xa c:/program files/codesourcery/sourcery g++ lite/bin/../lib/gcc/m68k-elf/4.4.1/../../../../m68k-elf/lib/m5208\libcs3coldfire.a(coldfire_isr_unsupported_instruction.o)
                0x0001598c                __cs3_isr_unsupported_instruction
 *fill*         0x00015996        0x2 00
 .text          0x00015998        0xe c:/program files/codesourcery/sourcery g++ lite/bin/../lib/gcc/m68k-elf/4.4.1/../../../../m68k-elf/lib/m5208\libc.a(lib_a-errno.o)
                0x00015998                __errno
 *fill*         0x000159a6        0x2 00
 .text          0x000159a8       0x5c c:/program files/codesourcery/sourcery g++ lite/bin/../lib/gcc/m68k-elf/4.4.1/../../../../m68k-elf/lib/m5208\libc.a(lib_a-init.o)
                0x000159a8                __libc_init_array
 .text          0x00015a04        0x0 c:/program files/codesourcery/sourcery g++ lite/bin/../lib/gcc/m68k-elf/4.4.1/../../../../m68k-elf/lib/m5208\libcs3.a(heap.o)
                0x00015a04                . = ALIGN (0x4)
 *crtbegin.o(.jcr)
 *(EXCLUDE_FILE(*crtend.o) .jcr)
 *crtend.o(.jcr)
                0x00015a04                . = ALIGN (0x4)
 *(.gcc_except_table .gcc_except_table.*)

.eh_frame_hdr
 *(.eh_frame_hdr)

.eh_frame       0x00015a04     0x3ac0
 *(.eh_frame)
 .eh_frame      0x00015a04      0x170 ./bin/main.o
 .eh_frame      0x00015b74      0x19c ./bin/uart0.o
                                0x1b4 (size before relaxing)
 .eh_frame      0x00015d10      0x19c ./bin/uart1.o
                                0x1b4 (size before relaxing)
 .eh_frame      0x00015eac      0x19c ./bin/uart2.o
                                0x1b4 (size before relaxing)
 .eh_frame      0x00016048      0x2ec ./bin/LCD.o
                                0x304 (size before relaxing)
 .eh_frame      0x00016334       0x5c ./bin/klavesnica.o
                                 0x74 (size before relaxing)
 .eh_frame      0x00016390       0x7c ./bin/flashUtilities.o
                                 0x94 (size before relaxing)
 .eh_frame      0x0001640c      0x1f4 ./bin/riadenie.o
                                0x20c (size before relaxing)
 .eh_frame      0x00016600      0x20c ./bin/webcam.o
                                0x224 (size before relaxing)
 .eh_frame      0x0001680c       0x94 ./bin/kom_modul.o
                                 0xac (size before relaxing)
 .eh_frame      0x000168a0       0x44 ./bin/rfid_reader.o
                                 0x5c (size before relaxing)
 .eh_frame      0x000168e4       0x68 ./bin/ParTest.o
                                 0x80 (size before relaxing)
 .eh_frame      0x0001694c       0x40 ./bin/flash.o
                                 0x58 (size before relaxing)
 .eh_frame      0x0001698c       0x48 ./bin/FreeRTOS_Tick_Setup.o
                                 0x60 (size before relaxing)
 .eh_frame      0x000169d4       0x78 ./bin/PollQ.o
                                 0x90 (size before relaxing)
 .eh_frame      0x00016a4c       0x74 ./bin/semtest.o
                                 0x8c (size before relaxing)
 .eh_frame      0x00016ac0      0x100 ./bin/GenQTest.o
                                0x118 (size before relaxing)
 .eh_frame      0x00016bc0       0xd4 ./bin/QPeek.o
                                 0xec (size before relaxing)
 .eh_frame      0x00016c94      0x31c ./bin/FEC.o
                                0x334 (size before relaxing)
 .eh_frame      0x00016fb0       0xb0 ./bin/blocktim.o
                                 0xc8 (size before relaxing)
 .eh_frame      0x00017060       0x98 ./bin/recmutex.o
                                 0xb0 (size before relaxing)
 .eh_frame      0x000170f8      0x408 ./bin/console_reader.o
                                0x420 (size before relaxing)
 .eh_frame      0x00017500      0x124 ./bin/printf-stdarg.o
                                0x13c (size before relaxing)
 .eh_frame      0x00017624       0xa0 ./bin/port.o
                                 0xb8 (size before relaxing)
 .eh_frame      0x000176c4       0x78 ./bin/list.o
                                 0x90 (size before relaxing)
 .eh_frame      0x0001773c      0x478 ./bin/tasks.o
                                0x490 (size before relaxing)
 .eh_frame      0x00017bb4      0x2a8 ./bin/queue.o
                                0x2c0 (size before relaxing)
 .eh_frame      0x00017e5c       0x60 ./bin/heap_1.o
                                 0x78 (size before relaxing)
 .eh_frame      0x00017ebc       0x60 ./bin/timer.o
                                 0x78 (size before relaxing)
 .eh_frame      0x00017f1c      0x210 ./bin/uip.o
                                0x228 (size before relaxing)
 .eh_frame      0x0001812c       0xbc ./bin/uip_arp.o
                                 0xd4 (size before relaxing)
 .eh_frame      0x000181e8       0x18 ./bin/uiplib.o
                                 0x30 (size before relaxing)
 .eh_frame      0x00018200       0x28 ./bin/uip-split.o
                                 0x40 (size before relaxing)
 .eh_frame      0x00018228      0x170 ./bin/psock.o
                                0x188 (size before relaxing)
 .eh_frame      0x00018398       0x88 ./bin/uIP_Task.o
                                 0xa0 (size before relaxing)
 .eh_frame      0x00018420      0x1b4 ./bin/httpd.o
                                0x1cc (size before relaxing)
 .eh_frame      0x000185d4      0x198 ./bin/httpd-cgi.o
                                0x1b0 (size before relaxing)
 .eh_frame      0x0001876c       0x7c ./bin/httpd-fs.o
                                 0x94 (size before relaxing)
 .eh_frame      0x000187e8       0x28 c:/program files/codesourcery/sourcery g++ lite/bin/../lib/gcc/m68k-elf/4.4.1/m5208\libgcc.a(_fixunssfsi.o)
                                 0x40 (size before relaxing)
 .eh_frame      0x00018810      0x130 c:/program files/codesourcery/sourcery g++ lite/bin/../lib/gcc/m68k-elf/4.4.1/m5208\libgcc.a(fpgnulib.o)
                                0x148 (size before relaxing)
 .eh_frame      0x00018940       0x1c c:/program files/codesourcery/sourcery g++ lite/bin/../lib/gcc/m68k-elf/4.4.1/../../../../m68k-elf/lib/m5208\libc.a(lib_a-atexit.o)
                                 0x34 (size before relaxing)
 .eh_frame      0x0001895c       0x38 c:/program files/codesourcery/sourcery g++ lite/bin/../lib/gcc/m68k-elf/4.4.1/../../../../m68k-elf/lib/m5208\libc.a(lib_a-atoi.o)
                                 0x50 (size before relaxing)
 .eh_frame      0x00018994       0x20 c:/program files/codesourcery/sourcery g++ lite/bin/../lib/gcc/m68k-elf/4.4.1/../../../../m68k-elf/lib/m5208\libc.a(lib_a-exit.o)
                                 0x38 (size before relaxing)
 .eh_frame      0x000189b4       0x20 c:/program files/codesourcery/sourcery g++ lite/bin/../lib/gcc/m68k-elf/4.4.1/../../../../m68k-elf/lib/m5208\libc.a(lib_a-memcmp.o)
                                 0x38 (size before relaxing)
 .eh_frame      0x000189d4       0x40 c:/program files/codesourcery/sourcery g++ lite/bin/../lib/gcc/m68k-elf/4.4.1/../../../../m68k-elf/lib/m5208\libc.a(lib_a-puts.o)
                                 0x58 (size before relaxing)
 .eh_frame      0x00018a14       0x20 c:/program files/codesourcery/sourcery g++ lite/bin/../lib/gcc/m68k-elf/4.4.1/../../../../m68k-elf/lib/m5208\libc.a(lib_a-strcat.o)
                                 0x38 (size before relaxing)
 .eh_frame      0x00018a34       0x20 c:/program files/codesourcery/sourcery g++ lite/bin/../lib/gcc/m68k-elf/4.4.1/../../../../m68k-elf/lib/m5208\libc.a(lib_a-strchr.o)
                                 0x38 (size before relaxing)
 .eh_frame      0x00018a54       0x18 c:/program files/codesourcery/sourcery g++ lite/bin/../lib/gcc/m68k-elf/4.4.1/../../../../m68k-elf/lib/m5208\libc.a(lib_a-strcmp.o)
                                 0x30 (size before relaxing)
 .eh_frame      0x00018a6c       0x18 c:/program files/codesourcery/sourcery g++ lite/bin/../lib/gcc/m68k-elf/4.4.1/../../../../m68k-elf/lib/m5208\libc.a(lib_a-strcpy.o)
                                 0x30 (size before relaxing)
 .eh_frame      0x00018a84       0x18 c:/program files/codesourcery/sourcery g++ lite/bin/../lib/gcc/m68k-elf/4.4.1/../../../../m68k-elf/lib/m5208\libc.a(lib_a-strlen.o)
                                 0x30 (size before relaxing)
 .eh_frame      0x00018a9c       0x1c c:/program files/codesourcery/sourcery g++ lite/bin/../lib/gcc/m68k-elf/4.4.1/../../../../m68k-elf/lib/m5208\libc.a(lib_a-strncmp.o)
                                 0x34 (size before relaxing)
 .eh_frame      0x00018ab8       0x20 c:/program files/codesourcery/sourcery g++ lite/bin/../lib/gcc/m68k-elf/4.4.1/../../../../m68k-elf/lib/m5208\libc.a(lib_a-strncpy.o)
                                 0x38 (size before relaxing)
 .eh_frame      0x00018ad8       0x24 c:/program files/codesourcery/sourcery g++ lite/bin/../lib/gcc/m68k-elf/4.4.1/../../../../m68k-elf/lib/m5208\libc.a(lib_a-strrchr.o)
                                 0x3c (size before relaxing)
 .eh_frame      0x00018afc       0x1c c:/program files/codesourcery/sourcery g++ lite/bin/../lib/gcc/m68k-elf/4.4.1/../../../../m68k-elf/lib/m5208\libc.a(lib_a-strtok.o)
                                 0x34 (size before relaxing)
 .eh_frame      0x00018b18       0x3c c:/program files/codesourcery/sourcery g++ lite/bin/../lib/gcc/m68k-elf/4.4.1/../../../../m68k-elf/lib/m5208\libc.a(lib_a-strtok_r.o)
                                 0x54 (size before relaxing)
 .eh_frame      0x00018b54       0x48 c:/program files/codesourcery/sourcery g++ lite/bin/../lib/gcc/m68k-elf/4.4.1/../../../../m68k-elf/lib/m5208\libc.a(lib_a-strtol.o)
                                 0x60 (size before relaxing)
 .eh_frame      0x00018b9c       0x24 c:/program files/codesourcery/sourcery g++ lite/bin/../lib/gcc/m68k-elf/4.4.1/../../../../m68k-elf/lib/m5208\libc.a(lib_a-__atexit.o)
                                 0x3c (size before relaxing)
 .eh_frame      0x00018bc0       0x54 c:/program files/codesourcery/sourcery g++ lite/bin/../lib/gcc/m68k-elf/4.4.1/../../../../m68k-elf/lib/m5208\libc.a(lib_a-__call_atexit.o)
                                 0x6c (size before relaxing)
 .eh_frame      0x00018c14       0x1c c:/program files/codesourcery/sourcery g++ lite/bin/../lib/gcc/m68k-elf/4.4.1/../../../../m68k-elf/lib/m5208\libc.a(lib_a-fini.o)
                                 0x34 (size before relaxing)
 .eh_frame      0x00018c30       0x5c c:/program files/codesourcery/sourcery g++ lite/bin/../lib/gcc/m68k-elf/4.4.1/../../../../m68k-elf/lib/m5208\libc.a(lib_a-fvwrite.o)
                                 0x74 (size before relaxing)
 .eh_frame      0x00018c8c       0x40 c:/program files/codesourcery/sourcery g++ lite/bin/../lib/gcc/m68k-elf/4.4.1/../../../../m68k-elf/lib/m5208\libc.a(lib_a-mallocr.o)
                                 0x58 (size before relaxing)
 .eh_frame      0x00018ccc       0x20 c:/program files/codesourcery/sourcery g++ lite/bin/../lib/gcc/m68k-elf/4.4.1/../../../../m68k-elf/lib/m5208\libc.a(lib_a-memchr.o)
                                 0x38 (size before relaxing)
 .eh_frame      0x00018cec       0x24 c:/program files/codesourcery/sourcery g++ lite/bin/../lib/gcc/m68k-elf/4.4.1/../../../../m68k-elf/lib/m5208\libc.a(lib_a-memmove.o)
                                 0x3c (size before relaxing)
 .eh_frame      0x00018d10       0x30 c:/program files/codesourcery/sourcery g++ lite/bin/../lib/gcc/m68k-elf/4.4.1/../../../../m68k-elf/lib/m5208\libc.a(lib_a-mlock.o)
                                 0x48 (size before relaxing)
 .eh_frame      0x00018d40       0x5c c:/program files/codesourcery/sourcery g++ lite/bin/../lib/gcc/m68k-elf/4.4.1/../../../../m68k-elf/lib/m5208\libc.a(lib_a-reallocr.o)
                                 0x74 (size before relaxing)
 .eh_frame      0x00018d9c       0x1c c:/program files/codesourcery/sourcery g++ lite/bin/../lib/gcc/m68k-elf/4.4.1/../../../../m68k-elf/lib/m5208\libc.a(lib_a-sbrkr.o)
                                 0x34 (size before relaxing)
 .eh_frame      0x00018db8       0x24 c:/program files/codesourcery/sourcery g++ lite/bin/../lib/gcc/m68k-elf/4.4.1/../../../../m68k-elf/lib/m5208\libc.a(lib_a-wsetup.o)
                                 0x3c (size before relaxing)
 .eh_frame      0x00018ddc       0x4c c:/program files/codesourcery/sourcery g++ lite/bin/../lib/gcc/m68k-elf/4.4.1/../../../../m68k-elf/lib/m5208\libc.a(lib_a-fflush.o)
                                 0x64 (size before relaxing)
 .eh_frame      0x00018e28       0xc4 c:/program files/codesourcery/sourcery g++ lite/bin/../lib/gcc/m68k-elf/4.4.1/../../../../m68k-elf/lib/m5208\libc.a(lib_a-findfp.o)
                                 0xdc (size before relaxing)
 .eh_frame      0x00018eec       0x64 c:/program files/codesourcery/sourcery g++ lite/bin/../lib/gcc/m68k-elf/4.4.1/../../../../m68k-elf/lib/m5208\libc.a(lib_a-freer.o)
                                 0x7c (size before relaxing)
 .eh_frame      0x00018f50       0x50 c:/program files/codesourcery/sourcery g++ lite/bin/../lib/gcc/m68k-elf/4.4.1/../../../../m68k-elf/lib/m5208\libc.a(lib_a-fwalk.o)
                                 0x68 (size before relaxing)
 .eh_frame      0x00018fa0       0x28 c:/program files/codesourcery/sourcery g++ lite/bin/../lib/gcc/m68k-elf/4.4.1/../../../../m68k-elf/lib/m5208\libc.a(lib_a-makebuf.o)
                                 0x40 (size before relaxing)
 .eh_frame      0x00018fc8       0x70 c:/program files/codesourcery/sourcery g++ lite/bin/../lib/gcc/m68k-elf/4.4.1/../../../../m68k-elf/lib/m5208\libc.a(lib_a-reent.o)
                                 0x88 (size before relaxing)
 .eh_frame      0x00019038       0x80 c:/program files/codesourcery/sourcery g++ lite/bin/../lib/gcc/m68k-elf/4.4.1/../../../../m68k-elf/lib/m5208\libc.a(lib_a-stdio.o)
                                 0x98 (size before relaxing)
 .eh_frame      0x000190b8       0x1c c:/program files/codesourcery/sourcery g++ lite/bin/../lib/gcc/m68k-elf/4.4.1/../../../../m68k-elf/lib/m5208\libc.a(lib_a-writer.o)
                                 0x34 (size before relaxing)
 .eh_frame      0x000190d4       0x1c c:/program files/codesourcery/sourcery g++ lite/bin/../lib/gcc/m68k-elf/4.4.1/../../../../m68k-elf/lib/m5208\libc.a(lib_a-closer.o)
                                 0x34 (size before relaxing)
 .eh_frame      0x000190f0       0x44 c:/program files/codesourcery/sourcery g++ lite/bin/../lib/gcc/m68k-elf/4.4.1/../../../../m68k-elf/lib/m5208\libc.a(lib_a-fclose.o)
                                 0x5c (size before relaxing)
 .eh_frame      0x00019134       0x1c c:/program files/codesourcery/sourcery g++ lite/bin/../lib/gcc/m68k-elf/4.4.1/../../../../m68k-elf/lib/m5208\libc.a(lib_a-fstatr.o)
                                 0x34 (size before relaxing)
 .eh_frame      0x00019150       0x1c c:/program files/codesourcery/sourcery g++ lite/bin/../lib/gcc/m68k-elf/4.4.1/../../../../m68k-elf/lib/m5208\libc.a(lib_a-isattyr.o)
                                 0x34 (size before relaxing)
 .eh_frame      0x0001916c       0x1c c:/program files/codesourcery/sourcery g++ lite/bin/../lib/gcc/m68k-elf/4.4.1/../../../../m68k-elf/lib/m5208\libc.a(lib_a-lseekr.o)
                                 0x34 (size before relaxing)
 .eh_frame      0x00019188       0x1c c:/program files/codesourcery/sourcery g++ lite/bin/../lib/gcc/m68k-elf/4.4.1/../../../../m68k-elf/lib/m5208\libc.a(lib_a-readr.o)
                                 0x34 (size before relaxing)
 .eh_frame      0x000191a4       0x28 c:/program files/codesourcery/sourcery g++ lite/bin/../lib/gcc/m68k-elf/4.4.1/../../../../m68k-elf/lib/m5208\libcs3.a(start_c.o)
                                 0x40 (size before relaxing)
 .eh_frame      0x000191cc       0x18 c:/program files/codesourcery/sourcery g++ lite/bin/../lib/gcc/m68k-elf/4.4.1/../../../../m68k-elf/lib/m5208\libcs3hosted.a(hosted-_exit.o)
                                 0x30 (size before relaxing)
 .eh_frame      0x000191e4       0x20 c:/program files/codesourcery/sourcery g++ lite/bin/../lib/gcc/m68k-elf/4.4.1/../../../../m68k-elf/lib/m5208\libcs3hosted.a(hosted-close.o)
                                 0x38 (size before relaxing)
 .eh_frame      0x00019204       0x24 c:/program files/codesourcery/sourcery g++ lite/bin/../lib/gcc/m68k-elf/4.4.1/../../../../m68k-elf/lib/m5208\libcs3hosted.a(hosted-fstat.o)
                                 0x3c (size before relaxing)
 .eh_frame      0x00019228       0x20 c:/program files/codesourcery/sourcery g++ lite/bin/../lib/gcc/m68k-elf/4.4.1/../../../../m68k-elf/lib/m5208\libcs3hosted.a(hosted-isatty.o)
                                 0x38 (size before relaxing)
 .eh_frame      0x00019248       0x24 c:/program files/codesourcery/sourcery g++ lite/bin/../lib/gcc/m68k-elf/4.4.1/../../../../m68k-elf/lib/m5208\libcs3hosted.a(hosted-lseek.o)
                                 0x3c (size before relaxing)
 .eh_frame      0x0001926c       0x20 c:/program files/codesourcery/sourcery g++ lite/bin/../lib/gcc/m68k-elf/4.4.1/../../../../m68k-elf/lib/m5208\libcs3hosted.a(hosted-read.o)
                                 0x38 (size before relaxing)
 .eh_frame      0x0001928c       0x18 c:/program files/codesourcery/sourcery g++ lite/bin/../lib/gcc/m68k-elf/4.4.1/../../../../m68k-elf/lib/m5208\libcs3hosted.a(hosted-sbrk.o)
                                 0x30 (size before relaxing)
 .eh_frame      0x000192a4       0x98 c:/program files/codesourcery/sourcery g++ lite/bin/../lib/gcc/m68k-elf/4.4.1/../../../../m68k-elf/lib/m5208\libcs3hosted.a(hosted-gdb.o)
                                 0xb0 (size before relaxing)
 .eh_frame      0x0001933c       0x18 c:/program files/codesourcery/sourcery g++ lite/bin/../lib/gcc/m68k-elf/4.4.1/../../../../m68k-elf/lib/m5208\libcs3coldfire.a(coldfire_isr_other_interrupt.o)
                                 0x30 (size before relaxing)
 .eh_frame      0x00019354       0x18 c:/program files/codesourcery/sourcery g++ lite/bin/../lib/gcc/m68k-elf/4.4.1/../../../../m68k-elf/lib/m5208\libcs3coldfire.a(coldfire_isr_unimplemented_opcode.o)
                                 0x30 (size before relaxing)
 .eh_frame      0x0001936c       0x18 c:/program files/codesourcery/sourcery g++ lite/bin/../lib/gcc/m68k-elf/4.4.1/../../../../m68k-elf/lib/m5208\libcs3coldfire.a(coldfire_isr_breakpoint_debug_interrupt.o)
                                 0x30 (size before relaxing)
 .eh_frame      0x00019384       0x18 c:/program files/codesourcery/sourcery g++ lite/bin/../lib/gcc/m68k-elf/4.4.1/../../../../m68k-elf/lib/m5208\libcs3coldfire.a(coldfire_isr_trap_interrupt.o)
                                 0x30 (size before relaxing)
 .eh_frame      0x0001939c       0x18 c:/program files/codesourcery/sourcery g++ lite/bin/../lib/gcc/m68k-elf/4.4.1/../../../../m68k-elf/lib/m5208\libcs3coldfire.a(coldfire_isr_fp_interrupt.o)
                                 0x30 (size before relaxing)
 .eh_frame      0x000193b4       0x18 c:/program files/codesourcery/sourcery g++ lite/bin/../lib/gcc/m68k-elf/4.4.1/../../../../m68k-elf/lib/m5208\libcs3coldfire.a(coldfire_isr_access_error.o)
                                 0x30 (size before relaxing)
 .eh_frame      0x000193cc       0x18 c:/program files/codesourcery/sourcery g++ lite/bin/../lib/gcc/m68k-elf/4.4.1/../../../../m68k-elf/lib/m5208\libcs3coldfire.a(coldfire_isr_address_error.o)
                                 0x30 (size before relaxing)
 .eh_frame      0x000193e4       0x18 c:/program files/codesourcery/sourcery g++ lite/bin/../lib/gcc/m68k-elf/4.4.1/../../../../m68k-elf/lib/m5208\libcs3coldfire.a(coldfire_isr_illegal_instruction.o)
                                 0x30 (size before relaxing)
 .eh_frame      0x000193fc       0x18 c:/program files/codesourcery/sourcery g++ lite/bin/../lib/gcc/m68k-elf/4.4.1/../../../../m68k-elf/lib/m5208\libcs3coldfire.a(coldfire_isr_divide_by_zero.o)
                                 0x30 (size before relaxing)
 .eh_frame      0x00019414       0x18 c:/program files/codesourcery/sourcery g++ lite/bin/../lib/gcc/m68k-elf/4.4.1/../../../../m68k-elf/lib/m5208\libcs3coldfire.a(coldfire_isr_privilege_violation.o)
                                 0x30 (size before relaxing)
 .eh_frame      0x0001942c       0x18 c:/program files/codesourcery/sourcery g++ lite/bin/../lib/gcc/m68k-elf/4.4.1/../../../../m68k-elf/lib/m5208\libcs3coldfire.a(coldfire_isr_trace.o)
                                 0x30 (size before relaxing)
 .eh_frame      0x00019444       0x18 c:/program files/codesourcery/sourcery g++ lite/bin/../lib/gcc/m68k-elf/4.4.1/../../../../m68k-elf/lib/m5208\libcs3coldfire.a(coldfire_isr_format_error.o)
                                 0x30 (size before relaxing)
 .eh_frame      0x0001945c       0x18 c:/program files/codesourcery/sourcery g++ lite/bin/../lib/gcc/m68k-elf/4.4.1/../../../../m68k-elf/lib/m5208\libcs3coldfire.a(coldfire_isr_spurious_interrupt.o)
                                 0x30 (size before relaxing)
 .eh_frame      0x00019474       0x18 c:/program files/codesourcery/sourcery g++ lite/bin/../lib/gcc/m68k-elf/4.4.1/../../../../m68k-elf/lib/m5208\libcs3coldfire.a(coldfire_isr_unsupported_instruction.o)
                                 0x30 (size before relaxing)
 .eh_frame      0x0001948c       0x18 c:/program files/codesourcery/sourcery g++ lite/bin/../lib/gcc/m68k-elf/4.4.1/../../../../m68k-elf/lib/m5208\libc.a(lib_a-errno.o)
                                 0x30 (size before relaxing)
 .eh_frame      0x000194a4       0x20 c:/program files/codesourcery/sourcery g++ lite/bin/../lib/gcc/m68k-elf/4.4.1/../../../../m68k-elf/lib/m5208\libc.a(lib_a-init.o)
                                 0x38 (size before relaxing)

.rodata         0x000194c4     0x960c
 *(.rodata .rodata.* .gnu.linkonce.r.*)
 .rodata        0x000194c4       0x35 ./bin/main.o
 .rodata.LCD_DATA_Table
                0x000194f9        0x4 ./bin/LCD.o
 .rodata.addrsrow
                0x000194fd        0x2 ./bin/LCD.o
                0x000194fd                addrsrow
 .rodata.konverTab
                0x000194ff       0x10 ./bin/klavesnica.o
                0x000194ff                konverTab
 .rodata        0x0001950f       0xaf ./bin/riadenie.o
 .rodata.commandSSS
                0x000195be       0x28 ./bin/riadenie.o
                0x000195be                commandSSS
 .rodata        0x000195e6       0x23 ./bin/webcam.o
 .rodata        0x00019609       0x6e ./bin/kom_modul.o
 .rodata        0x00019677       0x18 ./bin/rfid_reader.o
 .rodata        0x0001968f        0x5 ./bin/flash.o
 .rodata        0x00019694       0x20 ./bin/PollQ.o
 .rodata        0x000196b4       0x3e ./bin/semtest.o
 .rodata        0x000196f2       0x37 ./bin/GenQTest.o
 .rodata        0x00019729       0x2b ./bin/QPeek.o
 .rodata        0x00019754       0x1f ./bin/blocktim.o
 .rodata        0x00019773       0x1f ./bin/recmutex.o
 .rodata        0x00019792      0x293 ./bin/console_reader.o
 *fill*         0x00019a25        0x1 00
 .rodata.prikazy
                0x00019a26       0xa0 ./bin/console_reader.o
                0x00019a26                prikazy
 .rodata        0x00019ac6        0x7 ./bin/printf-stdarg.o
 .rodata        0x00019acd       0x1a ./bin/tasks.o
 .rodata.ucExpectedStackBytes.3340
                0x00019ae7       0x14 ./bin/tasks.o
 *fill*         0x00019afb        0x1 00
 .rodata.all_ones_addr
                0x00019afc        0x4 ./bin/uip.o
 .rodata.all_zeroes_addr
                0x00019b00        0x4 ./bin/uip.o
 .rodata.broadcast_ethaddr
                0x00019b04        0x6 ./bin/uip_arp.o
 .rodata.broadcast_ipaddr
                0x00019b0a        0x4 ./bin/uip_arp.o
 .rodata        0x00019b0e       0x13 ./bin/psock.o
 .rodata        0x00019b21      0x11c ./bin/httpd-cgi.o
 *fill*         0x00019c3d        0x1 00
 .rodata.file   0x00019c3e        0x8 ./bin/httpd-cgi.o
 .rodata.tcp    0x00019c46        0x8 ./bin/httpd-cgi.o
 .rodata.net    0x00019c4e        0x8 ./bin/httpd-cgi.o
 .rodata.rtos   0x00019c56        0x8 ./bin/httpd-cgi.o
 .rodata.io     0x00019c5e        0x8 ./bin/httpd-cgi.o
 .rodata.closed
                0x00019c66        0x7 ./bin/httpd-cgi.o
 .rodata.syn_rcvd
                0x00019c6d        0x9 ./bin/httpd-cgi.o
 .rodata.syn_sent
                0x00019c76        0x9 ./bin/httpd-cgi.o
 .rodata.established
                0x00019c7f        0xc ./bin/httpd-cgi.o
 .rodata.fin_wait_1
                0x00019c8b        0xb ./bin/httpd-cgi.o
 .rodata.fin_wait_2
                0x00019c96        0xb ./bin/httpd-cgi.o
 .rodata.closing
                0x00019ca1        0x8 ./bin/httpd-cgi.o
 .rodata.time_wait
                0x00019ca9        0xa ./bin/httpd-cgi.o
 .rodata.last_ack
                0x00019cb3        0x9 ./bin/httpd-cgi.o
 .rodata.data_404_html
                0x00019cbc       0xb2 ./bin/httpd-fs.o
 .rodata.data_image_html
                0x00019d6e      0x258 ./bin/httpd-fs.o
 .rodata.data_image_jpg
                0x00019fc6        0xc ./bin/httpd-fs.o
 .rodata.data_index_html
                0x00019fd2      0x1c0 ./bin/httpd-fs.o
 .rodata.data_index_shtml
                0x0001a192      0x362 ./bin/httpd-fs.o
 .rodata.data_io_shtml
                0x0001a4f4      0x320 ./bin/httpd-fs.o
 .rodata.data_logo_jpg
                0x0001a814     0x747e ./bin/httpd-fs.o
 .rodata.data_stats_shtml
                0x00021c92      0x58a ./bin/httpd-fs.o
 .rodata.data_tcp_shtml
                0x0002221c      0x2f5 ./bin/httpd-fs.o
 *fill*         0x00022511        0x1 00
 .rodata.file_404_html
                0x00022512       0x12 ./bin/httpd-fs.o
                0x00022512                file_404_html
 .rodata.file_image_html
                0x00022524       0x12 ./bin/httpd-fs.o
                0x00022524                file_image_html
 .rodata.file_image_jpg
                0x00022536       0x12 ./bin/httpd-fs.o
                0x00022536                file_image_jpg
 .rodata.file_index_html
                0x00022548       0x12 ./bin/httpd-fs.o
                0x00022548                file_index_html
 .rodata.file_index_shtml
                0x0002255a       0x12 ./bin/httpd-fs.o
                0x0002255a                file_index_shtml
 .rodata.file_io_shtml
                0x0002256c       0x12 ./bin/httpd-fs.o
                0x0002256c                file_io_shtml
 .rodata.file_logo_jpg
                0x0002257e       0x12 ./bin/httpd-fs.o
                0x0002257e                file_logo_jpg
 .rodata.file_stats_shtml
                0x00022590       0x12 ./bin/httpd-fs.o
                0x00022590                file_stats_shtml
 .rodata.file_tcp_shtml
                0x000225a2       0x12 ./bin/httpd-fs.o
                0x000225a2                file_tcp_shtml
 .rodata        0x000225b4       0x1a ./bin/httpd-fs.o
 .rodata.http_http
                0x000225ce        0x8 ./bin/http-strings.o
                0x000225ce                http_http
 .rodata.http_200
                0x000225d6        0x5 ./bin/http-strings.o
                0x000225d6                http_200
 .rodata.http_301
                0x000225db        0x5 ./bin/http-strings.o
                0x000225db                http_301
 .rodata.http_302
                0x000225e0        0x5 ./bin/http-strings.o
                0x000225e0                http_302
 .rodata.http_get
                0x000225e5        0x5 ./bin/http-strings.o
                0x000225e5                http_get
 .rodata.http_10
                0x000225ea        0x9 ./bin/http-strings.o
                0x000225ea                http_10
 .rodata.http_11
                0x000225f3        0x9 ./bin/http-strings.o
                0x000225f3                http_11
 .rodata.http_content_type
                0x000225fc        0xf ./bin/http-strings.o
                0x000225fc                http_content_type
 .rodata.http_texthtml
                0x0002260b        0xa ./bin/http-strings.o
                0x0002260b                http_texthtml
 .rodata.http_location
                0x00022615        0xb ./bin/http-strings.o
                0x00022615                http_location
 .rodata.http_host
                0x00022620        0x7 ./bin/http-strings.o
                0x00022620                http_host
 .rodata.http_crnl
                0x00022627        0x3 ./bin/http-strings.o
                0x00022627                http_crnl
 .rodata.http_index_html
                0x0002262a        0xc ./bin/http-strings.o
                0x0002262a                http_index_html
 .rodata.http_404_html
                0x00022636        0xa ./bin/http-strings.o
                0x00022636                http_404_html
 .rodata.http_referer
                0x00022640        0x9 ./bin/http-strings.o
                0x00022640                http_referer
 .rodata.http_header_200
                0x00022649       0x54 ./bin/http-strings.o
                0x00022649                http_header_200
 .rodata.http_header_404
                0x0002269d       0x5b ./bin/http-strings.o
                0x0002269d                http_header_404
 .rodata.http_content_type_plain
                0x000226f8       0x1d ./bin/http-strings.o
                0x000226f8                http_content_type_plain
 .rodata.http_content_type_html
                0x00022715       0x1c ./bin/http-strings.o
                0x00022715                http_content_type_html
 .rodata.http_content_type_css
                0x00022731       0x1b ./bin/http-strings.o
                0x00022731                http_content_type_css
 .rodata.http_content_type_text
                0x0002274c       0x1c ./bin/http-strings.o
                0x0002274c                http_content_type_text
 .rodata.http_content_type_png
                0x00022768       0x1c ./bin/http-strings.o
                0x00022768                http_content_type_png
 .rodata.http_content_type_gif
                0x00022784       0x1c ./bin/http-strings.o
                0x00022784                http_content_type_gif
 .rodata.http_content_type_jpg
                0x000227a0       0x1d ./bin/http-strings.o
                0x000227a0                http_content_type_jpg
 .rodata.http_content_type_binary
                0x000227bd       0x2b ./bin/http-strings.o
                0x000227bd                http_content_type_binary
 .rodata.http_html
                0x000227e8        0x6 ./bin/http-strings.o
                0x000227e8                http_html
 .rodata.http_shtml
                0x000227ee        0x7 ./bin/http-strings.o
                0x000227ee                http_shtml
 .rodata.http_htm
                0x000227f5        0x5 ./bin/http-strings.o
                0x000227f5                http_htm
 .rodata.http_css
                0x000227fa        0x5 ./bin/http-strings.o
                0x000227fa                http_css
 .rodata.http_png
                0x000227ff        0x5 ./bin/http-strings.o
                0x000227ff                http_png
 .rodata.http_gif
                0x00022804        0x5 ./bin/http-strings.o
                0x00022804                http_gif
 .rodata.http_jpg
                0x00022809        0x5 ./bin/http-strings.o
                0x00022809                http_jpg
 .rodata.http_text
                0x0002280e        0x5 ./bin/http-strings.o
                0x0002280e                http_text
 .rodata.http_txt
                0x00022813        0x5 ./bin/http-strings.o
                0x00022813                http_txt
 .rodata        0x00022818        0x4 c:/program files/codesourcery/sourcery g++ lite/bin/../lib/gcc/m68k-elf/4.4.1/../../../../m68k-elf/lib/m5208\libc.a(lib_a-impure.o)
                0x00022818                _global_impure_ptr
 .rodata.str1.1
                0x0002281c        0x2 c:/program files/codesourcery/sourcery g++ lite/bin/../lib/gcc/m68k-elf/4.4.1/../../../../m68k-elf/lib/m5208\libc.a(lib_a-impure.o)
 .rodata.str1.1
                0x0002281e        0x2 c:/program files/codesourcery/sourcery g++ lite/bin/../lib/gcc/m68k-elf/4.4.1/../../../../m68k-elf/lib/m5208\libc.a(lib_a-puts.o)
 .rodata        0x00022820      0x101 c:/program files/codesourcery/sourcery g++ lite/bin/../lib/gcc/m68k-elf/4.4.1/../../../../m68k-elf/lib/m5208\libc.a(lib_a-ctype_.o)
                0x00022820                _ctype_
 *fill*         0x00022921        0x1 00
 .rodata        0x00022922      0x17c c:/program files/codesourcery/sourcery g++ lite/bin/../lib/gcc/m68k-elf/4.4.1/../../../../m68k-elf/lib/m5208\libcs3hosted.a(hosted-gdb.o)
                0x00022aa0                . = ALIGN (0x4)
 *fill*         0x00022a9e        0x2 00
                0x00022aa0                _init = .
                0x00022aa0        0x4 LONG 0x4e560000
 *(.init)
                0x00022aa4        0x2 SHORT 0x4e5e
                0x00022aa6        0x2 SHORT 0x4e75
                0x00022aa8                . = ALIGN (0x4)
                0x00022aa8                __preinit_array_start = .
 *(.preinit_array)
                0x00022aa8                __preinit_array_end = .
                0x00022aa8                . = ALIGN (0x4)
                0x00022aa8                __init_array_start = .
 *(SORT(.init_array.*))
 *(.init_array)
                0x00022aa8                __init_array_end = .
                0x00022aa8                . = ALIGN (0x4)
                0x00022aa8                _fini = .
                0x00022aa8        0x4 LONG 0x4e560000
 *(.fini)
                0x00022aac        0x2 SHORT 0x4e5e
                0x00022aae        0x2 SHORT 0x4e75
                0x00022ab0                . = ALIGN (0x4)
                0x00022ab0                __fini_array_start = .
 *(.fini_array)
 *(SORT(.fini_array.*))
                0x00022ab0                __fini_array_end = .
                0x00022ab0                . = ALIGN (0x4)
 *crtbegin.o(.ctors)
 *(EXCLUDE_FILE(*crtend.o) .ctors)
 *(SORT(.ctors.*))
 .ctors.65535   0x00022ab0        0x4 c:/program files/codesourcery/sourcery g++ lite/bin/../lib/gcc/m68k-elf/4.4.1/../../../../m68k-elf/lib/m5208\libc.a(lib_a-__call_atexit.o)
 .ctors.65535   0x00022ab4        0x4 c:/program files/codesourcery/sourcery g++ lite/bin/../lib/gcc/m68k-elf/4.4.1/../../../../m68k-elf/lib/m5208\libcs3coldfire.a(coldfire-vector.o)
 *crtend.o(.ctors)
                0x00022ab8                . = ALIGN (0x4)
 *crtbegin.o(.dtors)
 *(EXCLUDE_FILE(*crtend.o) .dtors)
 *(SORT(.dtors.*))
 *crtend.o(.dtors)
 *(.lit)
                0x00022ab8                . = ALIGN (0x4)
                0x00022ab8                __cs3_regions = .
                0x00022ab8        0x4 LONG 0x0
                0x00022abc        0x4 LONG 0x22ad0 __cs3_region_init_ram
                0x00022ac0        0x4 LONG 0x20000000 __cs3_region_start_ram
                0x00022ac4        0x4 LONG 0x8c0 __cs3_region_init_size_ram
                0x00022ac8        0x4 LONG 0x5d38 __cs3_region_zero_size_ram
                0x00022acc                __cs3_regions_end = .
                0x00022ad0                . = ALIGN (0x8)
 *fill*         0x00022acc        0x4 00
                0x00022ad0                . = ALIGN (0x8)
 *(.rom)
 *(.rom.b)
                0x00022ad0                _etext = .
                0x0003fbe0                __cs3_region_end_rom = (__cs3_region_start_rom + 0x3fbe0)
                0x0003fbe0                __cs3_region_size_rom = 0x3fbe0

.cs3.ipsbar     0x40000000        0x0
                0x40000000                __cs3_region_start_ipsbar = .
 *(.cs3.region-head.ipsbar)
                0x40000000                . = ALIGN (0x8)
                0x40200000                __cs3_region_end_ipsbar = (__cs3_region_start_ipsbar + 0x200000)
                0x00200000                __cs3_region_size_ipsbar = 0x200000

.data           0x20000000      0x8c0 load address 0x00022ad0
                0x20000000                __cs3_region_start_ram = .
 *(.cs3.region-head.ram)
 *(.got.plt)
 *(.got)
 *(.shdata)
 *(.data .data.* .gnu.linkonce.d.*)
 .data          0x20000000        0x0 ./bin/main.o
 .data.ulRegTest1Counter
                0x20000000        0x4 ./bin/main.o
 .data.ulRegTest2Counter
                0x20000004        0x4 ./bin/main.o
 .data.vykon    0x20000008        0x1 ./bin/main.o
                0x20000008                vykon
 *fill*         0x20000009        0x3 00
 .data          0x2000000c        0x0 ./bin/uart0.o
 .data          0x2000000c        0x0 ./bin/uart1.o
 .data          0x2000000c        0x0 ./bin/uart2.o
 .data          0x2000000c        0x0 ./bin/LCD.o
 .data          0x2000000c        0x0 ./bin/klavesnica.o
 .data          0x2000000c        0x0 ./bin/flashUtilities.o
 .data.flashsemaphoreX
                0x2000000c        0x1 ./bin/flashUtilities.o
                0x2000000c                flashsemaphoreX
 *fill*         0x2000000d        0x1 00
 .data.pRAMfunction.1616
                0x2000000e        0x4 ./bin/flashUtilities.o
 *fill*         0x20000012        0x2 00
 .data          0x20000014        0x0 ./bin/riadenie.o
 .data          0x20000014        0x0 ./bin/webcam.o
 .data.PACKAGE_SIZE
                0x20000014        0x4 ./bin/webcam.o
                0x20000014                PACKAGE_SIZE
 .data.last_length
                0x20000018        0x4 ./bin/webcam.o
                0x20000018                last_length
 .data.next_length
                0x2000001c        0x4 ./bin/webcam.o
                0x2000001c                next_length
 .data          0x20000020        0x0 ./bin/kom_modul.o
 .data          0x20000020        0x0 ./bin/rfid_reader.o
 .data          0x20000020        0x0 ./bin/ParTest.o
 .data          0x20000020        0x0 ./bin/flash.o
 .data          0x20000020        0x0 ./bin/FreeRTOS_Tick_Setup.o
 .data          0x20000020        0x0 ./bin/PollQ.o
 .data          0x20000020        0x0 ./bin/semtest.o
 .data          0x20000020        0x0 ./bin/GenQTest.o
 .data          0x20000020        0x0 ./bin/QPeek.o
 .data          0x20000020        0x0 ./bin/FEC.o
 .data          0x20000020        0x0 ./bin/blocktim.o
 .data          0x20000020        0x0 ./bin/recmutex.o
 .data          0x20000020        0x0 ./bin/console_reader.o
 .data          0x20000020        0x0 ./bin/printf-stdarg.o
 .data          0x20000020        0x0 ./bin/portasm.o
 .data          0x20000020        0x0 ./bin/port.o
 .data.ulCriticalNesting
                0x20000020        0x4 ./bin/port.o
 .data          0x20000024        0x0 ./bin/list.o
 .data          0x20000024        0x0 ./bin/tasks.o
 .data.uxPreviousTask
                0x20000024        0x4 ./bin/tasks.o
 .data          0x20000028        0x0 ./bin/queue.o
 .data          0x20000028        0x0 ./bin/heap_1.o
 .data          0x20000028        0x0 ./bin/timer.o
 .data          0x20000028        0x0 ./bin/uip.o
 .data          0x20000028        0x0 ./bin/uip_arp.o
 .data          0x20000028        0x0 ./bin/uiplib.o
 .data          0x20000028        0x0 ./bin/uip-split.o
 .data          0x20000028        0x0 ./bin/psock.o
 .data          0x20000028        0x0 ./bin/uIP_Task.o
 .data          0x20000028        0x0 ./bin/httpd.o
 .data          0x20000028        0x0 ./bin/httpd-cgi.o
 .data.calls    0x20000028       0x18 ./bin/httpd-cgi.o
 .data.states   0x20000040       0x24 ./bin/httpd-cgi.o
 .data          0x20000064        0x0 ./bin/httpd-fs.o
 .data          0x20000064        0x0 ./bin/http-strings.o
 .data          0x20000064        0x0 c:/program files/codesourcery/sourcery g++ lite/bin/../lib/gcc/m68k-elf/4.4.1/m5208\libgcc.a(_float.o)
 .data          0x20000064       0x1c c:/program files/codesourcery/sourcery g++ lite/bin/../lib/gcc/m68k-elf/4.4.1/m5208\libgcc.a(_floatex.o)
                0x20000064                _fpCCR
 .data          0x20000080        0x0 c:/program files/codesourcery/sourcery g++ lite/bin/../lib/gcc/m68k-elf/4.4.1/m5208\libgcc.a(_fixunssfsi.o)
 .data          0x20000080        0x0 c:/program files/codesourcery/sourcery g++ lite/bin/../lib/gcc/m68k-elf/4.4.1/m5208\libgcc.a(fpgnulib.o)
 .data          0x20000080        0x0 c:/program files/codesourcery/sourcery g++ lite/bin/../lib/gcc/m68k-elf/4.4.1/m5208\libgcc.a(_gesf2.o)
 .data          0x20000080        0x0 c:/program files/codesourcery/sourcery g++ lite/bin/../lib/gcc/m68k-elf/4.4.1/../../../../m68k-elf/lib/m5208\libc.a(lib_a-atexit.o)
 .data          0x20000080        0x0 c:/program files/codesourcery/sourcery g++ lite/bin/../lib/gcc/m68k-elf/4.4.1/../../../../m68k-elf/lib/m5208\libc.a(lib_a-atoi.o)
 .data          0x20000080        0x0 c:/program files/codesourcery/sourcery g++ lite/bin/../lib/gcc/m68k-elf/4.4.1/../../../../m68k-elf/lib/m5208\libc.a(lib_a-exit.o)
 .data          0x20000080      0x41a c:/program files/codesourcery/sourcery g++ lite/bin/../lib/gcc/m68k-elf/4.4.1/../../../../m68k-elf/lib/m5208\libc.a(lib_a-impure.o)
                0x20000080                _impure_ptr
 *fill*         0x2000049a        0x2 00
 .data          0x2000049c        0x0 c:/program files/codesourcery/sourcery g++ lite/bin/../lib/gcc/m68k-elf/4.4.1/../../../../m68k-elf/lib/m5208\libc.a(lib_a-memcmp.o)
 .data          0x2000049c        0x0 c:/program files/codesourcery/sourcery g++ lite/bin/../lib/gcc/m68k-elf/4.4.1/../../../../m68k-elf/lib/m5208\libc.a(lib_a-memcpy.o)
 .data          0x2000049c        0x0 c:/program files/codesourcery/sourcery g++ lite/bin/../lib/gcc/m68k-elf/4.4.1/../../../../m68k-elf/lib/m5208\libc.a(lib_a-memset.o)
 .data          0x2000049c        0x0 c:/program files/codesourcery/sourcery g++ lite/bin/../lib/gcc/m68k-elf/4.4.1/../../../../m68k-elf/lib/m5208\libc.a(lib_a-puts.o)
 .data          0x2000049c        0x0 c:/program files/codesourcery/sourcery g++ lite/bin/../lib/gcc/m68k-elf/4.4.1/../../../../m68k-elf/lib/m5208\libc.a(lib_a-strcat.o)
 .data          0x2000049c        0x0 c:/program files/codesourcery/sourcery g++ lite/bin/../lib/gcc/m68k-elf/4.4.1/../../../../m68k-elf/lib/m5208\libc.a(lib_a-strchr.o)
 .data          0x2000049c        0x0 c:/program files/codesourcery/sourcery g++ lite/bin/../lib/gcc/m68k-elf/4.4.1/../../../../m68k-elf/lib/m5208\libc.a(lib_a-strcmp.o)
 .data          0x2000049c        0x0 c:/program files/codesourcery/sourcery g++ lite/bin/../lib/gcc/m68k-elf/4.4.1/../../../../m68k-elf/lib/m5208\libc.a(lib_a-strcpy.o)
 .data          0x2000049c        0x0 c:/program files/codesourcery/sourcery g++ lite/bin/../lib/gcc/m68k-elf/4.4.1/../../../../m68k-elf/lib/m5208\libc.a(lib_a-strlen.o)
 .data          0x2000049c        0x0 c:/program files/codesourcery/sourcery g++ lite/bin/../lib/gcc/m68k-elf/4.4.1/../../../../m68k-elf/lib/m5208\libc.a(lib_a-strncmp.o)
 .data          0x2000049c        0x0 c:/program files/codesourcery/sourcery g++ lite/bin/../lib/gcc/m68k-elf/4.4.1/../../../../m68k-elf/lib/m5208\libc.a(lib_a-strncpy.o)
 .data          0x2000049c        0x0 c:/program files/codesourcery/sourcery g++ lite/bin/../lib/gcc/m68k-elf/4.4.1/../../../../m68k-elf/lib/m5208\libc.a(lib_a-strrchr.o)
 .data          0x2000049c        0x0 c:/program files/codesourcery/sourcery g++ lite/bin/../lib/gcc/m68k-elf/4.4.1/../../../../m68k-elf/lib/m5208\libc.a(lib_a-strtok.o)
 .data          0x2000049c        0x0 c:/program files/codesourcery/sourcery g++ lite/bin/../lib/gcc/m68k-elf/4.4.1/../../../../m68k-elf/lib/m5208\libc.a(lib_a-strtok_r.o)
 .data          0x2000049c        0x0 c:/program files/codesourcery/sourcery g++ lite/bin/../lib/gcc/m68k-elf/4.4.1/../../../../m68k-elf/lib/m5208\libc.a(lib_a-strtol.o)
 .data          0x2000049c        0x0 c:/program files/codesourcery/sourcery g++ lite/bin/../lib/gcc/m68k-elf/4.4.1/../../../../m68k-elf/lib/m5208\libc.a(lib_a-__atexit.o)
 .data          0x2000049c        0x0 c:/program files/codesourcery/sourcery g++ lite/bin/../lib/gcc/m68k-elf/4.4.1/../../../../m68k-elf/lib/m5208\libc.a(lib_a-__call_atexit.o)
 .data          0x2000049c        0x8 c:/program files/codesourcery/sourcery g++ lite/bin/../lib/gcc/m68k-elf/4.4.1/../../../../m68k-elf/lib/m5208\libc.a(lib_a-ctype_.o)
                0x2000049c                __ctype_ptr
                0x200004a0                __ctype_ptr__
 .data          0x200004a4        0x0 c:/program files/codesourcery/sourcery g++ lite/bin/../lib/gcc/m68k-elf/4.4.1/../../../../m68k-elf/lib/m5208\libc.a(lib_a-fini.o)
 .data          0x200004a4        0x0 c:/program files/codesourcery/sourcery g++ lite/bin/../lib/gcc/m68k-elf/4.4.1/../../../../m68k-elf/lib/m5208\libc.a(lib_a-fvwrite.o)
 .data          0x200004a4      0x410 c:/program files/codesourcery/sourcery g++ lite/bin/../lib/gcc/m68k-elf/4.4.1/../../../../m68k-elf/lib/m5208\libc.a(lib_a-mallocr.o)
                0x200004a4                __malloc_av_
                0x200008ac                __malloc_trim_threshold
                0x200008b0                __malloc_sbrk_base
 .data          0x200008b4        0x0 c:/program files/codesourcery/sourcery g++ lite/bin/../lib/gcc/m68k-elf/4.4.1/../../../../m68k-elf/lib/m5208\libc.a(lib_a-memchr.o)
 .data          0x200008b4        0x0 c:/program files/codesourcery/sourcery g++ lite/bin/../lib/gcc/m68k-elf/4.4.1/../../../../m68k-elf/lib/m5208\libc.a(lib_a-memmove.o)
 .data          0x200008b4        0x0 c:/program files/codesourcery/sourcery g++ lite/bin/../lib/gcc/m68k-elf/4.4.1/../../../../m68k-elf/lib/m5208\libc.a(lib_a-mlock.o)
 .data          0x200008b4        0x0 c:/program files/codesourcery/sourcery g++ lite/bin/../lib/gcc/m68k-elf/4.4.1/../../../../m68k-elf/lib/m5208\libc.a(lib_a-reallocr.o)
 .data          0x200008b4        0x0 c:/program files/codesourcery/sourcery g++ lite/bin/../lib/gcc/m68k-elf/4.4.1/../../../../m68k-elf/lib/m5208\libc.a(lib_a-sbrkr.o)
 .data          0x200008b4        0x0 c:/program files/codesourcery/sourcery g++ lite/bin/../lib/gcc/m68k-elf/4.4.1/../../../../m68k-elf/lib/m5208\libc.a(lib_a-wsetup.o)
 .data          0x200008b4        0x0 c:/program files/codesourcery/sourcery g++ lite/bin/../lib/gcc/m68k-elf/4.4.1/../../../../m68k-elf/lib/m5208\libc.a(lib_a-fflush.o)
 .data          0x200008b4        0x0 c:/program files/codesourcery/sourcery g++ lite/bin/../lib/gcc/m68k-elf/4.4.1/../../../../m68k-elf/lib/m5208\libc.a(lib_a-findfp.o)
 .data          0x200008b4        0x0 c:/program files/codesourcery/sourcery g++ lite/bin/../lib/gcc/m68k-elf/4.4.1/../../../../m68k-elf/lib/m5208\libc.a(lib_a-freer.o)
 .data          0x200008b4        0x0 c:/program files/codesourcery/sourcery g++ lite/bin/../lib/gcc/m68k-elf/4.4.1/../../../../m68k-elf/lib/m5208\libc.a(lib_a-fwalk.o)
 .data          0x200008b4        0x0 c:/program files/codesourcery/sourcery g++ lite/bin/../lib/gcc/m68k-elf/4.4.1/../../../../m68k-elf/lib/m5208\libc.a(lib_a-makebuf.o)
 .data          0x200008b4        0x0 c:/program files/codesourcery/sourcery g++ lite/bin/../lib/gcc/m68k-elf/4.4.1/../../../../m68k-elf/lib/m5208\libc.a(lib_a-reent.o)
 .data          0x200008b4        0x0 c:/program files/codesourcery/sourcery g++ lite/bin/../lib/gcc/m68k-elf/4.4.1/../../../../m68k-elf/lib/m5208\libc.a(lib_a-stdio.o)
 .data          0x200008b4        0x0 c:/program files/codesourcery/sourcery g++ lite/bin/../lib/gcc/m68k-elf/4.4.1/../../../../m68k-elf/lib/m5208\libc.a(lib_a-writer.o)
 .data          0x200008b4        0x0 c:/program files/codesourcery/sourcery g++ lite/bin/../lib/gcc/m68k-elf/4.4.1/../../../../m68k-elf/lib/m5208\libc.a(lib_a-closer.o)
 .data          0x200008b4        0x0 c:/program files/codesourcery/sourcery g++ lite/bin/../lib/gcc/m68k-elf/4.4.1/../../../../m68k-elf/lib/m5208\libc.a(lib_a-fclose.o)
 .data          0x200008b4        0x0 c:/program files/codesourcery/sourcery g++ lite/bin/../lib/gcc/m68k-elf/4.4.1/../../../../m68k-elf/lib/m5208\libc.a(lib_a-fstatr.o)
 .data          0x200008b4        0x0 c:/program files/codesourcery/sourcery g++ lite/bin/../lib/gcc/m68k-elf/4.4.1/../../../../m68k-elf/lib/m5208\libc.a(lib_a-isattyr.o)
 .data          0x200008b4        0x0 c:/program files/codesourcery/sourcery g++ lite/bin/../lib/gcc/m68k-elf/4.4.1/../../../../m68k-elf/lib/m5208\libc.a(lib_a-lseekr.o)
 .data          0x200008b4        0x0 c:/program files/codesourcery/sourcery g++ lite/bin/../lib/gcc/m68k-elf/4.4.1/../../../../m68k-elf/lib/m5208\libc.a(lib_a-readr.o)
 .data          0x200008b4        0x0 c:/program files/codesourcery/sourcery g++ lite/bin/../lib/gcc/m68k-elf/4.4.1/../../../../m68k-elf/lib/m5208\libcs3.a(start_c.o)
 .data          0x200008b4        0x0 c:/program files/codesourcery/sourcery g++ lite/bin/../lib/gcc/m68k-elf/4.4.1/../../../../m68k-elf/lib/m5208\libcs3.a(m52235evb-reset.o)
 .data          0x200008b4        0x0 c:/program files/codesourcery/sourcery g++ lite/bin/../lib/gcc/m68k-elf/4.4.1/../../../../m68k-elf/lib/m5208\libcs3hosted.a(hosted-_exit.o)
 .data          0x200008b4        0x0 c:/program files/codesourcery/sourcery g++ lite/bin/../lib/gcc/m68k-elf/4.4.1/../../../../m68k-elf/lib/m5208\libcs3hosted.a(hosted-close.o)
 .data          0x200008b4        0x0 c:/program files/codesourcery/sourcery g++ lite/bin/../lib/gcc/m68k-elf/4.4.1/../../../../m68k-elf/lib/m5208\libcs3hosted.a(hosted-fstat.o)
 .data          0x200008b4        0x0 c:/program files/codesourcery/sourcery g++ lite/bin/../lib/gcc/m68k-elf/4.4.1/../../../../m68k-elf/lib/m5208\libcs3hosted.a(hosted-isatty.o)
 .data          0x200008b4        0x0 c:/program files/codesourcery/sourcery g++ lite/bin/../lib/gcc/m68k-elf/4.4.1/../../../../m68k-elf/lib/m5208\libcs3hosted.a(hosted-lseek.o)
 .data          0x200008b4        0x0 c:/program files/codesourcery/sourcery g++ lite/bin/../lib/gcc/m68k-elf/4.4.1/../../../../m68k-elf/lib/m5208\libcs3hosted.a(hosted-read.o)
 .data          0x200008b4        0x4 c:/program files/codesourcery/sourcery g++ lite/bin/../lib/gcc/m68k-elf/4.4.1/../../../../m68k-elf/lib/m5208\libcs3hosted.a(hosted-sbrk.o)
 .data          0x200008b8        0x0 c:/program files/codesourcery/sourcery g++ lite/bin/../lib/gcc/m68k-elf/4.4.1/../../../../m68k-elf/lib/m5208\libcs3hosted.a(hosted-gdb.o)
 .data          0x200008b8        0x0 c:/program files/codesourcery/sourcery g++ lite/bin/../lib/gcc/m68k-elf/4.4.1/../../../../m68k-elf/lib/m5208\libcs3hosted.a(hosted-start.o)
 .data          0x200008b8        0x0 c:/program files/codesourcery/sourcery g++ lite/bin/../lib/gcc/m68k-elf/4.4.1/../../../../m68k-elf/lib/m5208\libcs3coldfire.a(coldfire-vector.o)
 .data          0x200008b8        0x0 c:/program files/codesourcery/sourcery g++ lite/bin/../lib/gcc/m68k-elf/4.4.1/../../../../m68k-elf/lib/m5208\libcs3coldfire.a(coldfire_isr_other_interrupt.o)
 .data          0x200008b8        0x0 c:/program files/codesourcery/sourcery g++ lite/bin/../lib/gcc/m68k-elf/4.4.1/../../../../m68k-elf/lib/m5208\libcs3coldfire.a(coldfire_isr_unimplemented_opcode.o)
 .data          0x200008b8        0x0 c:/program files/codesourcery/sourcery g++ lite/bin/../lib/gcc/m68k-elf/4.4.1/../../../../m68k-elf/lib/m5208\libcs3coldfire.a(coldfire_isr_breakpoint_debug_interrupt.o)
 .data          0x200008b8        0x0 c:/program files/codesourcery/sourcery g++ lite/bin/../lib/gcc/m68k-elf/4.4.1/../../../../m68k-elf/lib/m5208\libcs3coldfire.a(coldfire_isr_trap_interrupt.o)
 .data          0x200008b8        0x0 c:/program files/codesourcery/sourcery g++ lite/bin/../lib/gcc/m68k-elf/4.4.1/../../../../m68k-elf/lib/m5208\libcs3coldfire.a(coldfire_isr_fp_interrupt.o)
 .data          0x200008b8        0x0 c:/program files/codesourcery/sourcery g++ lite/bin/../lib/gcc/m68k-elf/4.4.1/../../../../m68k-elf/lib/m5208\libcs3coldfire.a(coldfire_isr_access_error.o)
 .data          0x200008b8        0x0 c:/program files/codesourcery/sourcery g++ lite/bin/../lib/gcc/m68k-elf/4.4.1/../../../../m68k-elf/lib/m5208\libcs3coldfire.a(coldfire_isr_address_error.o)
 .data          0x200008b8        0x0 c:/program files/codesourcery/sourcery g++ lite/bin/../lib/gcc/m68k-elf/4.4.1/../../../../m68k-elf/lib/m5208\libcs3coldfire.a(coldfire_isr_illegal_instruction.o)
 .data          0x200008b8        0x0 c:/program files/codesourcery/sourcery g++ lite/bin/../lib/gcc/m68k-elf/4.4.1/../../../../m68k-elf/lib/m5208\libcs3coldfire.a(coldfire_isr_divide_by_zero.o)
 .data          0x200008b8        0x0 c:/program files/codesourcery/sourcery g++ lite/bin/../lib/gcc/m68k-elf/4.4.1/../../../../m68k-elf/lib/m5208\libcs3coldfire.a(coldfire_isr_privilege_violation.o)
 .data          0x200008b8        0x0 c:/program files/codesourcery/sourcery g++ lite/bin/../lib/gcc/m68k-elf/4.4.1/../../../../m68k-elf/lib/m5208\libcs3coldfire.a(coldfire_isr_trace.o)
 .data          0x200008b8        0x0 c:/program files/codesourcery/sourcery g++ lite/bin/../lib/gcc/m68k-elf/4.4.1/../../../../m68k-elf/lib/m5208\libcs3coldfire.a(coldfire_isr_format_error.o)
 .data          0x200008b8        0x0 c:/program files/codesourcery/sourcery g++ lite/bin/../lib/gcc/m68k-elf/4.4.1/../../../../m68k-elf/lib/m5208\libcs3coldfire.a(coldfire_isr_spurious_interrupt.o)
 .data          0x200008b8        0x0 c:/program files/codesourcery/sourcery g++ lite/bin/../lib/gcc/m68k-elf/4.4.1/../../../../m68k-elf/lib/m5208\libcs3coldfire.a(coldfire_isr_unsupported_instruction.o)
 .data          0x200008b8        0x0 c:/program files/codesourcery/sourcery g++ lite/bin/../lib/gcc/m68k-elf/4.4.1/../../../../m68k-elf/lib/m5208\libc.a(lib_a-errno.o)
 .data          0x200008b8        0x0 c:/program files/codesourcery/sourcery g++ lite/bin/../lib/gcc/m68k-elf/4.4.1/../../../../m68k-elf/lib/m5208\libc.a(lib_a-init.o)
 .data          0x200008b8        0x4 c:/program files/codesourcery/sourcery g++ lite/bin/../lib/gcc/m68k-elf/4.4.1/../../../../m68k-elf/lib/m5208\libcs3.a(heap.o)
                0x200008b8                __cs3_heap_limit
                0x200008c0                . = ALIGN (0x8)
 *fill*         0x200008bc        0x4 00
 *(.ram)
                0x200008c0                _edata = .

.bss            0x200008c0     0x5d38 load address 0x00023390
 *(.shbss)
 *(.bss .bss.* .gnu.linkonce.b.*)
 .bss           0x200008c0        0x0 ./bin/main.o
 .bss.ulErrorCode
                0x200008c0        0x4 ./bin/main.o
 .bss.xTimeStart
                0x200008c4        0x4 ./bin/main.o
                0x200008c4                xTimeStart
 .bss.xTimePrev
                0x200008c8        0x4 ./bin/main.o
                0x200008c8                xTimePrev
 .bss.IdleTime  0x200008cc        0x4 ./bin/main.o
                0x200008cc                IdleTime
 .bss.maxVykon  0x200008d0        0x1 ./bin/main.o
                0x200008d0                maxVykon
 *fill*         0x200008d1        0x3 00
 .bss           0x200008d4        0x0 ./bin/uart0.o
 .bss.EnUser    0x200008d4        0x1 ./bin/uart0.o
 *fill*         0x200008d5        0x1 00
 .bss.SerFlag   0x200008d6        0x2 ./bin/uart0.o
 .bss.InpPtrR   0x200008d8        0x4 ./bin/uart0.o
 .bss.InpPtrW   0x200008dc        0x4 ./bin/uart0.o
 .bss.InpBuffer
                0x200008e0       0xb4 ./bin/uart0.o
 .bss.OutPtrR   0x20000994        0x4 ./bin/uart0.o
 .bss.OutPtrW   0x20000998        0x4 ./bin/uart0.o
 .bss.OutBuffer
                0x2000099c       0x28 ./bin/uart0.o
 .bss           0x200009c4        0x0 ./bin/uart1.o
 .bss.SerFlag   0x200009c4        0x2 ./bin/uart1.o
 .bss.InpPtrR   0x200009c6        0x4 ./bin/uart1.o
 .bss.InpPtrW   0x200009ca        0x4 ./bin/uart1.o
 .bss.InpBuffer
                0x200009ce       0x1e ./bin/uart1.o
 .bss.OutPtrR   0x200009ec        0x4 ./bin/uart1.o
 .bss.OutPtrW   0x200009f0        0x4 ./bin/uart1.o
 .bss.OutBuffer
                0x200009f4       0x78 ./bin/uart1.o
 .bss           0x20000a6c        0x0 ./bin/uart2.o
 .bss.SerFlag   0x20000a6c        0x2 ./bin/uart2.o
 .bss.InpPtrR   0x20000a6e        0x4 ./bin/uart2.o
 .bss.InpPtrW   0x20000a72        0x4 ./bin/uart2.o
 .bss.InpBuffer
                0x20000a76       0x32 ./bin/uart2.o
 .bss.OutPtrR   0x20000aa8        0x4 ./bin/uart2.o
 .bss.OutPtrW   0x20000aac        0x4 ./bin/uart2.o
 .bss.OutBuffer
                0x20000ab0        0xf ./bin/uart2.o
 *fill*         0x20000abf        0x1 00
 .bss           0x20000ac0        0x0 ./bin/LCD.o
 .bss           0x20000ac0        0x0 ./bin/klavesnica.o
 .bss           0x20000ac0        0x0 ./bin/flashUtilities.o
 .bss.storage.1612
                0x20000ac0       0xc8 ./bin/flashUtilities.o
 .bss           0x20000b88        0x0 ./bin/riadenie.o
 .bss           0x20000b88        0x0 ./bin/webcam.o
 .bss.bytesin   0x20000b88        0x1 ./bin/webcam.o
                0x20000b88                bytesin
 .bss.writeblock
                0x20000b89        0x1 ./bin/webcam.o
                0x20000b89                writeblock
 .bss.readblock
                0x20000b8a        0x1 ./bin/webcam.o
                0x20000b8a                readblock
 .bss.overflow  0x20000b8b        0x1 ./bin/webcam.o
                0x20000b8b                overflow
 .bss.akt_package_counter
                0x20000b8c        0x4 ./bin/webcam.o
                0x20000b8c                akt_package_counter
 .bss.akt_total_packages
                0x20000b90        0x4 ./bin/webcam.o
                0x20000b90                akt_total_packages
 .bss.start_package_counter
                0x20000b94        0x4 ./bin/webcam.o
                0x20000b94                start_package_counter
 .bss           0x20000b98        0x0 ./bin/kom_modul.o
 .bss           0x20000b98        0x0 ./bin/rfid_reader.o
 .bss           0x20000b98        0x0 ./bin/ParTest.o
 .bss           0x20000b98        0x0 ./bin/flash.o
 .bss.uxFlashTaskNumber
                0x20000b98        0x4 ./bin/flash.o
 .bss           0x20000b9c        0x0 ./bin/FreeRTOS_Tick_Setup.o
 .bss           0x20000b9c        0x0 ./bin/PollQ.o
 .bss.xPollingConsumerCount
                0x20000b9c        0x4 ./bin/PollQ.o
 .bss.xPollingProducerCount
                0x20000ba0        0x4 ./bin/PollQ.o
 .bss.xPolledQueue.1979
                0x20000ba4        0x4 ./bin/PollQ.o
 .bss           0x20000ba8        0x0 ./bin/semtest.o
 .bss.sCheckVariables
                0x20000ba8        0x8 ./bin/semtest.o
 .bss.sNextCheckVariable
                0x20000bb0        0x2 ./bin/semtest.o
 .bss.sLastCheckVariables.2075
                0x20000bb2        0x8 ./bin/semtest.o
 *fill*         0x20000bba        0x2 00
 .bss           0x20000bbc        0x0 ./bin/GenQTest.o
 .bss.xErrorDetected
                0x20000bbc        0x4 ./bin/GenQTest.o
 .bss.ulLoopCounter
                0x20000bc0        0x4 ./bin/GenQTest.o
 .bss.ulLoopCounter2
                0x20000bc4        0x4 ./bin/GenQTest.o
 .bss.ulGuardedVariable
                0x20000bc8        0x4 ./bin/GenQTest.o
 .bss.xHighPriorityMutexTask
                0x20000bcc        0x4 ./bin/GenQTest.o
 .bss.xMediumPriorityMutexTask
                0x20000bd0        0x4 ./bin/GenQTest.o
 .bss.ulLastLoopCounter.2172
                0x20000bd4        0x4 ./bin/GenQTest.o
 .bss.ulLastLoopCounter2.2173
                0x20000bd8        0x4 ./bin/GenQTest.o
 .bss           0x20000bdc        0x0 ./bin/QPeek.o
 .bss.xErrorDetected
                0x20000bdc        0x4 ./bin/QPeek.o
 .bss.ulLoopCounter
                0x20000be0        0x4 ./bin/QPeek.o
 .bss.ulLastLoopCounter.2103
                0x20000be4        0x4 ./bin/QPeek.o
 .bss           0x20000be8        0x0 ./bin/FEC.o
 .bss.xFECSemaphore
                0x20000be8        0x4 ./bin/FEC.o
                0x20000be8                xFECSemaphore
 .bss.xTxSemaphore
                0x20000bec        0x4 ./bin/FEC.o
                0x20000bec                xTxSemaphore
 .bss.xFECTxDescriptors_unaligned
                0x20000bf0       0x18 ./bin/FEC.o
 .bss.xFECRxDescriptors_unaligned
                0x20000c08       0x28 ./bin/FEC.o
 .bss.xFECTxDescriptors
                0x20000c30        0x4 ./bin/FEC.o
 .bss.xFECRxDescriptors
                0x20000c34        0x4 ./bin/FEC.o
 .bss.ucFECRxBuffers
                0x20000c38     0x17b0 ./bin/FEC.o
 .bss.uxNextRxBuffer
                0x200023e8        0x4 ./bin/FEC.o
 .bss.uxIndexToBufferOwner
                0x200023ec        0x4 ./bin/FEC.o
 .bss           0x200023f0        0x0 ./bin/blocktim.o
 .bss.xTestQueue
                0x200023f0        0x4 ./bin/blocktim.o
 .bss.xSecondary
                0x200023f4        0x4 ./bin/blocktim.o
 .bss.xPrimaryCycles
                0x200023f8        0x4 ./bin/blocktim.o
 .bss.xSecondaryCycles
                0x200023fc        0x4 ./bin/blocktim.o
 .bss.xErrorOccurred
                0x20002400        0x4 ./bin/blocktim.o
 .bss.xRunIndicator
                0x20002404        0x4 ./bin/blocktim.o
 .bss.xLastPrimaryCycleCount.1626
                0x20002408        0x4 ./bin/blocktim.o
 .bss.xLastSecondaryCycleCount.1627
                0x2000240c        0x4 ./bin/blocktim.o
 .bss           0x20002410        0x0 ./bin/recmutex.o
 .bss.xMutex    0x20002410        0x4 ./bin/recmutex.o
 .bss.xErrorOccurred
                0x20002414        0x4 ./bin/recmutex.o
 .bss.xControllingIsSuspended
                0x20002418        0x4 ./bin/recmutex.o
 .bss.xBlockingIsSuspended
                0x2000241c        0x4 ./bin/recmutex.o
 .bss.uxControllingCycles
                0x20002420        0x4 ./bin/recmutex.o
 .bss.uxBlockingCycles
                0x20002424        0x4 ./bin/recmutex.o
 .bss.uxPollingCycles
                0x20002428        0x4 ./bin/recmutex.o
 .bss.xControllingTaskHandle
                0x2000242c        0x4 ./bin/recmutex.o
 .bss.xBlockingTaskHandle
                0x20002430        0x4 ./bin/recmutex.o
 .bss.uxLastControllingCycles.1550
                0x20002434        0x4 ./bin/recmutex.o
 .bss.uxLastBlockingCycles.1551
                0x20002438        0x4 ./bin/recmutex.o
 .bss.uxLastPollingCycles.1552
                0x2000243c        0x4 ./bin/recmutex.o
 .bss           0x20002440        0x0 ./bin/console_reader.o
 .bss           0x20002440        0x0 ./bin/printf-stdarg.o
 .bss           0x20002440        0x0 ./bin/portasm.o
 .bss           0x20002440        0x0 ./bin/port.o
 .bss           0x20002440        0x0 ./bin/list.o
 .bss           0x20002440        0x0 ./bin/tasks.o
 .bss.pxCurrentTCB
                0x20002440        0x4 ./bin/tasks.o
                0x20002440                pxCurrentTCB
 .bss.pxReadyTasksLists
                0x20002444       0x50 ./bin/tasks.o
 .bss.xDelayedTaskList1
                0x20002494       0x14 ./bin/tasks.o
 .bss.xDelayedTaskList2
                0x200024a8       0x14 ./bin/tasks.o
 .bss.pxDelayedTaskList
                0x200024bc        0x4 ./bin/tasks.o
 .bss.pxOverflowDelayedTaskList
                0x200024c0        0x4 ./bin/tasks.o
 .bss.xPendingReadyList
                0x200024c4       0x14 ./bin/tasks.o
 .bss.xTasksWaitingTermination
                0x200024d8       0x14 ./bin/tasks.o
 .bss.uxTasksDeleted
                0x200024ec        0x4 ./bin/tasks.o
 .bss.xSuspendedTaskList
                0x200024f0       0x14 ./bin/tasks.o
 .bss.uxCurrentNumberOfTasks
                0x20002504        0x4 ./bin/tasks.o
 .bss.xTickCount
                0x20002508        0x4 ./bin/tasks.o
 .bss.uxTopUsedPriority
                0x2000250c        0x4 ./bin/tasks.o
 .bss.uxTopReadyPriority
                0x20002510        0x4 ./bin/tasks.o
 .bss.xSchedulerRunning
                0x20002514        0x4 ./bin/tasks.o
 .bss.uxSchedulerSuspended
                0x20002518        0x4 ./bin/tasks.o
 .bss.uxMissedTicks
                0x2000251c        0x4 ./bin/tasks.o
 .bss.xMissedYield
                0x20002520        0x4 ./bin/tasks.o
 .bss.xNumOfOverflows
                0x20002524        0x4 ./bin/tasks.o
 .bss.uxTaskNumber
                0x20002528        0x4 ./bin/tasks.o
 .bss.pcTraceBuffer
                0x2000252c        0x4 ./bin/tasks.o
 .bss.pcTraceBufferStart
                0x20002530        0x4 ./bin/tasks.o
 .bss.pcTraceBufferEnd
                0x20002534        0x4 ./bin/tasks.o
 .bss.xTracing  0x20002538        0x4 ./bin/tasks.o
 .bss.pcStatusString
                0x2000253c       0x32 ./bin/tasks.o
 *fill*         0x2000256e        0x2 00
 .bss           0x20002570        0x0 ./bin/queue.o
 .bss           0x20002570        0x0 ./bin/heap_1.o
 .bss.xHeap     0x20002570     0x2710 ./bin/heap_1.o
 .bss.xNextFreeByte
                0x20004c80        0x4 ./bin/heap_1.o
 .bss           0x20004c84        0x0 ./bin/timer.o
 .bss           0x20004c84        0x0 ./bin/uip.o
 .bss.uip_ethaddr
                0x20004c84        0x6 ./bin/uip.o
                0x20004c84                uip_ethaddr
 .bss.ipid      0x20004c8a        0x2 ./bin/uip.o
 .bss.iss       0x20004c8c        0x4 ./bin/uip.o
 .bss.lastport  0x20004c90        0x2 ./bin/uip.o
 .bss.c         0x20004c92        0x1 ./bin/uip.o
 .bss.opt       0x20004c93        0x1 ./bin/uip.o
 .bss.tmp16     0x20004c94        0x2 ./bin/uip.o
 *fill*         0x20004c96        0x2 00
 .bss           0x20004c98        0x0 ./bin/uip_arp.o
 .bss.arp_table
                0x20004c98       0x60 ./bin/uip_arp.o
 .bss.ipaddr    0x20004cf8        0x4 ./bin/uip_arp.o
 .bss.i         0x20004cfc        0x1 ./bin/uip_arp.o
 .bss.c         0x20004cfd        0x1 ./bin/uip_arp.o
 .bss.arptime   0x20004cfe        0x1 ./bin/uip_arp.o
 .bss.tmpage    0x20004cff        0x1 ./bin/uip_arp.o
 .bss           0x20004d00        0x0 ./bin/uiplib.o
 .bss           0x20004d00        0x0 ./bin/uip-split.o
 .bss           0x20004d00        0x0 ./bin/psock.o
 .bss           0x20004d00        0x0 ./bin/uIP_Task.o
 .bss           0x20004d00        0x0 ./bin/httpd.o
 .bss           0x20004d00        0x0 ./bin/httpd-cgi.o
 .bss.cCountBuf
                0x20004d00       0x20 ./bin/httpd-cgi.o
 .bss.lRefreshCount
                0x20004d20        0x4 ./bin/httpd-cgi.o
                0x20004d20                lRefreshCount
 .bss           0x20004d24        0x0 ./bin/httpd-fs.o
 .bss.count     0x20004d24       0x12 ./bin/httpd-fs.o
 *fill*         0x20004d36        0x2 00
 .bss           0x20004d38        0x0 ./bin/http-strings.o
 .bss           0x20004d38        0x0 c:/program files/codesourcery/sourcery g++ lite/bin/../lib/gcc/m68k-elf/4.4.1/m5208\libgcc.a(_float.o)
 .bss           0x20004d38        0x0 c:/program files/codesourcery/sourcery g++ lite/bin/../lib/gcc/m68k-elf/4.4.1/m5208\libgcc.a(_floatex.o)
 .bss           0x20004d38        0x0 c:/program files/codesourcery/sourcery g++ lite/bin/../lib/gcc/m68k-elf/4.4.1/m5208\libgcc.a(_fixunssfsi.o)
 .bss           0x20004d38        0x0 c:/program files/codesourcery/sourcery g++ lite/bin/../lib/gcc/m68k-elf/4.4.1/m5208\libgcc.a(fpgnulib.o)
 .bss           0x20004d38        0x0 c:/program files/codesourcery/sourcery g++ lite/bin/../lib/gcc/m68k-elf/4.4.1/m5208\libgcc.a(_gesf2.o)
 .bss           0x20004d38        0x0 c:/program files/codesourcery/sourcery g++ lite/bin/../lib/gcc/m68k-elf/4.4.1/../../../../m68k-elf/lib/m5208\libc.a(lib_a-atexit.o)
 .bss           0x20004d38        0x0 c:/program files/codesourcery/sourcery g++ lite/bin/../lib/gcc/m68k-elf/4.4.1/../../../../m68k-elf/lib/m5208\libc.a(lib_a-atoi.o)
 .bss           0x20004d38        0x0 c:/program files/codesourcery/sourcery g++ lite/bin/../lib/gcc/m68k-elf/4.4.1/../../../../m68k-elf/lib/m5208\libc.a(lib_a-exit.o)
 .bss           0x20004d38        0x0 c:/program files/codesourcery/sourcery g++ lite/bin/../lib/gcc/m68k-elf/4.4.1/../../../../m68k-elf/lib/m5208\libc.a(lib_a-impure.o)
 .bss           0x20004d38        0x0 c:/program files/codesourcery/sourcery g++ lite/bin/../lib/gcc/m68k-elf/4.4.1/../../../../m68k-elf/lib/m5208\libc.a(lib_a-memcmp.o)
 .bss           0x20004d38        0x0 c:/program files/codesourcery/sourcery g++ lite/bin/../lib/gcc/m68k-elf/4.4.1/../../../../m68k-elf/lib/m5208\libc.a(lib_a-memcpy.o)
 .bss           0x20004d38        0x0 c:/program files/codesourcery/sourcery g++ lite/bin/../lib/gcc/m68k-elf/4.4.1/../../../../m68k-elf/lib/m5208\libc.a(lib_a-memset.o)
 .bss           0x20004d38        0x0 c:/program files/codesourcery/sourcery g++ lite/bin/../lib/gcc/m68k-elf/4.4.1/../../../../m68k-elf/lib/m5208\libc.a(lib_a-puts.o)
 .bss           0x20004d38        0x0 c:/program files/codesourcery/sourcery g++ lite/bin/../lib/gcc/m68k-elf/4.4.1/../../../../m68k-elf/lib/m5208\libc.a(lib_a-strcat.o)
 .bss           0x20004d38        0x0 c:/program files/codesourcery/sourcery g++ lite/bin/../lib/gcc/m68k-elf/4.4.1/../../../../m68k-elf/lib/m5208\libc.a(lib_a-strchr.o)
 .bss           0x20004d38        0x0 c:/program files/codesourcery/sourcery g++ lite/bin/../lib/gcc/m68k-elf/4.4.1/../../../../m68k-elf/lib/m5208\libc.a(lib_a-strcmp.o)
 .bss           0x20004d38        0x0 c:/program files/codesourcery/sourcery g++ lite/bin/../lib/gcc/m68k-elf/4.4.1/../../../../m68k-elf/lib/m5208\libc.a(lib_a-strcpy.o)
 .bss           0x20004d38        0x0 c:/program files/codesourcery/sourcery g++ lite/bin/../lib/gcc/m68k-elf/4.4.1/../../../../m68k-elf/lib/m5208\libc.a(lib_a-strlen.o)
 .bss           0x20004d38        0x0 c:/program files/codesourcery/sourcery g++ lite/bin/../lib/gcc/m68k-elf/4.4.1/../../../../m68k-elf/lib/m5208\libc.a(lib_a-strncmp.o)
 .bss           0x20004d38        0x0 c:/program files/codesourcery/sourcery g++ lite/bin/../lib/gcc/m68k-elf/4.4.1/../../../../m68k-elf/lib/m5208\libc.a(lib_a-strncpy.o)
 .bss           0x20004d38        0x0 c:/program files/codesourcery/sourcery g++ lite/bin/../lib/gcc/m68k-elf/4.4.1/../../../../m68k-elf/lib/m5208\libc.a(lib_a-strrchr.o)
 .bss           0x20004d38        0x0 c:/program files/codesourcery/sourcery g++ lite/bin/../lib/gcc/m68k-elf/4.4.1/../../../../m68k-elf/lib/m5208\libc.a(lib_a-strtok.o)
 .bss           0x20004d38        0x0 c:/program files/codesourcery/sourcery g++ lite/bin/../lib/gcc/m68k-elf/4.4.1/../../../../m68k-elf/lib/m5208\libc.a(lib_a-strtok_r.o)
 .bss           0x20004d38        0x0 c:/program files/codesourcery/sourcery g++ lite/bin/../lib/gcc/m68k-elf/4.4.1/../../../../m68k-elf/lib/m5208\libc.a(lib_a-strtol.o)
 .bss           0x20004d38        0x0 c:/program files/codesourcery/sourcery g++ lite/bin/../lib/gcc/m68k-elf/4.4.1/../../../../m68k-elf/lib/m5208\libc.a(lib_a-__atexit.o)
 .bss           0x20004d38        0x0 c:/program files/codesourcery/sourcery g++ lite/bin/../lib/gcc/m68k-elf/4.4.1/../../../../m68k-elf/lib/m5208\libc.a(lib_a-__call_atexit.o)
 .bss           0x20004d38        0x0 c:/program files/codesourcery/sourcery g++ lite/bin/../lib/gcc/m68k-elf/4.4.1/../../../../m68k-elf/lib/m5208\libc.a(lib_a-ctype_.o)
 .bss           0x20004d38        0x0 c:/program files/codesourcery/sourcery g++ lite/bin/../lib/gcc/m68k-elf/4.4.1/../../../../m68k-elf/lib/m5208\libc.a(lib_a-fini.o)
 .bss           0x20004d38        0x0 c:/program files/codesourcery/sourcery g++ lite/bin/../lib/gcc/m68k-elf/4.4.1/../../../../m68k-elf/lib/m5208\libc.a(lib_a-fvwrite.o)
 .bss           0x20004d38       0x34 c:/program files/codesourcery/sourcery g++ lite/bin/../lib/gcc/m68k-elf/4.4.1/../../../../m68k-elf/lib/m5208\libc.a(lib_a-mallocr.o)
                0x20004d38                __malloc_top_pad
                0x20004d3c                __malloc_max_sbrked_mem
                0x20004d40                __malloc_max_total_mem
                0x20004d44                __malloc_current_mallinfo
 .bss           0x20004d6c        0x0 c:/program files/codesourcery/sourcery g++ lite/bin/../lib/gcc/m68k-elf/4.4.1/../../../../m68k-elf/lib/m5208\libc.a(lib_a-memchr.o)
 .bss           0x20004d6c        0x0 c:/program files/codesourcery/sourcery g++ lite/bin/../lib/gcc/m68k-elf/4.4.1/../../../../m68k-elf/lib/m5208\libc.a(lib_a-memmove.o)
 .bss           0x20004d6c        0x0 c:/program files/codesourcery/sourcery g++ lite/bin/../lib/gcc/m68k-elf/4.4.1/../../../../m68k-elf/lib/m5208\libc.a(lib_a-mlock.o)
 .bss           0x20004d6c        0x0 c:/program files/codesourcery/sourcery g++ lite/bin/../lib/gcc/m68k-elf/4.4.1/../../../../m68k-elf/lib/m5208\libc.a(lib_a-reallocr.o)
 .bss           0x20004d6c        0x0 c:/program files/codesourcery/sourcery g++ lite/bin/../lib/gcc/m68k-elf/4.4.1/../../../../m68k-elf/lib/m5208\libc.a(lib_a-sbrkr.o)
 .bss           0x20004d6c        0x0 c:/program files/codesourcery/sourcery g++ lite/bin/../lib/gcc/m68k-elf/4.4.1/../../../../m68k-elf/lib/m5208\libc.a(lib_a-wsetup.o)
 .bss           0x20004d6c        0x0 c:/program files/codesourcery/sourcery g++ lite/bin/../lib/gcc/m68k-elf/4.4.1/../../../../m68k-elf/lib/m5208\libc.a(lib_a-fflush.o)
 .bss           0x20004d6c        0x0 c:/program files/codesourcery/sourcery g++ lite/bin/../lib/gcc/m68k-elf/4.4.1/../../../../m68k-elf/lib/m5208\libc.a(lib_a-findfp.o)
 .bss           0x20004d6c        0x0 c:/program files/codesourcery/sourcery g++ lite/bin/../lib/gcc/m68k-elf/4.4.1/../../../../m68k-elf/lib/m5208\libc.a(lib_a-freer.o)
 .bss           0x20004d6c        0x0 c:/program files/codesourcery/sourcery g++ lite/bin/../lib/gcc/m68k-elf/4.4.1/../../../../m68k-elf/lib/m5208\libc.a(lib_a-fwalk.o)
 .bss           0x20004d6c        0x0 c:/program files/codesourcery/sourcery g++ lite/bin/../lib/gcc/m68k-elf/4.4.1/../../../../m68k-elf/lib/m5208\libc.a(lib_a-makebuf.o)
 .bss           0x20004d6c        0x0 c:/program files/codesourcery/sourcery g++ lite/bin/../lib/gcc/m68k-elf/4.4.1/../../../../m68k-elf/lib/m5208\libc.a(lib_a-reent.o)
 .bss           0x20004d6c        0x0 c:/program files/codesourcery/sourcery g++ lite/bin/../lib/gcc/m68k-elf/4.4.1/../../../../m68k-elf/lib/m5208\libc.a(lib_a-stdio.o)
 .bss           0x20004d6c        0x0 c:/program files/codesourcery/sourcery g++ lite/bin/../lib/gcc/m68k-elf/4.4.1/../../../../m68k-elf/lib/m5208\libc.a(lib_a-writer.o)
 .bss           0x20004d6c        0x0 c:/program files/codesourcery/sourcery g++ lite/bin/../lib/gcc/m68k-elf/4.4.1/../../../../m68k-elf/lib/m5208\libc.a(lib_a-closer.o)
 .bss           0x20004d6c        0x0 c:/program files/codesourcery/sourcery g++ lite/bin/../lib/gcc/m68k-elf/4.4.1/../../../../m68k-elf/lib/m5208\libc.a(lib_a-fclose.o)
 .bss           0x20004d6c        0x0 c:/program files/codesourcery/sourcery g++ lite/bin/../lib/gcc/m68k-elf/4.4.1/../../../../m68k-elf/lib/m5208\libc.a(lib_a-fstatr.o)
 .bss           0x20004d6c        0x0 c:/program files/codesourcery/sourcery g++ lite/bin/../lib/gcc/m68k-elf/4.4.1/../../../../m68k-elf/lib/m5208\libc.a(lib_a-isattyr.o)
 .bss           0x20004d6c        0x0 c:/program files/codesourcery/sourcery g++ lite/bin/../lib/gcc/m68k-elf/4.4.1/../../../../m68k-elf/lib/m5208\libc.a(lib_a-lseekr.o)
 .bss           0x20004d6c        0x0 c:/program files/codesourcery/sourcery g++ lite/bin/../lib/gcc/m68k-elf/4.4.1/../../../../m68k-elf/lib/m5208\libc.a(lib_a-readr.o)
 .bss           0x20004d6c        0x0 c:/program files/codesourcery/sourcery g++ lite/bin/../lib/gcc/m68k-elf/4.4.1/../../../../m68k-elf/lib/m5208\libcs3.a(start_c.o)
 .bss           0x20004d6c        0x0 c:/program files/codesourcery/sourcery g++ lite/bin/../lib/gcc/m68k-elf/4.4.1/../../../../m68k-elf/lib/m5208\libcs3.a(m52235evb-reset.o)
 .bss           0x20004d6c        0x0 c:/program files/codesourcery/sourcery g++ lite/bin/../lib/gcc/m68k-elf/4.4.1/../../../../m68k-elf/lib/m5208\libcs3hosted.a(hosted-_exit.o)
 .bss           0x20004d6c        0x0 c:/program files/codesourcery/sourcery g++ lite/bin/../lib/gcc/m68k-elf/4.4.1/../../../../m68k-elf/lib/m5208\libcs3hosted.a(hosted-close.o)
 .bss           0x20004d6c        0x0 c:/program files/codesourcery/sourcery g++ lite/bin/../lib/gcc/m68k-elf/4.4.1/../../../../m68k-elf/lib/m5208\libcs3hosted.a(hosted-fstat.o)
 .bss           0x20004d6c        0x0 c:/program files/codesourcery/sourcery g++ lite/bin/../lib/gcc/m68k-elf/4.4.1/../../../../m68k-elf/lib/m5208\libcs3hosted.a(hosted-isatty.o)
 .bss           0x20004d6c        0x0 c:/program files/codesourcery/sourcery g++ lite/bin/../lib/gcc/m68k-elf/4.4.1/../../../../m68k-elf/lib/m5208\libcs3hosted.a(hosted-lseek.o)
 .bss           0x20004d6c        0x0 c:/program files/codesourcery/sourcery g++ lite/bin/../lib/gcc/m68k-elf/4.4.1/../../../../m68k-elf/lib/m5208\libcs3hosted.a(hosted-read.o)
 .bss           0x20004d6c        0x0 c:/program files/codesourcery/sourcery g++ lite/bin/../lib/gcc/m68k-elf/4.4.1/../../../../m68k-elf/lib/m5208\libcs3hosted.a(hosted-sbrk.o)
 .bss           0x20004d6c        0x0 c:/program files/codesourcery/sourcery g++ lite/bin/../lib/gcc/m68k-elf/4.4.1/../../../../m68k-elf/lib/m5208\libcs3hosted.a(hosted-gdb.o)
 .bss           0x20004d6c        0x0 c:/program files/codesourcery/sourcery g++ lite/bin/../lib/gcc/m68k-elf/4.4.1/../../../../m68k-elf/lib/m5208\libcs3hosted.a(hosted-start.o)
 .bss           0x20004d6c        0x0 c:/program files/codesourcery/sourcery g++ lite/bin/../lib/gcc/m68k-elf/4.4.1/../../../../m68k-elf/lib/m5208\libcs3coldfire.a(coldfire-vector.o)
 .bss           0x20004d6c        0x0 c:/program files/codesourcery/sourcery g++ lite/bin/../lib/gcc/m68k-elf/4.4.1/../../../../m68k-elf/lib/m5208\libcs3coldfire.a(coldfire_isr_other_interrupt.o)
 .bss           0x20004d6c        0x0 c:/program files/codesourcery/sourcery g++ lite/bin/../lib/gcc/m68k-elf/4.4.1/../../../../m68k-elf/lib/m5208\libcs3coldfire.a(coldfire_isr_unimplemented_opcode.o)
 .bss           0x20004d6c        0x0 c:/program files/codesourcery/sourcery g++ lite/bin/../lib/gcc/m68k-elf/4.4.1/../../../../m68k-elf/lib/m5208\libcs3coldfire.a(coldfire_isr_breakpoint_debug_interrupt.o)
 .bss           0x20004d6c        0x0 c:/program files/codesourcery/sourcery g++ lite/bin/../lib/gcc/m68k-elf/4.4.1/../../../../m68k-elf/lib/m5208\libcs3coldfire.a(coldfire_isr_trap_interrupt.o)
 .bss           0x20004d6c        0x0 c:/program files/codesourcery/sourcery g++ lite/bin/../lib/gcc/m68k-elf/4.4.1/../../../../m68k-elf/lib/m5208\libcs3coldfire.a(coldfire_isr_fp_interrupt.o)
 .bss           0x20004d6c        0x0 c:/program files/codesourcery/sourcery g++ lite/bin/../lib/gcc/m68k-elf/4.4.1/../../../../m68k-elf/lib/m5208\libcs3coldfire.a(coldfire_isr_access_error.o)
 .bss           0x20004d6c        0x0 c:/program files/codesourcery/sourcery g++ lite/bin/../lib/gcc/m68k-elf/4.4.1/../../../../m68k-elf/lib/m5208\libcs3coldfire.a(coldfire_isr_address_error.o)
 .bss           0x20004d6c        0x0 c:/program files/codesourcery/sourcery g++ lite/bin/../lib/gcc/m68k-elf/4.4.1/../../../../m68k-elf/lib/m5208\libcs3coldfire.a(coldfire_isr_illegal_instruction.o)
 .bss           0x20004d6c        0x0 c:/program files/codesourcery/sourcery g++ lite/bin/../lib/gcc/m68k-elf/4.4.1/../../../../m68k-elf/lib/m5208\libcs3coldfire.a(coldfire_isr_divide_by_zero.o)
 .bss           0x20004d6c        0x0 c:/program files/codesourcery/sourcery g++ lite/bin/../lib/gcc/m68k-elf/4.4.1/../../../../m68k-elf/lib/m5208\libcs3coldfire.a(coldfire_isr_privilege_violation.o)
 .bss           0x20004d6c        0x0 c:/program files/codesourcery/sourcery g++ lite/bin/../lib/gcc/m68k-elf/4.4.1/../../../../m68k-elf/lib/m5208\libcs3coldfire.a(coldfire_isr_trace.o)
 .bss           0x20004d6c        0x0 c:/program files/codesourcery/sourcery g++ lite/bin/../lib/gcc/m68k-elf/4.4.1/../../../../m68k-elf/lib/m5208\libcs3coldfire.a(coldfire_isr_format_error.o)
 .bss           0x20004d6c        0x0 c:/program files/codesourcery/sourcery g++ lite/bin/../lib/gcc/m68k-elf/4.4.1/../../../../m68k-elf/lib/m5208\libcs3coldfire.a(coldfire_isr_spurious_interrupt.o)
 .bss           0x20004d6c        0x0 c:/program files/codesourcery/sourcery g++ lite/bin/../lib/gcc/m68k-elf/4.4.1/../../../../m68k-elf/lib/m5208\libcs3coldfire.a(coldfire_isr_unsupported_instruction.o)
 .bss           0x20004d6c        0x0 c:/program files/codesourcery/sourcery g++ lite/bin/../lib/gcc/m68k-elf/4.4.1/../../../../m68k-elf/lib/m5208\libc.a(lib_a-errno.o)
 .bss           0x20004d6c        0x0 c:/program files/codesourcery/sourcery g++ lite/bin/../lib/gcc/m68k-elf/4.4.1/../../../../m68k-elf/lib/m5208\libc.a(lib_a-init.o)
 .bss           0x20004d6c        0x0 c:/program files/codesourcery/sourcery g++ lite/bin/../lib/gcc/m68k-elf/4.4.1/../../../../m68k-elf/lib/m5208\libcs3.a(heap.o)
 *(COMMON)
 COMMON         0x20004d6c       0xa4 ./bin/main.o
                0x20004d6c                cam_podmienka
                0x20004d6d                komOutSocketbuffer
                0x20004dd2                casovacQueue
                0x20004dd6                CamPictureMutex
                0x20004dda                uart1_Mutex
                0x20004de6                komOutSocketQueue
                0x20004dea                pripojenie
                0x20004dee                uart2_Mutex
                0x20004dfa                klavesnicaGetKeyMutex
                0x20004dfe                kom_podmienka
                0x20004e00                komInSocketQueue
                0x20004e04                uart0_Mutex
 COMMON         0x20004e10        0x4 ./bin/uart0.o
                0x20004e10                uart0_InpLen
                0x20004e12                uart0_OutLen
 COMMON         0x20004e14        0x4 ./bin/uart1.o
                0x20004e14                uart1_OutLen
                0x20004e16                uart1_InpLen
 COMMON         0x20004e18        0x4 ./bin/uart2.o
                0x20004e18                uart2_InpLen
                0x20004e1a                uart2_OutLen
 COMMON         0x20004e1c        0x4 ./bin/klavesnica.o
                0x20004e1c                xTimeLast
 COMMON         0x20004e20       0x8a ./bin/webcam.o
                0x20004e20                cam_data_Length
                0x20004e24                command
                0x20004e2a                rxfifo
 COMMON         0x20004eaa        0xc ./bin/QPeek.o
                0x20004eaa                xHighPriorityTask
                0x20004eae                xMediumPriorityTask
                0x20004eb2                xHighestPriorityTask
 COMMON         0x20004eb6        0x4 ./bin/FEC.o
                0x20004eb6                uip_buf
 COMMON         0x20004eba        0x4 ./bin/console_reader.o
                0x20004eba                temp_velkost
 COMMON         0x20004ebe       0x50 ./bin/queue.o
                0x20004ebe                xQueueRegistry
 COMMON         0x20004f0e     0x16e0 ./bin/uip.o
                0x20004f0e                uip_len
                0x20004f10                uip_sappdata
                0x20004f14                uip_acc32
                0x20004f18                uip_flags
                0x20004f1a                uip_appdata
                0x20004f1e                uip_conn
                0x20004f22                uip_conns
                0x200065a2                uip_listenports
                0x200065ac                uip_draddr
                0x200065b0                uip_stat
                0x200065dc                uip_surglen
                0x200065de                uip_urgdata
                0x200065e2                uip_netmask
                0x200065e6                uip_hostaddr
                0x200065ea                uip_urglen
                0x200065ec                uip_slen
 COMMON         0x200065ee        0x4 ./bin/httpd-cgi.o
                0x200065ee                pcStatus
 COMMON         0x200065f2        0x4 c:/program files/codesourcery/sourcery g++ lite/bin/../lib/gcc/m68k-elf/4.4.1/../../../../m68k-elf/lib/m5208\libc.a(lib_a-reent.o)
                0x200065f2                errno
                0x200065f8                . = ALIGN (0x8)
 *fill*         0x200065f6        0x2 00
 *(.ram.b)
                0x200065f8                _end = .
                0x200065f8                __end = .
                0x20008000                __cs3_region_end_ram = (__cs3_region_start_ram + 0x8000)
                0x00008000                __cs3_region_size_ram = 0x8000
                0x00022ad0                __cs3_region_init_ram = LOADADDR (.data)
                0x000008c0                __cs3_region_init_size_ram = (_edata - ADDR (.data))
                0x00005d38                __cs3_region_zero_size_ram = (_end - _edata)

.stab
 *(.stab)

.stabstr
 *(.stabstr)

.debug
 *(.debug)

.line
 *(.line)

.debug_srcinfo
 *(.debug_srcinfo)

.debug_sfnames
 *(.debug_sfnames)

.comment        0x00000000      0x5f1
 .comment       0x00000000       0x27 ./bin/main.o
 .comment       0x00000027       0x27 ./bin/uart0.o
 .comment       0x0000004e       0x27 ./bin/uart1.o
 .comment       0x00000075       0x27 ./bin/uart2.o
 .comment       0x0000009c       0x27 ./bin/LCD.o
 .comment       0x000000c3       0x27 ./bin/klavesnica.o
 .comment       0x000000ea       0x27 ./bin/flashUtilities.o
 .comment       0x00000111       0x27 ./bin/riadenie.o
 .comment       0x00000138       0x27 ./bin/webcam.o
 .comment       0x0000015f       0x27 ./bin/kom_modul.o
 .comment       0x00000186       0x27 ./bin/rfid_reader.o
 .comment       0x000001ad       0x27 ./bin/ParTest.o
 .comment       0x000001d4       0x27 ./bin/flash.o
 .comment       0x000001fb       0x27 ./bin/FreeRTOS_Tick_Setup.o
 .comment       0x00000222       0x27 ./bin/PollQ.o
 .comment       0x00000249       0x27 ./bin/semtest.o
 .comment       0x00000270       0x27 ./bin/GenQTest.o
 .comment       0x00000297       0x27 ./bin/QPeek.o
 .comment       0x000002be       0x27 ./bin/FEC.o
 .comment       0x000002e5       0x27 ./bin/blocktim.o
 .comment       0x0000030c       0x27 ./bin/recmutex.o
 .comment       0x00000333       0x27 ./bin/console_reader.o
 .comment       0x0000035a       0x27 ./bin/printf-stdarg.o
 .comment       0x00000381       0x27 ./bin/port.o
 .comment       0x000003a8       0x27 ./bin/list.o
 .comment       0x000003cf       0x27 ./bin/tasks.o
 .comment       0x000003f6       0x27 ./bin/queue.o
 .comment       0x0000041d       0x27 ./bin/heap_1.o
 .comment       0x00000444       0x27 ./bin/timer.o
 .comment       0x0000046b       0x27 ./bin/uip.o
 .comment       0x00000492       0x27 ./bin/uip_arp.o
 .comment       0x000004b9       0x27 ./bin/uiplib.o
 .comment       0x000004e0       0x27 ./bin/uip-split.o
 .comment       0x00000507       0x27 ./bin/psock.o
 .comment       0x0000052e       0x27 ./bin/uIP_Task.o
 .comment       0x00000555       0x27 ./bin/httpd.o
 .comment       0x0000057c       0x27 ./bin/httpd-cgi.o
 .comment       0x000005a3       0x27 ./bin/httpd-fs.o
 .comment       0x000005ca       0x27 ./bin/http-strings.o

.debug_aranges  0x00000000      0xf30
 *(.debug_aranges)
 .debug_aranges
                0x00000000       0x78 ./bin/main.o
 .debug_aranges
                0x00000078       0x90 ./bin/uart0.o
 .debug_aranges
                0x00000108       0x90 ./bin/uart1.o
 .debug_aranges
                0x00000198       0x90 ./bin/uart2.o
 .debug_aranges
                0x00000228       0xf0 ./bin/LCD.o
 .debug_aranges
                0x00000318       0x30 ./bin/klavesnica.o
 .debug_aranges
                0x00000348       0x40 ./bin/flashUtilities.o
 .debug_aranges
                0x00000388       0x78 ./bin/riadenie.o
 .debug_aranges
                0x00000400       0x90 ./bin/webcam.o
 .debug_aranges
                0x00000490       0x38 ./bin/kom_modul.o
 .debug_aranges
                0x000004c8       0x28 ./bin/rfid_reader.o
 .debug_aranges
                0x000004f0       0x38 ./bin/ParTest.o
 .debug_aranges
                0x00000528       0x28 ./bin/flash.o
 .debug_aranges
                0x00000550       0x28 ./bin/FreeRTOS_Tick_Setup.o
 .debug_aranges
                0x00000578       0x38 ./bin/PollQ.o
 .debug_aranges
                0x000005b0       0x30 ./bin/semtest.o
 .debug_aranges
                0x000005e0       0x48 ./bin/GenQTest.o
 .debug_aranges
                0x00000628       0x48 ./bin/QPeek.o
 .debug_aranges
                0x00000670       0xe0 ./bin/FEC.o
 .debug_aranges
                0x00000750       0x38 ./bin/blocktim.o
 .debug_aranges
                0x00000788       0x40 ./bin/recmutex.o
 .debug_aranges
                0x000007c8       0xe8 ./bin/console_reader.o
 .debug_aranges
                0x000008b0       0x60 ./bin/printf-stdarg.o
 .debug_aranges
                0x00000910       0x20 ./bin/portasm.o
 .debug_aranges
                0x00000930       0x48 ./bin/port.o
 .debug_aranges
                0x00000978       0x40 ./bin/list.o
 .debug_aranges
                0x000009b8      0x148 ./bin/tasks.o
 .debug_aranges
                0x00000b00       0xc0 ./bin/queue.o
 .debug_aranges
                0x00000bc0       0x38 ./bin/heap_1.o
 .debug_aranges
                0x00000bf8       0x38 ./bin/timer.o
 .debug_aranges
                0x00000c30       0xa0 ./bin/uip.o
 .debug_aranges
                0x00000cd0       0x48 ./bin/uip_arp.o
 .debug_aranges
                0x00000d18       0x20 ./bin/uiplib.o
 .debug_aranges
                0x00000d38       0x20 ./bin/uip-split.o
 .debug_aranges
                0x00000d58       0x78 ./bin/psock.o
 .debug_aranges
                0x00000dd0       0x38 ./bin/uIP_Task.o
 .debug_aranges
                0x00000e08       0x70 ./bin/httpd.o
 .debug_aranges
                0x00000e78       0x80 ./bin/httpd-cgi.o
 .debug_aranges
                0x00000ef8       0x38 ./bin/httpd-fs.o

.debug_pubnames
                0x00000000     0x2b1b
 *(.debug_pubnames)
 .debug_pubnames
                0x00000000      0x19b ./bin/main.o
 .debug_pubnames
                0x0000019b      0x14d ./bin/uart0.o
 .debug_pubnames
                0x000002e8      0x15a ./bin/uart1.o
 .debug_pubnames
                0x00000442      0x15a ./bin/uart2.o
 .debug_pubnames
                0x0000059c      0x206 ./bin/LCD.o
 .debug_pubnames
                0x000007a2       0xb6 ./bin/klavesnica.o
 .debug_pubnames
                0x00000858       0xa2 ./bin/flashUtilities.o
 .debug_pubnames
                0x000008fa      0x1a4 ./bin/riadenie.o
 .debug_pubnames
                0x00000a9e      0x257 ./bin/webcam.o
 .debug_pubnames
                0x00000cf5       0xef ./bin/kom_modul.o
 .debug_pubnames
                0x00000de4       0xdc ./bin/rfid_reader.o
 .debug_pubnames
                0x00000ec0       0x78 ./bin/ParTest.o
 .debug_pubnames
                0x00000f38       0x4c ./bin/flash.o
 .debug_pubnames
                0x00000f84       0x60 ./bin/FreeRTOS_Tick_Setup.o
 .debug_pubnames
                0x00000fe4       0x61 ./bin/PollQ.o
 .debug_pubnames
                0x00001045       0x60 ./bin/semtest.o
 .debug_pubnames
                0x000010a5       0x66 ./bin/GenQTest.o
 .debug_pubnames
                0x0000110b       0xa7 ./bin/QPeek.o
 .debug_pubnames
                0x000011b2      0x287 ./bin/FEC.o
 .debug_pubnames
                0x00001439       0x65 ./bin/blocktim.o
 .debug_pubnames
                0x0000149e       0x6a ./bin/recmutex.o
 .debug_pubnames
                0x00001508      0x290 ./bin/console_reader.o
 .debug_pubnames
                0x00001798       0x64 ./bin/printf-stdarg.o
 .debug_pubnames
                0x000017fc       0xaf ./bin/port.o
 .debug_pubnames
                0x000018ab       0x83 ./bin/list.o
 .debug_pubnames
                0x0000192e      0x2d5 ./bin/tasks.o
 .debug_pubnames
                0x00001c03      0x1c0 ./bin/queue.o
 .debug_pubnames
                0x00001dc3       0x76 ./bin/heap_1.o
 .debug_pubnames
                0x00001e39       0x66 ./bin/timer.o
 .debug_pubnames
                0x00001e9f      0x274 ./bin/uip.o
 .debug_pubnames
                0x00002113       0xf1 ./bin/uip_arp.o
 .debug_pubnames
                0x00002204       0xb1 ./bin/uiplib.o
 .debug_pubnames
                0x000022b5       0xb0 ./bin/uip-split.o
 .debug_pubnames
                0x00002365      0x119 ./bin/psock.o
 .debug_pubnames
                0x0000247e       0xd7 ./bin/uIP_Task.o
 .debug_pubnames
                0x00002555       0xcc ./bin/httpd.o
 .debug_pubnames
                0x00002621       0xf9 ./bin/httpd-cgi.o
 .debug_pubnames
                0x0000271a      0x190 ./bin/httpd-fs.o
 .debug_pubnames
                0x000028aa      0x271 ./bin/http-strings.o

.debug_info     0x00000000     0xd6b9
 *(.debug_info .gnu.linkonce.wi.*)
 .debug_info    0x00000000      0x7d7 ./bin/main.o
 .debug_info    0x000007d7      0x483 ./bin/uart0.o
 .debug_info    0x00000c5a      0x463 ./bin/uart1.o
 .debug_info    0x000010bd      0x463 ./bin/uart2.o
 .debug_info    0x00001520      0x5fb ./bin/LCD.o
 .debug_info    0x00001b1b      0x1b7 ./bin/klavesnica.o
 .debug_info    0x00001cd2      0x2d3 ./bin/flashUtilities.o
 .debug_info    0x00001fa5      0x82a ./bin/riadenie.o
 .debug_info    0x000027cf      0x6d8 ./bin/webcam.o
 .debug_info    0x00002ea7      0x5d9 ./bin/kom_modul.o
 .debug_info    0x00003480      0x4a4 ./bin/rfid_reader.o
 .debug_info    0x00003924      0x126 ./bin/ParTest.o
 .debug_info    0x00003a4a      0x19a ./bin/flash.o
 .debug_info    0x00003be4       0xce ./bin/FreeRTOS_Tick_Setup.o
 .debug_info    0x00003cb2      0x1d0 ./bin/PollQ.o
 .debug_info    0x00003e82      0x268 ./bin/semtest.o
 .debug_info    0x000040ea      0x294 ./bin/GenQTest.o
 .debug_info    0x0000437e      0x27c ./bin/QPeek.o
 .debug_info    0x000045fa      0x963 ./bin/FEC.o
 .debug_info    0x00004f5d      0x236 ./bin/blocktim.o
 .debug_info    0x00005193      0x23c ./bin/recmutex.o
 .debug_info    0x000053cf      0xc46 ./bin/console_reader.o
 .debug_info    0x00006015      0x4b9 ./bin/printf-stdarg.o
 .debug_info    0x000064ce       0xb8 ./bin/portasm.o
 .debug_info    0x00006586      0x177 ./bin/port.o
 .debug_info    0x000066fd      0x2d0 ./bin/list.o
 .debug_info    0x000069cd      0xfbb ./bin/tasks.o
 .debug_info    0x00007988      0x920 ./bin/queue.o
 .debug_info    0x000082a8      0x18d ./bin/heap_1.o
 .debug_info    0x00008435      0x161 ./bin/timer.o
 .debug_info    0x00008596      0xf0f ./bin/uip.o
 .debug_info    0x000094a5      0x769 ./bin/uip_arp.o
 .debug_info    0x00009c0e      0x3db ./bin/uiplib.o
 .debug_info    0x00009fe9      0x555 ./bin/uip-split.o
 .debug_info    0x0000a53e      0x848 ./bin/psock.o
 .debug_info    0x0000ad86      0x63f ./bin/uIP_Task.o
 .debug_info    0x0000b3c5      0xa09 ./bin/httpd.o
 .debug_info    0x0000bdce      0xc94 ./bin/httpd-cgi.o
 .debug_info    0x0000ca62      0x815 ./bin/httpd-fs.o
 .debug_info    0x0000d277      0x442 ./bin/http-strings.o

.debug_abbrev   0x00000000     0x32cf
 *(.debug_abbrev)
 .debug_abbrev  0x00000000      0x1aa ./bin/main.o
 .debug_abbrev  0x000001aa      0x182 ./bin/uart0.o
 .debug_abbrev  0x0000032c      0x1a8 ./bin/uart1.o
 .debug_abbrev  0x000004d4      0x1a8 ./bin/uart2.o
 .debug_abbrev  0x0000067c      0x182 ./bin/LCD.o
 .debug_abbrev  0x000007fe       0xea ./bin/klavesnica.o
 .debug_abbrev  0x000008e8      0x103 ./bin/flashUtilities.o
 .debug_abbrev  0x000009eb      0x17d ./bin/riadenie.o
 .debug_abbrev  0x00000b68      0x1bb ./bin/webcam.o
 .debug_abbrev  0x00000d23      0x1ab ./bin/kom_modul.o
 .debug_abbrev  0x00000ece      0x112 ./bin/rfid_reader.o
 .debug_abbrev  0x00000fe0       0xa7 ./bin/ParTest.o
 .debug_abbrev  0x00001087       0xc9 ./bin/flash.o
 .debug_abbrev  0x00001150       0x71 ./bin/FreeRTOS_Tick_Setup.o
 .debug_abbrev  0x000011c1       0xc6 ./bin/PollQ.o
 .debug_abbrev  0x00001287      0x115 ./bin/semtest.o
 .debug_abbrev  0x0000139c       0xf9 ./bin/GenQTest.o
 .debug_abbrev  0x00001495       0xf9 ./bin/QPeek.o
 .debug_abbrev  0x0000158e      0x1f9 ./bin/FEC.o
 .debug_abbrev  0x00001787       0xec ./bin/blocktim.o
 .debug_abbrev  0x00001873       0xfb ./bin/recmutex.o
 .debug_abbrev  0x0000196e      0x1b5 ./bin/console_reader.o
 .debug_abbrev  0x00001b23      0x17b ./bin/printf-stdarg.o
 .debug_abbrev  0x00001c9e       0x14 ./bin/portasm.o
 .debug_abbrev  0x00001cb2       0xeb ./bin/port.o
 .debug_abbrev  0x00001d9d       0xc8 ./bin/list.o
 .debug_abbrev  0x00001e65      0x185 ./bin/tasks.o
 .debug_abbrev  0x00001fea      0x171 ./bin/queue.o
 .debug_abbrev  0x0000215b      0x11a ./bin/heap_1.o
 .debug_abbrev  0x00002275       0xc8 ./bin/timer.o
 .debug_abbrev  0x0000233d      0x23e ./bin/uip.o
 .debug_abbrev  0x0000257b      0x1b3 ./bin/uip_arp.o
 .debug_abbrev  0x0000272e       0xf8 ./bin/uiplib.o
 .debug_abbrev  0x00002826      0x125 ./bin/uip-split.o
 .debug_abbrev  0x0000294b      0x1f8 ./bin/psock.o
 .debug_abbrev  0x00002b43      0x180 ./bin/uIP_Task.o
 .debug_abbrev  0x00002cc3      0x213 ./bin/httpd.o
 .debug_abbrev  0x00002ed6      0x213 ./bin/httpd-cgi.o
 .debug_abbrev  0x000030e9      0x192 ./bin/httpd-fs.o
 .debug_abbrev  0x0000327b       0x54 ./bin/http-strings.o

.debug_line     0x00000000     0xf962
 *(.debug_line)
 .debug_line    0x00000000      0x982 ./bin/main.o
 .debug_line    0x00000982      0x5a9 ./bin/uart0.o
 .debug_line    0x00000f2b      0x5a3 ./bin/uart1.o
 .debug_line    0x000014ce      0x5a3 ./bin/uart2.o
 .debug_line    0x00001a71      0x7bc ./bin/LCD.o
 .debug_line    0x0000222d      0x495 ./bin/klavesnica.o
 .debug_line    0x000026c2      0x594 ./bin/flashUtilities.o
 .debug_line    0x00002c56      0x883 ./bin/riadenie.o
 .debug_line    0x000034d9      0x7ce ./bin/webcam.o
 .debug_line    0x00003ca7      0x6f1 ./bin/kom_modul.o
 .debug_line    0x00004398      0x59c ./bin/rfid_reader.o
 .debug_line    0x00004934      0x3e8 ./bin/ParTest.o
 .debug_line    0x00004d1c      0x648 ./bin/flash.o
 .debug_line    0x00005364      0x38e ./bin/FreeRTOS_Tick_Setup.o
 .debug_line    0x000056f2      0x5fb ./bin/PollQ.o
 .debug_line    0x00005ced      0x618 ./bin/semtest.o
 .debug_line    0x00006305      0x68f ./bin/GenQTest.o
 .debug_line    0x00006994      0x652 ./bin/QPeek.o
 .debug_line    0x00006fe6      0x7ab ./bin/FEC.o
 .debug_line    0x00007791      0x483 ./bin/blocktim.o
 .debug_line    0x00007c14      0x460 ./bin/recmutex.o
 .debug_line    0x00008074      0xa08 ./bin/console_reader.o
 .debug_line    0x00008a7c      0x562 ./bin/printf-stdarg.o
 .debug_line    0x00008fde       0x7b ./bin/portasm.o
 .debug_line    0x00009059      0x3fe ./bin/port.o
 .debug_line    0x00009457      0x5b1 ./bin/list.o
 .debug_line    0x00009a08      0x9e4 ./bin/tasks.o
 .debug_line    0x0000a3ec      0x808 ./bin/queue.o
 .debug_line    0x0000abf4      0x5a9 ./bin/heap_1.o
 .debug_line    0x0000b19d      0x3d5 ./bin/timer.o
 .debug_line    0x0000b572      0xac2 ./bin/uip.o
 .debug_line    0x0000c034      0x766 ./bin/uip_arp.o
 .debug_line    0x0000c79a      0x51b ./bin/uiplib.o
 .debug_line    0x0000ccb5      0x6e8 ./bin/uip-split.o
 .debug_line    0x0000d39d      0x804 ./bin/psock.o
 .debug_line    0x0000dba1      0x78f ./bin/uIP_Task.o
 .debug_line    0x0000e330      0x832 ./bin/httpd.o
 .debug_line    0x0000eb62      0x818 ./bin/httpd-cgi.o
 .debug_line    0x0000f37a      0x5ad ./bin/httpd-fs.o
 .debug_line    0x0000f927       0x3b ./bin/http-strings.o

.debug_frame
 *(.debug_frame)

.debug_str      0x00000000     0x3903
 *(.debug_str)
 .debug_str     0x00000000      0x438 ./bin/main.o
                                0x494 (size before relaxing)
 .debug_str     0x00000438      0x1b1 ./bin/uart0.o
                                0x318 (size before relaxing)
 .debug_str     0x000005e9      0x136 ./bin/uart1.o
                                0x31f (size before relaxing)
 .debug_str     0x0000071f      0x136 ./bin/uart2.o
                                0x31f (size before relaxing)
 .debug_str     0x00000855      0x1b4 ./bin/LCD.o
                                0x2ca (size before relaxing)
 .debug_str     0x00000a09       0x75 ./bin/klavesnica.o
                                0x1f3 (size before relaxing)
 .debug_str     0x00000a7e       0x88 ./bin/flashUtilities.o
                                0x1ea (size before relaxing)
 .debug_str     0x00000b06      0x129 ./bin/riadenie.o
                                0x411 (size before relaxing)
 .debug_str     0x00000c2f      0x289 ./bin/webcam.o
                                0x44d (size before relaxing)
 .debug_str     0x00000eb8       0xf4 ./bin/kom_modul.o
                                0x388 (size before relaxing)
 .debug_str     0x00000fac       0x33 ./bin/rfid_reader.o
                                0x2ef (size before relaxing)
 .debug_str     0x00000fdf       0x6e ./bin/ParTest.o
                                0x139 (size before relaxing)
 .debug_str     0x0000104d       0x81 ./bin/flash.o
                                0x1ee (size before relaxing)
 .debug_str     0x000010ce       0x73 ./bin/FreeRTOS_Tick_Setup.o
                                0x13e (size before relaxing)
 .debug_str     0x00001141       0xe3 ./bin/PollQ.o
                                0x20d (size before relaxing)
 .debug_str     0x00001224      0x15d ./bin/semtest.o
                                0x2b6 (size before relaxing)
 .debug_str     0x00001381      0x162 ./bin/GenQTest.o
                                0x2af (size before relaxing)
 .debug_str     0x000014e3       0xfa ./bin/QPeek.o
                                0x253 (size before relaxing)
 .debug_str     0x000015dd      0x372 ./bin/FEC.o
                                0x600 (size before relaxing)
 .debug_str     0x0000194f      0x146 ./bin/blocktim.o
                                0x252 (size before relaxing)
 .debug_str     0x00001a95      0x18a ./bin/recmutex.o
                                0x2aa (size before relaxing)
 .debug_str     0x00001c1f      0x166 ./bin/console_reader.o
                                0x59e (size before relaxing)
 .debug_str     0x00001d85       0xa5 ./bin/printf-stdarg.o
                                0x20e (size before relaxing)
 .debug_str     0x00001e2a       0xd7 ./bin/port.o
                                0x1c4 (size before relaxing)
 .debug_str     0x00001f01      0x137 ./bin/list.o
                                0x247 (size before relaxing)
 .debug_str     0x00002038      0x79a ./bin/tasks.o
                                0x9b7 (size before relaxing)
 .debug_str     0x000027d2      0x3b5 ./bin/queue.o
                                0x5d4 (size before relaxing)
 .debug_str     0x00002b87       0xb1 ./bin/heap_1.o
                                0x1b5 (size before relaxing)
 .debug_str     0x00002c38       0x75 ./bin/timer.o
                                0x14c (size before relaxing)
 .debug_str     0x00002cad      0x394 ./bin/uip.o
                                0x6f8 (size before relaxing)
 .debug_str     0x00003041      0x13d ./bin/uip_arp.o
                                0x45b (size before relaxing)
 .debug_str     0x0000317e       0x48 ./bin/uiplib.o
                                0x2a9 (size before relaxing)
 .debug_str     0x000031c6       0x53 ./bin/uip-split.o
                                0x357 (size before relaxing)
 .debug_str     0x00003219       0xe2 ./bin/psock.o
                                0x401 (size before relaxing)
 .debug_str     0x000032fb       0x5a ./bin/uIP_Task.o
                                0x3c6 (size before relaxing)
 .debug_str     0x00003355      0x1dd ./bin/httpd.o
                                0x583 (size before relaxing)
 .debug_str     0x00003532      0x16b ./bin/httpd-cgi.o
                                0x563 (size before relaxing)
 .debug_str     0x0000369d      0x1a1 ./bin/httpd-fs.o
                                0x447 (size before relaxing)
 .debug_str     0x0000383e       0xc5 ./bin/http-strings.o
                                0x25d (size before relaxing)

.debug_loc      0x00000000     0x2e00
 *(.debug_loc)
 .debug_loc     0x00000000      0x180 ./bin/main.o
 .debug_loc     0x00000180      0x1e0 ./bin/uart0.o
 .debug_loc     0x00000360      0x1e0 ./bin/uart1.o
 .debug_loc     0x00000540      0x1e0 ./bin/uart2.o
 .debug_loc     0x00000720      0x360 ./bin/LCD.o
 .debug_loc     0x00000a80       0x60 ./bin/klavesnica.o
 .debug_loc     0x00000ae0       0xa0 ./bin/flashUtilities.o
 .debug_loc     0x00000b80      0x180 ./bin/riadenie.o
 .debug_loc     0x00000d00      0x1e0 ./bin/webcam.o
 .debug_loc     0x00000ee0       0x80 ./bin/kom_modul.o
 .debug_loc     0x00000f60       0x40 ./bin/rfid_reader.o
 .debug_loc     0x00000fa0       0x80 ./bin/ParTest.o
 .debug_loc     0x00001020       0x40 ./bin/flash.o
 .debug_loc     0x00001060       0x40 ./bin/FreeRTOS_Tick_Setup.o
 .debug_loc     0x000010a0       0x80 ./bin/PollQ.o
 .debug_loc     0x00001120       0x60 ./bin/semtest.o
 .debug_loc     0x00001180       0xc0 ./bin/GenQTest.o
 .debug_loc     0x00001240       0xc0 ./bin/QPeek.o
 .debug_loc     0x00001300      0x320 ./bin/FEC.o
 .debug_loc     0x00001620       0x80 ./bin/blocktim.o
 .debug_loc     0x000016a0       0xa0 ./bin/recmutex.o
 .debug_loc     0x00001740      0x340 ./bin/console_reader.o
 .debug_loc     0x00001a80      0x120 ./bin/printf-stdarg.o
 .debug_loc     0x00001ba0       0xc0 ./bin/port.o
 .debug_loc     0x00001c60       0xa0 ./bin/list.o
 .debug_loc     0x00001d00      0x4c0 ./bin/tasks.o
 .debug_loc     0x000021c0      0x2a0 ./bin/queue.o
 .debug_loc     0x00002460       0x80 ./bin/heap_1.o
 .debug_loc     0x000024e0       0x80 ./bin/timer.o
 .debug_loc     0x00002560      0x220 ./bin/uip.o
 .debug_loc     0x00002780       0xc0 ./bin/uip_arp.o
 .debug_loc     0x00002840       0x20 ./bin/uiplib.o
 .debug_loc     0x00002860       0x20 ./bin/uip-split.o
 .debug_loc     0x00002880      0x180 ./bin/psock.o
 .debug_loc     0x00002a00       0x80 ./bin/uIP_Task.o
 .debug_loc     0x00002a80      0x160 ./bin/httpd.o
 .debug_loc     0x00002be0      0x1a0 ./bin/httpd-cgi.o
 .debug_loc     0x00002d80       0x80 ./bin/httpd-fs.o

.debug_macinfo  0x00000000   0xc3ac3b
 *(.debug_macinfo)
 .debug_macinfo
                0x00000000    0x75bca ./bin/main.o
 .debug_macinfo
                0x00075bca    0x71931 ./bin/uart0.o
 .debug_macinfo
                0x000e74fb    0x71931 ./bin/uart1.o
 .debug_macinfo
                0x00158e2c    0x71930 ./bin/uart2.o
 .debug_macinfo
                0x001ca75c    0x7369d ./bin/LCD.o
 .debug_macinfo
                0x0023ddf9    0x71b4d ./bin/klavesnica.o
 .debug_macinfo
                0x002af946    0x1e84f ./bin/flashUtilities.o
 .debug_macinfo
                0x002ce195    0x74e2c ./bin/riadenie.o
 .debug_macinfo
                0x00342fc1    0x74a41 ./bin/webcam.o
 .debug_macinfo
                0x003b7a02    0x757af ./bin/kom_modul.o
 .debug_macinfo
                0x0042d1b1    0x72d86 ./bin/rfid_reader.o
 .debug_macinfo
                0x0049ff37    0x1d351 ./bin/ParTest.o
 .debug_macinfo
                0x004bd288    0x7364a ./bin/flash.o
 .debug_macinfo
                0x005308d2    0x1d37b ./bin/FreeRTOS_Tick_Setup.o
 .debug_macinfo
                0x0054dc4d    0x1f626 ./bin/PollQ.o
 .debug_macinfo
                0x0056d273    0x1fb32 ./bin/semtest.o
 .debug_macinfo
                0x0058cda5    0x1fb3d ./bin/GenQTest.o
 .debug_macinfo
                0x005ac8e2    0x1fb4d ./bin/QPeek.o
 .debug_macinfo
                0x005cc42f    0x74508 ./bin/FEC.o
 .debug_macinfo
                0x00640937    0x1dab8 ./bin/blocktim.o
 .debug_macinfo
                0x0065e3ef    0x1e07f ./bin/recmutex.o
 .debug_macinfo
                0x0067c46e    0x750d8 ./bin/console_reader.o
 .debug_macinfo
                0x006f1546    0x71a6a ./bin/printf-stdarg.o
 .debug_macinfo
                0x00762fb0    0x1d368 ./bin/port.o
 .debug_macinfo
                0x00780318    0x1eab0 ./bin/list.o
 .debug_macinfo
                0x0079edc8    0x2063b ./bin/tasks.o
 .debug_macinfo
                0x007bf403    0x1f719 ./bin/queue.o
 .debug_macinfo
                0x007deb1c    0x1ee4d ./bin/heap_1.o
 .debug_macinfo
                0x007fd969    0x1cc34 ./bin/timer.o
 .debug_macinfo
                0x0081a59d    0x7593c ./bin/uip.o
 .debug_macinfo
                0x0088fed9    0x756d3 ./bin/uip_arp.o
 .debug_macinfo
                0x009055ac    0x73971 ./bin/uiplib.o
 .debug_macinfo
                0x00978f1d    0x76081 ./bin/uip-split.o
 .debug_macinfo
                0x009eef9e    0x76118 ./bin/psock.o
 .debug_macinfo
                0x00a650b6    0x7604a ./bin/uIP_Task.o
 .debug_macinfo
                0x00adb100    0x758fa ./bin/httpd.o
 .debug_macinfo
                0x00b509fa    0x758a8 ./bin/httpd-cgi.o
 .debug_macinfo
                0x00bc62a2    0x73c80 ./bin/httpd-fs.o
 .debug_macinfo
                0x00c39f22      0xd19 ./bin/http-strings.o

.debug_weaknames
 *(.debug_weaknames)

.debug_funcnames
 *(.debug_funcnames)

.debug_typenames
 *(.debug_typenames)

.debug_varnames
 *(.debug_varnames)
OUTPUT(./bin/RTOSDemo.elf elf32-m68k)

.debug_ranges   0x00000000      0xdf8
 .debug_ranges  0x00000000       0x70 ./bin/main.o
 .debug_ranges  0x00000070       0x88 ./bin/uart0.o
 .debug_ranges  0x000000f8       0x88 ./bin/uart1.o
 .debug_ranges  0x00000180       0x88 ./bin/uart2.o
 .debug_ranges  0x00000208       0xe8 ./bin/LCD.o
 .debug_ranges  0x000002f0       0x28 ./bin/klavesnica.o
 .debug_ranges  0x00000318       0x38 ./bin/flashUtilities.o
 .debug_ranges  0x00000350       0x70 ./bin/riadenie.o
 .debug_ranges  0x000003c0       0xa0 ./bin/webcam.o
 .debug_ranges  0x00000460       0x30 ./bin/kom_modul.o
 .debug_ranges  0x00000490       0x20 ./bin/rfid_reader.o
 .debug_ranges  0x000004b0       0x30 ./bin/ParTest.o
 .debug_ranges  0x000004e0       0x20 ./bin/flash.o
 .debug_ranges  0x00000500       0x20 ./bin/FreeRTOS_Tick_Setup.o
 .debug_ranges  0x00000520       0x30 ./bin/PollQ.o
 .debug_ranges  0x00000550       0x28 ./bin/semtest.o
 .debug_ranges  0x00000578       0x40 ./bin/GenQTest.o
 .debug_ranges  0x000005b8       0x40 ./bin/QPeek.o
 .debug_ranges  0x000005f8       0xd8 ./bin/FEC.o
 .debug_ranges  0x000006d0       0x30 ./bin/blocktim.o
 .debug_ranges  0x00000700       0x38 ./bin/recmutex.o
 .debug_ranges  0x00000738       0xe0 ./bin/console_reader.o
 .debug_ranges  0x00000818       0x58 ./bin/printf-stdarg.o
 .debug_ranges  0x00000870       0x40 ./bin/port.o
 .debug_ranges  0x000008b0       0x38 ./bin/list.o
 .debug_ranges  0x000008e8      0x140 ./bin/tasks.o
 .debug_ranges  0x00000a28       0xb8 ./bin/queue.o
 .debug_ranges  0x00000ae0       0x30 ./bin/heap_1.o
 .debug_ranges  0x00000b10       0x30 ./bin/timer.o
 .debug_ranges  0x00000b40       0x98 ./bin/uip.o
 .debug_ranges  0x00000bd8       0x40 ./bin/uip_arp.o
 .debug_ranges  0x00000c18       0x18 ./bin/uiplib.o
 .debug_ranges  0x00000c30       0x18 ./bin/uip-split.o
 .debug_ranges  0x00000c48       0x70 ./bin/psock.o
 .debug_ranges  0x00000cb8       0x30 ./bin/uIP_Task.o
 .debug_ranges  0x00000ce8       0x68 ./bin/httpd.o
 .debug_ranges  0x00000d50       0x78 ./bin/httpd-cgi.o
 .debug_ranges  0x00000dc8       0x30 ./bin/httpd-fs.o
